:020000040800F2
:10000000000002206D030108B1A60008B3A6000895
:10001000B5A60008B7A60008B9A6000800000000B1
:10002000000000000000000000000000BBA6000867
:10003000BDA6000800000000BFA60008C1A6000879
:10004000B1030108B1030108B1030108B1030108BC
:10005000B1030108B1030108B1030108B1030108AC
:10006000B1030108B1030108B1030108E567000805
:10007000B1030108B1030108B1030108B10301088C
:10008000B1030108B1030108B1030108B10301087C
:10009000B1030108B1030108B10301086DA900080B
:1000A000B1030108B1030108B1030108B10301085C
:1000B000BDA80008B1030108B1030108B10301089C
:1000C000B1030108B1030108B1030108B10301083C
:1000D000B1030108B103010881AA0008B1030108B6
:1000E000B1030108B1030108C5A60008B103010866
:1000F000B1030108B1030108B1030108B10301080C
:10010000B1030108B1030108B1030108B1030108FB
:10011000B1030108B1030108B1030108B1030108EB
:10012000B1030108B1030108B1030108B1030108DB
:10013000B1030108B1030108B1030108B1030108CB
:10014000B1030108B1030108B1030108F5A60008D5
:10015000B1030108B1030108B1030108B1030108AB
:10016000B1030108B1030108B1030108B10301089B
:10017000B1030108B1030108B1030108B10301088B
:08018000B1030108B1030108FD
:10018800CCAF050800000020FC0C0020000D00206A
:1001980004530020064B07481A68074B1A60074BA0
:1001A80000221A70064B01221A7001F012BA00BF21
:1001B800A83E0020700F0020AC440020903E002094
:1001C800483E002008B5034801F003FA024B00221C
:1001D8001A7008BD48130020483E002008B5054B9A
:1001E800012200201A7004F019FE0348BDE80840F7
:1001F80001F0EFB9C0440020EC1300202DE9F041D4
:10020800144C204602F069FF00201349134A02F0FB
:100218001BFD1349134A0746002002F015FD124939
:10022800124A0646002002F00FFDD22105463A4642
:1002380023460A2002F020FED22132462346FA2025
:1002480002F01AFE5A20D2212A462346BDE8F04180
:1002580002F012BE00120020D69E0508CD0100084B
:10026800DF9E0508E5010008E79E05089D010008D6
:1002780008B5054B012200201A7004F0CFFD034891
:10028800BDE8084001F0A5B9C0440020EC130020E7
:10029800044B054800221A70044B02221A7001F020
:1002A80098B900BF903E002000120020483E002070
:1002B80008B5034801F08DF9024B00221A7008BDF9
:1002C80048130020483E00202DE9F041144C2046F8
:1002D80002F003FF00201349134A02F0B5FC13494A
:1002E800134A0746002002F0AFFC1249124A06469C
:1002F800002002F0A9FCD22105463A4623460A20EE
:1003080002F0BAFDD221324623465A2002F0B4FD4B
:10031800AA20D2212A462346BDE8F04102F0ACBD0E
:10032800700F0020D69E0508B9020008F09E050847
:1003380099020008F99E050879020008014801F0B1
:1003480048B900BF1410002010B5094C204602F02F
:10035800C4FE00200749084A02F076FCD221024672
:1003680023464FF48270BDE8104002F085BD00BFFF
:1003780034150020029F05084503000810B5074CF6
:100388004FF6E071206801F0A3FF2068044901F0EE
:100398004DFFBDE8104003F0D9B800BF000D0020A4
:1003A800099F050810B5074C4FF6E071206801F069
:1003B8008FFF2068044901F039FFBDE8104003F0C1
:1003C800C5B800BF000D00201E9F050810B5074CDA
:1003D8004FF6E071206801F07BFF2068044901F0C6
:1003E80025FFBDE8104003F0B1B800BF000D0020A4
:1003F800339F050810B5074C4FF6E071206801F0EF
:1004080067FF2068044901F011FFBDE8104003F0C0
:100418009DB800BF000D0020489F050810B51E4C70
:10042800FFF7C0FF002004F0F9FC23790BB9FFF7B0
:10043800A5FF63790BB9FFF7C9FFA3790BB9FFF7DC
:10044800D9FF154B5A79E2B11A79D2B199790022BC
:100458001A715A7101B19A71104B0F4C1A7008F049
:1004680001FF20684FF6E07101F032FF20680C4967
:1004780001F0DCFE08F053F803F068F8094803F0CF
:10048800A9F8FFF78FFF002008F00AF80648BDE832
:10049800104001F09EB800BF000D0020483E00202B
:1004A8005D9F0508809698004813002008B5002035
:1004B80007F0F6FF0248BDE8084001F08AB800BF1F
:1004C8004813002010B586B04FF07E5302930023E6
:1004D800039308F0C2FD8DED000ACDED010A9DE8F9
:1004E800030006AB03E903009DED020ADDED030AF4
:1004F8009DED041ADDED051A08F061FD104C002091
:1005080084ED040AC4ED050A07F0DAFF20644FF60B
:10051800E07004F057FCB7206E215E22002304F03F
:100528006DFD084B1A68084B1A60084B02224FF001
:10053800804001211A7006B0BDE810400EF049B99C
:1005480040480020983E0020AC440020190E0020AE
:100558001FB508F082FD8DED000ACDED010A9DE87A
:100568000300104A02AB83E8030082E803004FF659
:10057800E07004F027FCFFF73DFFB7203C215E2226
:10058800002304F03BFD084B1A68084B1A60084B1F
:1005980001214FF08040197005B05DF804EB0EF0B2
:1005A80018B900BF40480020983E0020AC44002005
:1005B800190E002010B5224B2248234C86B0029316
:1005C8000023039303F006F808F047FD20460121B5
:1005D80084ED080AC4ED090A08F05FFD8DED000AF4
:1005E800CDED010A9DE8030006AB03E903009DED8C
:1005F800020ADDED030A9DED041ADDED051A08F087
:10060800DEFC4FF6E07084ED0C0AC4ED0D0A04F030
:10061800D9FBFFF7B3FEB720A0215E22002304F028
:10062800EDFC0A4B1A680A4B1A600A4B03224FF07A
:10063800804001211A7006B0BDE810400EF0C9B81C
:1006480000004842A086010040480020983E002053
:10065800AC440020190E00202DE9F04F434D444EC4
:1006680085B000244FF6FF78284602F036FD414653
:10067800224623463F480094019401F0EDFD0427EB
:10068800B060224623464FF6E0713B48009701943C
:1006980001F0E2FD23463060414622463748009784
:1006A800019401F0D9FD3649F060364A204602F03F
:1006B800CBFA3549354A0746204602F0C5FA34498F
:1006C800344A8046204602F0BFFA3349334A81460D
:1006D800204602F0B9FA3249324A8246204602F0F0
:1006E800B3FA3149314A84462046CDF80CC002F0AD
:1006F800ABFA21468346B2682B46204602F0BCFB83
:10070800214632682B467D2002F0B6FB2321F26891
:100718002B46B42002F0B0FB9B213A462B46FA2028
:1007280002F0AAFB372142462B46FA2002F0A4FB2E
:1007380069214A462B46FA2002F09EFBC821524600
:100748002B466E2002F098FBC8215A462B46AA2059
:1007580002F092FBDDF80CC0F0206246C8212B465F
:1007680005B0BDE8F04F02F087BB00BFA41200201F
:10077800000D0020719F0508799F05088C9F0508CA
:10078800949F0508BD0500089C9F050859050008A9
:10079800A49F0508CD040008AC9F0508610B00085C
:1007A800B39F0508B5040008BA9F0508250400088A
:1007B8001FB5134802F00EFF08F04FFC8DED000A3C
:1007C800CDED010A9DE803000E4A02AB83E8030061
:1007D80082E803004FF6E07004F0F4FAFFF70AFE2F
:1007E8005E220023DF203C2104F008FC064B012296
:1007F8001A71064B1A68064B1A6005B000BD00BF97
:10080800A086010048480020000D0020A83E0020D6
:10081800AC44002010B586B04FF07E5302930023FD
:10082800039308F01AFC8DED000ACDED010A9DE84E
:10083800030006AB03E903009DED020ADDED030AA0
:100848009DED041ADDED051A08F0B9FB0E4C0020E9
:1008580084ED060AC4ED070A07F03EFE60644FF611
:10086800E07004F0AFFADF206E215E22002304F06E
:10087800C5FB064B01229A71FFF7A8FD044B1A68C5
:10088800044B1A6006B010BD40480020000D00203F
:10089800A83E0020AC44002008B5FFF76FFDBDE876
:1008A800084002F053BE70B52DED028B9FED238AF0
:1008B80088B00A26F0EE488A03E0B0EE608AF0EECF
:1008C800418A08F0CAFB8DED000ACDED010A9DE8CA
:1008D800030004AB83E80300F0EE680AB0EE480AB0
:1008E8009DED041ADDED051A8DED028ACDED038A22
:1008F80008F04AFBCDED010A8DED000A9DE80300E2
:1009080002AD85E80300013E6C46DDED020A9DED6F
:10091800031AD2D19FED0A0A08F096FB8DED000A62
:10092800CDED010A9DE8030085E80300DDED030A2B
:100938009DED020A08B0BDEC028B70BD00000000FE
:10094800CDCCCC3D2DE9F74F564D574CDFF864918F
:10095800DFF864814FF6E07004F034FA28680EF08E
:1009680089FE064668680F460EF084FE3246CDE9D9
:1009780000013B464946204613F0D4FB224600239B
:100988000520372104F058FB2869484F484E0EF0DF
:1009980071FE824668698B460EF06CFE5246CDE9C0
:1009A80000015B463946204613F0BCFB2246002373
:1009B8000520692104F040FB286B0EF05BFE82469F
:1009C800686B8B460EF056FE5246CDE900015B4639
:1009D8004146204613F0A6FB002305209B21224612
:1009E80004F02AFB31462A6C204613F09BFB224672
:1009F80000239B21A22004F01FFB4FF4FC6004F0AD
:100A0800E1F9A8680EF036FE8246E8688B460EF0DB
:100A180031FE5246CDE900015B464946204613F0B7
:100A280081FB224605205021002304F005FBA8691C
:100A38000EF020FE8246E8698B460EF01BFE5246F9
:100A4800CDE900015B463946204613F06BFB224690
:100A580000230520822104F0EFFAA86B0EF00AFEAD
:100A68008246E86B8B460EF005FE5246CDE9000142
:100A78005B464146204613F055FB00230520B42170
:100A8800224604F0D9FA31466A6C204613F04AFB34
:100A9800A220B4212246002303B0BDE8F04F04F0A1
:100AA800CBBA00BF40480020100D0020D39F050896
:100AB800F69F0508C19F0508E59F050810B5204B5E
:100AC8002048214C86B002930023039302F082FD54
:100AD80008F0C3FA2046022184ED0A0AC4ED0B0A85
:100AE80008F0DBFA8DED000ACDED010A9DE8030060
:100AF80006AB03E903009DED020ADDED030A9DED57
:100B0800041ADDED051A08F05AFA4FF6E07084ED84
:100B18000E0AC4ED0F0A04F055F9DF20A0215E2269
:100B2800002304F06BFAFFF73DFC084B01225A71D1
:100B3800FFF708FF064B1A68064B1A6006B010BD8F
:100B480000004842A086010040480020000D002017
:100B5800A83E0020AC44002008B5FFF723FCBDE800
:100B68000840EFE6002008B504F058F9074A0023CA
:100B78001370074A1370074B1B78022B0CBF0648EB
:100B88000648BDE8084000F024BD00BF903E0020A4
:100B9800C0440020483E002000120020700F0020B2
:100BA8002DE9F14F2D4C204602F097FA00202C49F0
:100BB8002C4A02F049F82C492C4A8146002002F0C0
:100BC80043F82B492B4A0746002002F03DF82A49F2
:100BD8002A4A0646002002F037F82949294A0546DC
:100BE800002002F031F82849284A8046002002F007
:100BF8002BF82749274A8246002002F025F8D221FF
:100C080083464A462346E62002F036F928203A462B
:100C18002346014602F030F9462132462346282071
:100C280002F02AF964212A462346282002F024F9F2
:100C3800822142462346282002F01EF952462346C6
:100C48002820A02102F018F928205A46BE21234660
:100C580001B0BDE8F04F02F00FB900BFEC1300205F
:100C6800FB9F05086D0B000804A005088911000802
:100C78000FA005086511000819A005084111000812
:100C880024A005081D1100082FA00508F910000868
:100C980039A00508D5100008023810B5052800F25B
:100CA800CE81DFE810F006000A005F00C90081016C
:100CB8001701BDE8104007F09FBC00204FF6E07117
:100CC80007F0A0FD63204FF6E07107F09BFDB3200D
:100CD8004FF4F06107F096FDC7204FF6E07107F07A
:100CE80091FD4FF6FF7004F06DF8DC2100237D20A4
:100CF800D34A04F0A1F94EF29C7004F063F8052081
:100D080001210023CF4A04F097F90520522100233E
:100D1800CD4A04F091F9B62100230520CB4A04F00E
:100D28008BF94FF4F06004F04DF80121002340F2F4
:100D38001310C44A04F080F9002340F21310522122
:100D4800C24A04F079F9B621C14A40F213100023CF
:100D580004F072F94EF29C7004F034F80520A221D8
:100D6800BC4A67E100204FF6E07107F04BFD3120E7
:100D78004FF6E07107F046FD63204FF6E07107F08B
:100D880041FD95204FF6E07107F03CFDC7204FF676
:100D9800E07107F037FD4EF29C7004F013F805205F
:100DA80001210023AC4A04F047F905202021002343
:100DB800AA4A04F041F9052052210023A84A04F068
:100DC8003BF9052084210023A64A04F035F9B62111
:100DD80005209E4A002304F02FF94FF4F06003F039
:100DE800F1FF012140F2131000239B4A04F024F97B
:100DF80040F2131020219C4A002304F01DF940F210
:100E080013105221914A002304F016F940F21310EE
:100E18008421964A002304F00FF9B621944A40F23F
:100E28001310002304F008F94FF6FF7003F0CAFF0F
:100E38007D20DC218F4AFDE000204FF6E07107F0AD
:100E4800E1FC27204FF6E07107F0DCFC4F204FF65D
:100E5800E07107F0D7FC77204FF6E07107F0D2FC7D
:100E68009F204FF6E07107F0CDFCC7204FF6E071E8
:100E780007F0C8FC4EF29C7003F0A4FF0520012186
:100E88000023724A04F0D8F80520162100237A4A74
:100E980004F0D2F805203E210023784A04F0CCF86B
:100EA800052066210023764A04F0C6F88E21002327
:100EB8000520744A04F0C0F80520734AB6210023BF
:100EC80004F0BAF84FF6FF7003F07CFF7D20DC21B8
:100ED8006E4AAFE000204FF6E07107F093FC312036
:100EE8004FF6E07107F08EFC63204FF6E07107F0D3
:100EF80089FC95204FF6E07107F084FCC7204FF677
:100F0800E07107F07FFC4EF29C7003F05BFF052058
:100F1800012100235E4A04F08FF8052020210023D8
:100F28005C4A04F089F80520522100235A4A04F04B
:100F380083F8052084210023584A04F07DF8B6215F
:100F48000520424A002304F077F84FF4F06003F0DC
:100F580039FF012140F213100023514A04F06CF8C4
:100F680040F2131020214F4A002304F065F840F2A4
:100F780013105221354A002304F05EF840F2131092
:100F88008421494A002304F057F8B621474A40F221
:100F98001310002304F050F84FF6FF7003F012FF0F
:100FA8007D20DC21424A45E000204FF6E07107F041
:100FB80029FC31204FF6E07107F024FC63204FF63E
:100FC800E07107F01FFC95204FF6E07107F01AFC5E
:100FD800C7204FF4FC6107F015FC4EF29C7003F03B
:100FE800F1FE052001210023324A04F025F80520EE
:100FF80020210023304A04F01FF805205221002345
:101008002E4A04F019F88421002305202C4A04F004
:1010180013F84FF4F06003F0D5FEB6210520294AF5
:10102800002304F009F84FF6FF7003F0CBFE264AC0
:101038008720DC210023BDE8104003F0FDBF10BD70
:101048000FA0050843A005083EA00508FAA4050856
:1010580042A0050870A005085CA0050847A005087F
:1010680057A005084CA0050851A0050856A005087A
:101078005BA0050819A005085FA0050863A005087E
:1010880067A005086BA005086FA0050873A00508F0
:101098007FA0050883A0050887A005088AA0050881
:1010A80093A005088FA005088EA0050892A0050842
:1010B80097A00508A2A0050868A0050860A0050873
:1010C800A6A0050811A6050839A0050810B5064C04
:1010D80006480623237000F07CFA2078FFF7DCFD31
:1010E800BDE8104007F020BFC04400207C16002057
:1010F80010B5064C06480723237000F06AFA2078DA
:10110800FFF7CAFDBDE8104007F00EBFC04400203D
:101118007C16002010B5064C06480523237000F005
:1011280058FA2078FFF7B8FDBDE8104007F0FCBE7C
:10113800C04400207C16002010B5064C0648042345
:10114800237000F046FA2078FFF7A6FDBDE81040AE
:1011580007F0EABEC04400207C16002010B5064CFB
:1011680006480323237000F034FA2078FFF794FD33
:10117800BDE8104007F0D8BEC04400207C1600200F
:1011880010B5064C06480223237000F022FA207896
:10119800FFF782FDBDE8104007F0C6BEC04400203E
:1011A8007C1600200F4A012310B513700E4A002444
:1011B80014700E4A2046137007F072F9204603F0A7
:1011C8002DFE0B4B04221A7007F0FAFD07F098FE6B
:1011D800084B09481C70094B1C70BDE8104000F012
:1011E800F8B900BFC0440020100E00200D0E0020EA
:1011F800483E002044460020B8100020903E0020C1
:101208000F4A38B5012313700E4A002414700E4A91
:101218002046137007F044F9204603F0FFFD0B4BFE
:1012280002251D7007F0CCFD07F06AFE084B09483F
:101238001D70094B1C70BDE8384000F0CAB900BFEA
:10124800180E0020100E0020C0440020483E002048
:1012580044460020EC130020903E0020034B01225E
:101268004FF4FC601A7003F0ADBD00BF100E0020F3
:101278000B4B10B5002420461C7003F0CFFD07F07F
:1012880025FB06F037FE074B1C70074B01221A702E
:1012980007F016FB0548BDE8104000F09AB900BFFA
:1012A800100E0020C0440020483E0020700F00208F
:1012B8000A4B10B5002420461C7003F0AFFD07F060
:1012C80005FB074B1C70074B02221A7007F0F8FA4F
:1012D8000548BDE8104000F07CB900BF100E0020A2
:1012E800C0440020483E00200012002008B5074BEB
:1012F8000020187003F092FD054B064803221A706F
:1013080000F067F9BDE80840FFF7C6BA100E0020E4
:10131800483E0020A41200200C4B10B500220C4CB3
:101328001A7007F0D3FA04F013FD07F0FEF807F07F
:10133800C7FA20684FF6E07100F0CAFF2068054937
:1013480000F074FFBDE8104002F000B9100E002054
:101358002C0D0020A8A005080E4B002210B51A700D
:101368000088C83880B2042805D90B480B4A0C4BB2
:10137800912102F013FB0B4CC0B204F073FD2068FE
:101388004FF6E07100F0A4FF20680749BDE810405F
:1013980000F04CBF100E0020BCA00508F4DF0308C5
:1013A800DCA005082C0D00200DA105082DE9F04F43
:1013B8006448654D89B0002401F08FFE4FF6FF7137
:1013C8002246234661480094019400F045FF042614
:1013D80007464FF6E071224623465D480096019481
:1013E80000F03AFF4FF6E0718046224623465948FE
:1013F8000096019400F030FF4FF6FF7181462246B7
:10140800234655480096019400F026FF234628609D
:101418004FF6FF71224651480096019400F01CFFD8
:101428004F4968604F4A204601F00EFC4E494F4A2A
:101438008246204601F008FC4D494E4A8346204624
:1014480001F002FC4C4903904C4A204601F0FCFB99
:101458004B4904904B4A204601F0F6FB4A49059057
:101468004A4A204601F0F0FB49490690494A20467D
:1014780001F0EAFB3A4607902146324B204601F03C
:10148800FBFC214642462F4BC82001F0F5FC0A21FF
:101498004A462C4BC82001F0EFFC2A68294B5521FD
:1014A800782001F0E9FC6A68264B7820692101F070
:1014B800E3FCC82505262327E0B204F003FC364ADE
:1014C8000146284601F0C0FB94FBF6F106FB1141EA
:1014D80079431E31024689B200201A4B0134013586
:1014E80001F0CAFC042CADB2E6D1D2215246052047
:1014F800144B01F0C1FCD2215A464C20114B01F08B
:10150800BBFCD221039A0F4B9C2001F0B5FCD221E1
:10151800049A0C4BEC2001F0AFFCB421059A094B5E
:10152800EC2001F0A9FCB421069A064B9C2001F09E
:10153800A3FC079A034B4C20B42109B0BDE8F04F37
:1015480001F09ABC481300202C0D00201DA10508AD
:1015580027A1050834A105083FA105081F9F050814
:1015680053A10508211300085BA10508F51200081E
:1015780064A10508B91200086DA1050879120008D0
:1015880076A10508651200087FA105080912000860
:1015980088A10508AD1100086113000808B500F01E
:1015A8004FFBFEF72BFE00F083F8FFF755F8FEF728
:1015B8008BFEFFF7F5FA00F01BFDFFF7F7FEFEF7CD
:1015C800C3FE00F0F3FB00F047FABDE8084000F066
:1015D80015BB10B5044628B90F48104A104B4921CD
:1015E80002F0DCF90F4B1868844213D010B1C369BC
:1015F80000219847002003F011FC002003F0F8FBBD
:101608004FF6FF7003F0DEFBE3692046012198479F
:10161800044B1C6010BD00BF91A1050803E003083E
:10162800ADA10508340D00200048D2E7481300207A
:1016380008B5124B124A1B780D2B8CBF00210121D3
:10164800117014225A430F4988588B184FF47A7234
:101658000D495043086059684A430C490A609A6822
:101668000B4B1A6006F0DAFE07F02AF9094B0A4814
:1016780000221A70BDE80840FFF7ABBFAE3E00205D
:101688002C0F002000000020B03E0020CC44002099
:10169800A4440020483E002048130020024B034881
:1016A80000221A70FFF795BF483E0020481300201B
:1016B8002DE9F347384DDFF8FC80384E00242846E2
:1016C80001F00BFD2246234647F6FF71344800948B
:1016D800019400F0C1FD4FF6FF7904278246494680
:1016E8002246234640460097019400F0B5FD49463E
:1016F80030602246234640460097019400F0ACFD36
:10170800494670602246234640460097019400F0FF
:10171800A3FD2346B06049462246404600970194FF
:1017280000F09AFD1F49F0601F4A204601F08CFA2C
:101738001E491F4A0746204601F086FA2146804680
:1017480052462B46204601F097FB3C2132682B4637
:101758005A2001F091FB5A2072682B46014601F08D
:101768008BFB7821B2682B465A2001F085FB962125
:10177800F2682B465A2001F07FFBD2213A462B46CD
:10178800EC2001F079FB9C20D22142462B4602B086
:10179800BDE8F04701F070BBB8100020380D0020FC
:1017A800BDA10508CAA10508A5160008D3A105080A
:1017B800391600081F9F050870B5474E474C327808
:1017C80047492DED028B142592B005FB02420C32DD
:1017D8000FA812F0A7FC33780D2B05FB03F504EBDB
:1017E800050332D8D3ED016A9B6807EE103A6359B6
:1017F800B8EEE68A06EE903ADFED3A7AF8EEC78A56
:10180800B8EEE67A88EE278AC8EEA78AC7EE277A66
:1018180017EE900A0DF02EFF02460B466846324935
:1018280012F080FC18EE100A0DF024FF02460B4659
:1018380005A82E4912F076FC18EE900A0DF01AFF52
:1018480002460B460AA82A4929E093ED017A9B68CB
:1018580007EE903A635906EE903AF8EEE78AF8EE0A
:10186800E67AB8EEC78A17EE900A0DF003FF024633
:101878000B4668461F4912F055FC18EE100A0DF089
:10188800F9FE02460B4605A81B4912F04BFC18EE60
:10189800900A0DF0EFFE0B46184902460AA8184CAC
:1018A80012F040FC2068174900F0C0FC20680FA91E
:1018B80000F0BCFC6068694600F0B8FCA06805A9A7
:1018C80000F0B4FCE0680AA900F0B0FC01F03EFEAC
:1018D80012B0BDEC028B70BDAE3E002000000020AF
:1018E800DCA1050800007A44E7A10508F8A105086D
:1018F80009A205081AA205082BA205083CA205089A
:10190800380D0020289F05084FF6FF7070474FF6E6
:10191800FF7070471FB5002947D04FF2DE7003F003
:101928007DFA002003F050FB0F2003F04BFA1F4C08
:101938001F4A412101230A2003F07EFB042003F003
:1019480043FB236828209621042B24DC0123194A11
:1019580003F072FB03A90DF10E02206803F0F4FDF9
:101968000F2003F02FFABDF80C00BDF80E10143844
:101978000F242822002380B2009403F053FABDF804
:101988000E10BDF80C000094143989B228220123E6
:1019980003F048FA09E0084A012303F04DFB1E2032
:1019A800A521064A012303F047FB1FBD480D00206F
:1019B8004DA2050860A205087CA2050892A20508A8
:1019C80037B51E4C2368042B05462BDC01A80DF106
:1019D800060103F0B7FDBDF80630BDF8042018492C
:1019E80004200AF0FBFE2368002B04DA1548164A87
:1019F800164B592105E0042B05DD1248124A144BF9
:101A08005A2101F0CBFF04EB8302BDF80410013327
:101A18009180BDF806102360052BD18008D1201DC8
:101A280003F012FE00230B482360FFF7D2FD03E00A
:101A380028460121FFF76EFF3EBD00BF480D00207C
:101A4800A9A20508EEA2050815E0030810A30508D9
:101A580027A305089014002037B50B4C204601F049
:101A68003CFB0A4B0A49009300250120094A0A4B0E
:101A7800019501F0DAF9294602462346284603B0C3
:101A8800BDE8304001F0F8B95C1100201D190008CC
:101A98001119000817190008C91900084FF6FF7036
:101AA80070474FF6FF70704730B54FF6E07087B05B
:101AB80003F0B4F9002003F087FA0F2003F082F94D
:101AC80000212C4A2C4C01230A2003F0B5FA0020EF
:101AD80003F078F9042003F077FA0A201921274A3D
:101AE800012303F0A9FA2521254A01230A2003F03E
:101AF800A3FA1F2003F066F901230A203721214A9F
:101B080003F09AFA2378002B31D001231E20962166
:101B18001D4A03F091FA62881C4902A812F002FBE0
:101B280001231E20A22102AA03F086FAA2881849DE
:101B380002A812F0F7FAAE2102AA01231E2003F030
:101B48007BFA0F2003F03EF96088A188143880B230
:101B58000F2528220023009503F064F9A1886088E6
:101B68000095143989B22822012303F05BF907B0E4
:101B780030BD00BF55A30508600D002067A3050808
:101B880087A30508A7A30508CAA30508DCA30508B9
:101B9800E9A3050801B187E7704713B50DF1060100
:101BA80001A803F083FC144B01221A705988BDF870
:101BB8000420891A0E311C2919460AD89C88BDF8B8
:101BC8000600201A0E301C2803D899680131996044
:101BD80001E000238B60084B9968012905DD00228C
:101BE8009A601A70FFF720FD05E05A80BDF80620BC
:101BF8009A80FFF759FF1CBD600D002037B50B4CCC
:101C0800204601F06AFA0A4B0A4900930025012090
:101C1800094A0A4B019501F008F92946024623466C
:101C2800284603B0BDE8304001F026B990140020E2
:101C38009D1B0008A51A0008AB1A0008A31B000882
:101C480010B50B4C204601F048FA00200146224608
:101C580000F062FB00200749074A00F0F5FFD22197
:101C6800024623464FF48270BDE8104001F004B9E3
:101C78007C160020F6A30508A91C000870B5C92425
:101C88000AE0A8B200223146013502F025FAF02D0B
:101C9800F7D10134EF2C02D00025A6B2F1E770BDD0
:101CA80008B5FFF7EBFF044B044800221A70BDE8A3
:101CB8000840FFF78EBC00BF180E0020141000204B
:101CC80010B5064C4FF6FF71206800F001FB044B7D
:101CD80020681968BDE8104000F0A8BA6C0D002013
:101CE800EC02002008B5FFF7EBFF0020014606F0E4
:101CF800B7FABDE8084001F029BC08B5002003F098
:101D08008DF8054B1868054B196800F08FFA0448E0
:101D1800BDE80840FFF75DBC6C0D0020E80200201C
:101D2800481300200088A0F5C87080B2092808B5BB
:101D380005D90848084A094B902101F02FFE084BA5
:101D48001880084BFF21197006F08AFABDE8084090
:101D5800B6E700BFFBA3050827E003081EA4050893
:101D680020170020221700200088A0F5967080B266
:101D7800092808B505D90848084A094B842101F003
:101D88000DFE084B1880084B0121197006F068FAFF
:101D9800BDE8084094E700BFFBA305083CE0030842
:101DA8001EA405082017002022170020F7B50024DC
:101DB8003648374D01F091F9224623464FF6FF7118
:101DC80034480094019400F047FA0426224623463A
:101DD80007464FF6FF7130480096019400F03CFA30
:101DE8002346286022464FF6FF712B48009601943F
:101DF80000F032FA29496860294A204600F024FF99
:101E080020462849284A00F01FFF214606463A4640
:101E180020461E4B01F030F82A681C4B204628212A
:101E280001F02AF83246AA20D221184B01F024F8F2
:101E38000F254FF4967440F2351620461B491C4A6C
:101E480000F002FF01340246782128460F4BA4B265
:101E5800233501F011F8B442ADB2EED10F254FF49D
:101E6800C87440F2991620461249134A00F0ECFE55
:101E7800013402469B212846044BA4B2233500F0C6
:101E8800FBFFB442ADB2EED1FEBD00BFD8150020B5
:101E98006C0D00204FA40508309F05085BA40508B9
:101EA800ED1C000864A40508031D00086DA40508BE
:101EB800711D00086FA405082D1D000808B5FFF75F
:101EC800FFFE0020014606F0CBF9BDE8084001F00E
:101ED8003DBB00BF10B506F07BFF1A4B1A4A002421
:101EE8001C701A4B02201C70CA21234603F0A4F868
:101EF800204606F0D5FA164B1C80164B1C70164B64
:101F08001B78023B052B1CD8DFE803F003070B13F3
:101F1800170FBDE81040FFF733B9BDE81040FFF7D1
:101F28001DB9BDE81040FFF707B9BDE81040FFF73D
:101F3800DFB8BDE81040FFF7EDB8BDE81040FFF787
:101F4800C5B810BD180E00201E9F0508903E002041
:101F58002445002044460020C044002008B5084B12
:101F680001221A70074B1A68074B00201A6002F00A
:101F780055FF06F025FF0548BDE80840FFF729BBD7
:101F8800180E0020A83E0020AC440020EC130020CE
:101F980038B50E4B0E4D00241C700E4B1C700E4BAA
:101FA8001C700E4B1A680E4B20461A6002F036FF62
:101FB8000C4B1B78022B0CBF0B480C48FFF709FB96
:101FC8002C70BDE8384006F0FBBE00BF180E00209C
:101FD80044460020C0440020903E0020A83E002037
:101FE800AC440020483E002000120020700F002062
:101FF8002DE9F041144C204601F06FF800201349F8
:10200800134A00F021FE1349134A0746002000F046
:102018001BFE1249124A0646002000F015FED22186
:1020280005463A462346E62000F026FF4B21324675
:102038002346642000F020FF642069212A462346B5
:10204800BDE8F04100F018BF14100020FB9F050800
:10205800991F000871A40508651F00087DA40508DC
:10206800DD1E000808B508B143682BB90348044AC7
:10207800044B9B2101F092FC586908BD8AA405080D
:1020880050E00308ACA4050808B5FFF7EBFF80682B
:10209800123080B208BD08B5FFF7E4FF406806308B
:1020A80080B208BD2DE9F84F04468846FFF7DAFFED
:1020B8006689E589074606F1030905F10F0AB8F1B3
:1020C800000F1FD01F2002F07DFE2046FFF7DCFF27
:1020D80083462046FFF7DFFF294603465FFA8BF267
:1020E800F0B202F0AFFE042002F06EFF0B364FF69E
:1020F800FF70033502F066FEB0B2A9B23A68012358
:1021080002F09AFF3D69204641464A465346A84791
:10211800BDE8F88F13B504460DF1060101A803F0D8
:10212800C5F92046FFF79EFF6389BDF80410BDF886
:102138000620C91AE389D21A0339C3680F3A204620
:1021480098471CBDF7B5044614200D4616461F4691
:1021580011F076FC089BC7600361064B0649074AE5
:1021680080E8700000930190054B002000F05DFEB0
:10217800FEBD00BFAD2000089F2000089120000888
:102188001D210008704708B508B143682BB90448F9
:10219800044A054BAD2101F001FC586908BD00BF98
:1021A800CBA4050868E00308ACA40508F8B5054603
:1021B8000E46FFF7E8FF836B04461BB128463146FD
:1021C800984700E018466F8994F83C30ED890EB9BD
:1021D800034310D0208E02F0F5FD608E02F008FE59
:1021E80094F8350002F0F0FE94F834303846294669
:1021F800224602F021FF002384F83C30F8BD08B5E0
:10220800FFF7C1FF90F83500BDE8084002F0F1BEC5
:1022180038B5FFF7B8FF044612F00AF8054694F8F7
:10222800350002F0E1FE684380B238BD38B50D468E
:10223800FFF7A9FF29462E22044612F029F850B1CB
:10224800204629462E2212F075F8002384F82E30F5
:10225800012384F83C3038BD2DE9F7430746402078
:102268000E461546984611F0EBFB044628B911486E
:10227800114A124B4E2101F091FB114B114A1249A0
:102288008DE818000020114B00F0CFFD394681463B
:10229800FFF7CCFF9DF82830268684F835300B9B55
:1022A8006586A363002384F8348084F83C3048466C
:1022B800BDE8FE83CBA4050880E00308E9A405086F
:1022C800B521000807220008192200088D210008FE
:1022D80010B50C46FFF757FF0123048680F83C3001
:1022E80010BD00BF4FF4A0707047C82070477047FA
:1022F800074B1B78022B07B508D1064B1B78022B1E
:1023080004D001A80DF1060103F0D0F80EBD00BFFE
:1023180044460020C044002073B50A4B06460D46CB
:102328001446009300200849084A094B019000F020
:102338007CFD294602462346304602B0BDE870407F
:1023480000F09ABDF7220008ED220008F3220008E9
:10235800F922000813B502AB03E90600436843B14C
:10236800027C0124082A9C7004D11B6921469847E5
:1023780000E01C4620461CBD30B500282BD0058B3C
:10238800002425E0036A1A7C012A05D15B681A88B3
:102398008A421BD1187F30BD052A06D15B681A888E
:1023A8008A4213D193F82C0030BD032A06D15B680A
:1023B8001A888A420AD193F8250030BD062A05D129
:1023C8005B681A888A4201D1D87A30BD013404305A
:1023D800AC42D7D3002030BD08B1817501207047C9
:1023E800F8B504460D46D0B1E175D0F89830984755
:1023F800012D0DD12746002606E0F86900F10802F4
:10240800436906CA98470136238B04379E42F4D3A2
:10241800D4F898302046294698470120F8BDF8BDE1
:10242800F8B50546084617460E4611F001FF013F6C
:10243800B84234BF04463C463CB1284631462246A1
:1024480011F078FF00232B55F8BD2C70F8BDF7B5B7
:10245800044600200090019000296CD00E8B68E0A3
:1024680000F1080351F823301D7C042D04D15D6868
:102478002D88954247D0013000F1080351F82330E8
:102488001D7C012D04D15D682D8895423BD001301B
:1024980000F1080351F823301D7C052D04D15D6837
:1024A8002D8895422FD0013000F1080351F82330D0
:1024B8001D7C032D04D15D682D88954223D0013001
:1024C80000F1080351F823301D7C022D04D15D680A
:1024D8002D88954217D0013000F1080351F82330B8
:1024E8001D7C072D04D15D682D8A95420BD00130E3
:1024F80000F1080351F823301D7C062D08D15D68D2
:102508002D88954203D103F10801204615E00130DA
:1025180000F1080351F823502B7C082B09D16F6870
:102528003F88974204D105F1080120461A4605E084
:102538000130B04294D320466946082211F030FD9C
:102548002046FEBDF8B505460F461646002830D091
:102558004388032B2FD0202011F072FA044600285C
:102568002BD040F80C5B39460C22FFF759FF182096
:10257800E66111F065FA0646B8B102230374012337
:1025880063760F4B446063600E4BA3600023237691
:102598006B8805EB830201339BB2012B50606B8083
:1025A8000CD16A685268137608E0204611F050FA98
:1025B80004E0064602E0002600E006463046F8BD84
:1025C800CC5F04086A5C040837B5456802AB03E9C8
:1025D80006003DB3037C0124042B85F8314022D149
:1025E800688E02F0EFFB95F8300002F0EDFC95F8EC
:1025F800343043B9BDF80200BDF80610AA1C2346C2
:1026080002F01AFD0FE0012B03D1084840F23951BE
:1026180004E0022B07D1054840F24151044A054B1A
:1026280001F0BCF92C4620463EBD00BFFCA40508BD
:10263800402B0408FAA40508F8B504460F461646C8
:1026480010B3838A0A2B20D0202011F0F9F905460F
:10265800E8B14460102200F108003946FFF7E0FEB7
:102668004FF6FF73A08A2B801F236B8000232B76E5
:10267800831D013080B20128EE6144F82350A08206
:1026880007D1A3691876F8BDF8BD0020F8BD012070
:10269800F8BD0120F8BD2DE9F3471D464B1C9842B3
:1026A80082460C461746BDF828600DDD95420BDCC6
:1026B80001320AF101035B1A521BC8B2D2B29BB2B3
:1026C8002946009602F0B6FBAAF1020A3046C4EB8E
:1026D8000A0A02F077FB4FF000084FF001091FFAD1
:1026E8008AFA0BE0601C08EB050180B289B25246F9
:1026F8000023009602F096FB09F101097B1B08F103
:10270800010899451FFA88F8ECD3BDE8FC87F8B5AD
:10271800C7B2144638461E460D4602F095FB621EA7
:1027280092B23846294602F08FFB304602F04AFB47
:10273800022606E0A21B92B23846294602F084FB24
:102748000136A642F6D3F8BD73B504460E4600F12D
:102758001E001546009200233C2280B21E3E02F065
:1027680061FBB1B220463C220123009502F05AFBDE
:102778007CBD73B504460E46013815460092002309
:10278800032280B2013E02F04DFBB1B22046032283
:102798000123009502F046FB7CBDF7B5089D2E7B12
:1027A800EF7A1C463604AB7A06EB0726F618431A6E
:1027B800687B06EB00602D1800200190121B08466C
:1027C8002146009501F026FFFEBD30B5456885B06D
:1027D80004AB03E906007DB101242C736D68BDF8D4
:1027E8000800BDF80A109DF80C209DF80E300095E1
:1027F800FFF7D3FF204600E0284605B030BD2DE99D
:10280800F04385B004AB03E906004468BDF80860EE
:10281800BDF80C70002C41D0012384F8263094F8C0
:1028280025300BB9A26800E06268FFB2BDF80A1053
:102838009DF80E30009230463A46FFF7AEFF04F19D
:102848000C08022002F0C0FB404611F0F1FC0546DE
:1028580000B1451E0F3F0024153E1FFA87F90DE011
:1028680002F0BCFB02F0C0FB04FB106189B24846D1
:102878002022002302F0FAFB0134E4B2AC42EFD389
:10288800002002F09FFAB8B2B1B24246012302F02A
:10289800EDFB002002F098FB012000E0204605B087
:1028A800BDE8F0832DE9F04385B004AB03E90600E9
:1028B8004568BDF80860BDF80C70002D3CD00123B8
:1028C8006B762B7EBDF80A10012B0CBF6A68AA68CC
:1028D8009DF80E300092FFB23A463046FFF75DFF92
:1028E8000C35022002F070FB284611F0A1FC0E3FC7
:1028F80081460024163E1FFA87F80DE002F06EFBB1
:1029080002F072FB04FB106189B2404620220023CA
:1029180002F0ACFB0134E4B24C45EFD9002002F0E0
:1029280051FAB8B2B1B22A46012302F09FFB002047
:1029380002F04AFB012000E0284605B0BDE8F0831C
:102948002DE9F04F85B00546DDF8409002914846E4
:102958009046039311F06CFCDDF838A0DDF83CB02C
:102968000646294600242F4611E024B1B4420CBF84
:102978005B46534600E0039B01F10805ADB20093A6
:102988002846029A4346FFF708FF01342946B44215
:10299800EBDD002002F016FA022002F015FB7D1D87
:1029A80008F10508A8B21FFA88F14A46012305B0C4
:1029B800BDE8F04F02F040BB70B5406886B006AB8A
:1029C80003E9060000282ED0012380F82D30866800
:1029D800164BF21A534243EB020390F82C205AB1DB
:1029E800002B134D134B144A08BF1D46134B00F11F
:1029F8001C0418BF13460AE0002B0D4D0D4B0E4A60
:102A080018BF1D460D4B00F10C0408BF1346BDF856
:102A18001200BDF81410BDF8162000960195029416
:102A2800FFF78EFF012006B070BD00BFB034040868
:102A3800EC30040892360408CE32040874380408CE
:102A480070B5446886B006AB03E9060004B30123F9
:102A58006377A668104B227FF11A4B4243EB0103C0
:102A68000AB10BB904E01BB966680C4D0C4B01E0C8
:102A78000C4D0D4BBDF81200BDF81410BDF8162012
:102A880000960C3401950294FFF75AFF012000E0EC
:102A9800204606B070BD00BFFC3F0408383C04085F
:102AA8001A3E0408D2410408A84304082DE9F0435B
:102AB80085B004AB03E906004468BDF80860BDF8BA
:102AC8000A90BDF80C50BDF80E80002C00F08C80E8
:102AD8000123A3740220676802F076FA4FF6FF70AC
:102AE80002F086F9002002F06DF9EDB25FFA88F87D
:102AF800A6F1160189B230462A4643460097FFF7E9
:102B08004CFE277A002F2ED1A28A234600E00137F7
:102B1800974204D29969097E04330029F7D002F05C
:102B28005DFA02F061FAA9F116091FFA89F90E2176
:102B380001FB10914FF6FF7208F101085FFA88F364
:102B480089B2009248462A46FFF7A5FD022002F006
:102B58003BFA1F2002F036F9A38A002B38D0103D2B
:102B6800E8B2303E2CE0E3685C68A28A2346013A6A
:102B7800002700E00137974204D29969097E04339F
:102B88000029F7D002F02AFA02F02EFA0E2101FBF2
:102B980010914FF6FF7208F101085FFA88F389B2C5
:102BA800009248462A46FFF776FD022002F00CFA0A
:102BB8001F2002F007F9A38A53B1103DE8B21A3E6C
:102BC8000637B1B254F827200123083202F04EFA32
:102BD800002002F0F9F94FF6FF7002F009F91F2002
:102BE80002F0F0F8012000E0204605B0BDE8F083CF
:102BF8002DE9F04105463620884614461F4610F058
:102C08001FFF0646E0B120F8025B41462E22FFF77F
:102C180007FCBDF8183086F8344073861820012365
:102C280086F8307086F8313010F00AFF044618B183
:102C380004234660037404E0304610F009FF00E006
:102C480004462046BDE8F081F8B5064624200F4624
:102C5800154610F0F5FE0446D8B10F4B0680836088
:102C68000E4B39464360102200F10C00FFF7D8FBE9
:102C780001260023182025622377667710F0E0FEEE
:102C8800054610B14460067404E0204610F0E0FEEA
:102C980000E005462846F8BDFC3F0408563A0408FB
:102CA800F8B506462C200F46154610F0C9FE044616
:102CB800E8B120F80C6B39461922FFF7B1FB0D4B30
:102CC800A562A3600C4B6360002384F825301820AC
:102CD800012384F8263010F0B3FE054618B103230B
:102CE8004460037404E0204610F0B2FE00E005469C
:102CF8002846F8BD08590408A655040810B5044626
:102D0800142010F09DFE20B100234380014B048065
:102D1800036110BD4D25000838B50546442010F064
:102D28008FFE0446C0B10E4B058243600D4B036015
:102D3800012383740023037283820B4B03641820DE
:102D480010F07EFE054618B107234460037404E0C2
:102D5800204610F07DFE00E00546284638BD00BF3D
:102D68009C510408924D0408412600082DE9F041C1
:102D780005463420884614461F4610F061FE064674
:102D880020B3144B05808360134B414643601022E7
:102D980000F10C00FFF744FB214606F11C0010224D
:102DA800FFF73EFB002386F82C30182001233763F9
:102DB80086F82D3010F044FE044618B1052346600D
:102DC800037404E0304610F043FE00E00446204659
:102DD800BDE8F081B03404080A2F04082DE9F04159
:102DE800044614200D461646984610F029FE07465C
:102DF800B8B1069B048003610023C37201234560B8
:102E0800068180F80A800373182010F019FE044622
:102E180018B106234760037404E0384610F018FE22
:102E280000E004462046BDE8F0812DE9F041044663
:102E380018200D461646984610F002FE0746B8B10F
:102E480001238370069B04800361079B45608660AD
:102E5800C0F80C804361182010F0F2FD044618B148
:102E680008234760037404E0384610F0F1FD00E0E1
:102E780004462046BDE8F0812DE9F34198461B8BB6
:102E88001D2B05460C4617464FF0000000F2B48093
:102E9800B5F5A07F0090019000F2AE80F02900F215
:102EA800AB80127CADF80610511EADF80250072910
:102EB80000F28A80DFE801F045595E04456A14761D
:102EC8007B684E4A7A611A8893F834303A80013B1D
:102ED800DBB2012B7FD8ADF80240ADF806507AE09E
:102EE80005F11602ADF8002004F11602ADF8042031
:102EF80002AE434A16E903007A6107F1080282E844
:102F0800030003F10802013348F82270A8F81830CA
:102F18007B681A8A187A3A8000286CD1FFF7FCFE81
:102F28003849436859603849DF600126163D196001
:102F380002461E72A8B2E1B24346FFF79DFF304633
:102F48005AE0012A0CBF314B314B78687B6130F86D
:102F58000C3B3B8011F06CF9431CDB001A34ED1874
:102F6800ADF80440ADF8005035E07B68294A1B688D
:102F78007A6102E0284A7B687A611B8814353B80B5
:102F8800ADF800501434ADF8044024E07B68234ABF
:102F98007A611A883A801A899B7AAD18ADF8005080
:102FA800E418F0E77E681E4B7B61338838463B8027
:102FB80073689847013D4519ADF80050B368384625
:102FC8009847013C0419DEE71648174A174B40F2A8
:102FD8001A3100F0E3FC02AA12E9030007F1080322
:102FE80083E80300B8F8183003F10802013348F801
:102FF8002270A8F818300120BDE8FC81D12500080E
:10300800B52A0008884904087E450408492A0008AA
:10301800C1290008AD28000807280008D3270008A0
:103028005D230008FCA40508502B0408FAA4050831
:10303800F8B51646002834D01378002B2ED0028B12
:10304800002327E0046A257C042D21D165682F8898
:103058008F421DD195F8313053B16F8E01F0D8FEF3
:1030680004F1080268866369204606CA98476F8695
:10307800A81C31462E22FFF7D3F995F831307BB1E1
:1030880004F108026369204606CA98470120F8BD82
:10309800013304309342D5D30020F8BD1846F8BD5B
:1030A8000120F8BD70B5B8B1068B0446002310E0C6
:1030B800256A287C04280AD16D682888884206D1A8
:1030C8001046A91C2E22FFF7ABF9012070BD013371
:1030D8000434B342ECD3002070BD38B5044620B3A5
:1030E800134BC361134BC0F89830134BC0F89C3096
:1030F800124B00257822C0F8A0308575C575058368
:10310800294600F1200010F08DFFD4F898302046B1
:10311800294698470A4A1388312B07D8094941F8A4
:10312800234001331380012038BD38BD284638BDFF
:10313800E9230008E1230008812300085724000838
:10314800740D0020241700202DE9F04104460028C2
:1031580000F0B380078B02460025A8E0136A1E7CA6
:10316800042E00F08780012E23D1586803888B42F3
:1031780040F09B8005F1080710F06AFC54F827001E
:103188004FF00008C0F8048010F062FC228B531E38
:103198009D4208D00732238354F8221044F82710A0
:1031A80044F8228002E044F8278025833046BDE8B1
:1031B800F081052E5ED0032E5CD0022E13D15B6801
:1031C800186803888B4270D14388013B9BB24380C7
:1031D8000BB910F03DFC05F1080654F82630586884
:1031E80010F036FC4EE0072E21D15E68338A8B4200
:1031F8005BD1002706E0BB1D013756F8230010F00D
:1032080027FCFFB2B38ABB42F5D80027B78205F185
:10321800080654F82630586810F01AFC54F82600AE
:1032280033E044F8267025830120BDE8F081062E9E
:103238001ED1586803888B4237D105F1080610F073
:1032480007FC54F826000027476010F001FC228B89
:10325800531E9D4209D00833013A54F823102283A3
:1032680044F8261044F82370DEE744F826701AE084
:10327800082E1AD1586803888B4216D110F0E8FB43
:1032880005F1080654F826000027476010F0E0FB17
:10329800228B531E9D42C4D0073254F8221044F8A2
:1032A800261044F822702383BEE701350432BD425C
:1032B800FFF454AF0020BDE8F081BDE8F08170B59F
:1032C800044600282AD0068B751E083600EB8606B1
:1032D8001EE056F8043D1A7C042A13D0012A11D0A6
:1032E800052A0FD0032A0DD0022A02D15B681B6879
:1032F80009E0072A02D15B68198A05E0062A01D08D
:10330800082A04D15B6819882046FFF71DFF013D94
:10331800681CDED100232383012070BD70BDF0B589
:1033280028B30023068B1A461EE0046A257C072D65
:1033380018D16468258A8D4214D1A78A002504EB28
:1033480083040DE004EB050C0435DCF818C09CF888
:1033580018C0BCF1010F03F1010301D1D8B2F0BDCF
:10336800BB42EFD301320430B242DED30020F0BDBD
:1033780070B508B3048B00231BE0026A157C072D87
:1033880015D15268158A8D4211D10023958A1146AC
:103398001C46012007E013B99669307601E08E6972
:1033A800347601330431AB42F5D3012070BD0133CB
:1033B8000430A342E1D3002070BD2DE9F04128B3C9
:1033C8000023078B1A461EE0046A257C072D18D1B6
:1033D8006468258A8D4214D1B4F814C0002504EB22
:1033E80083040CE066190435B66996F81880B8F1BC
:1033F800010F03D106F10800BDE8F08101336345F0
:10340800F0D301320430BA42DED30020BDE8F081A7
:103418002DE9F04700282FD00023B0F818C01D462A
:1034280027E0046A267C072E21D16468268A8E420A
:103438001DD1B4F81480002604EB830915E009EBCC
:103448000604A7693C7E012C0DD192F800A0BAF1C0
:10345800000F08D007F1080011461022FEF7E0FF20
:103468002046BDE8F087013304364345E7D30135EC
:1034780004306545D5D30020BDE8F087F0B5B0B17C
:10348800068B002510E0046A277C062F0AD16468A1
:1034980027888F4206D123819DF814306260A37279
:1034A8000120F0BD01350430B542ECD30020F0BD59
:1034B80010B500210446FEF793FF20460121BDE820
:1034C8001040FEF78DBF38B598B1048B0246002333
:1034D8000CE0106A058804328D4206D100F108021A
:1034E800436906CA9847012038BD0133A342F0D387
:1034F800002038BD10B50C460021FEF771FF2046AC
:103508000121BDE81040FEF76BBF13B502AC04E91A
:103518000C00BDF80230834206D8BDF80030834263
:1035280034BF0020012000E00020BDF806308B42A7
:1035380006D8BDF804308B4234BF0021012100E0D9
:103548000021002818BF0846C0B21CBD38B5114B71
:10355800114A1988002319E052F8045FA87D012850
:1035680012D100240CE004F1080355F82300037C71
:10357800082B03D1436800211B6998470134A4B282
:103588002B8BA342EFD838BD01339BB28B42E3D1DA
:1035980038BD00BF740D002020170020704770B59B
:1035A800094CA5787DB9094B1E78012E0BD16368AB
:1035B800013363606268064B9A4204D9284601F0D9
:1035C800C5FCA670656070BD740D002084010020E4
:1035D80040420F00054A9060134602E0996801399D
:1035E800996091680029F9D1704700BF740D0020D7
:1035F800F0B585B001F058FF002800F0498100259A
:1036080002A80DF10A01ADF80850ADF80A5001F012
:103618004DFF03A80DF10E01ADF80C50ADF80E509A
:1036280001F090FFBDF80C10BDF808200091BDF81E
:103638000E10BDF80A3001912C46964D9649082087
:1036480009F0CCF8A878012803D101F07FFCAC7010
:1036580019E1924B5B78012B40F01581AB78002B78
:1036680040F011816B6029888D4A09E152F8046F96
:10367800B07D012840F002810025FAE005F1080339
:10368800BDF8080056F82340BDF80A1004F10803F5
:103698000CCBFFF73AFF002800F0E980237C013BC0
:1036A800062B00F29F80DFE803F00429159D1F9D7B
:1036B8004C006668012304F10805337795E8060095
:1036C800636920469847002333772046636995E865
:1036D800060086E0636893F8252012F1FF3218BFD0
:1036E800012283F8252077E0636893F82C2012F1F3
:1036F800FF3218BF012283F82C206DE06268137E28
:103708001568002B6ED16E882F462946184606E0AC
:1037180051F804EFDEF804E001338EF81800B342E4
:10372800F6D301231376002607E057F8040F00F1BB
:103738000802436906CA984701366B889E42F4D34B
:1037480050E0656820892E68A37B227B0096A0F153
:10375800160189B2FFF721F81420FFF73BFF2B7AF7
:10376800C3B9AF8A29461A461E4609E0886990F807
:1037780018E00676BEF1010F08BF13460431013286
:10378800BA42F3D301220BB9AB6924E0053355F8EB
:10379800233020E06368DB685A680023908A154666
:1037A80019461F4609E0AE6996F818E03776BEF16B
:1037B800010F08BF0B46043501318142F3D3411E86
:1037C8008B4203D1053052F8203003E004D207338E
:1037D80052F8233001221A7604F1080206CA6369F6
:1037E80020469847237C013B072B4CD8DFE803F0A1
:1037F8000410074B0A0D123A63681B6A34E06368C9
:103808009B6A2DE063681B6B2AE063681B6927E0ED
:10381800636824E063681A7A7AB9988A1946013885
:1038280000E00132824204D28C69247E0431002CEB
:10383800F7D0063253F8223011E0DB685A68908AD4
:1038480011460138002300E00133834204D28C6919
:10385800247E0431002CF7D0063352F82330DB697C
:10386800984710E06368DB68204698470BE001350D
:10387800ADB2338BAB423FF601AF04E001339BB2EC
:103888008B427FF4F3AE01F055FE0F20FFF7A2FE46
:1038980005B0F0BD740D002022A5050884010020A4
:1038A80020170020034B9A6812B19A68013A9A606F
:1038B800704700BF740D00202DE9F3470120DFF8A1
:1038C800D080DFF8D09001460AF022FB01240025C1
:1038D8004FF4807602274046694600968DF80470BA
:1038E8008DF805408DF806508DF8074009F068FFFF
:1038F80040460821224609F0E3FF244BDFF8988070
:103908001A6844F2A243B2FBF3FA0AF1FF3A2046DE
:1039180021461FFA8AFA0AF02BFBC8F804A0484689
:103928004146A8F80050A8F80250A8F8085088F8AE
:103938000A500AF0B9FE7023A8F80C300423A8F83E
:1039480010300AF1FF3A6323642203FB0AF3B3FB46
:10395800F2F39BB2C8F8143008F10C014846A8F8F5
:103968000E40A8F81870A8F81A50A8F81C60A8F813
:103978001E500AF0B7FF484621460AF02AFF48467B
:1039880021460BF030FABDE8FC8700BFF0020020AA
:103998000000024000000140840D002083B50E465F
:1039A8000746154910201C46154608F017FF102039
:1039B800124908F013FF1020114908F00FFF1020DA
:1039C8000E4908F00BFF002310200E49019308F060
:1039D80005FF334610200C493A4608F0FFFE102038
:1039E8000A492A4608F0FAFE10200949224608F03A
:1039F800F5FE019B0133E7E75CA5050861A505080D
:103A080081A5050891A50508A1A50508B6A505087D
:103A1800C7A5050808B5164B1A6A01321A621A6A50
:103A2800012A1A4603D0134840F21D210FE05862BC
:103A3800194602E04B6A013B4B62506A0C4B002866
:103A4800F8D11A6A012A06D00A484FF40A710A4ABC
:103A58000A4BFFF7A3FF1A6A013A1A621B6A2BB1D5
:103A68000448054A064B40F22A21F2E708BD00BF88
:103A7800840D0020D8A505082E63040802A60508B1
:103A880013A6050810B5084C02210022204609F0AB
:103A98000CFF44F6FF70FFF7BDFF2046022101220C
:103AA800BDE8104009F001BF000402400C4B0D496D
:103AB8001A6844F2A2436428B2FBF3F3D4BF20EAA5
:103AC800E0706420013B9BB24B60013B5843642289
:103AD800B0FBF2F080B2486103480C310AF085BEB1
:103AE800F0020020840D00200000014010B5134BA7
:103AF80093F828202AB11248124A134B4FF4427106
:103B08000EE0012283F8282066234FF0C042013BD3
:103B1800DBB2108033B90A480A4A0C4B40F2123122
:103B2800FFF73CFF1488A4B28442F0D1084B1980F7
:103B3800024B002283F8282010BD00BF840D00200E
:103B4800D8A505083863040824A60508FAA40508BA
:103B58000000026010B5FFF7AFFE6420FFF7A6FF74
:103B680021210720FFF7C2FF3220FFF753FF012171
:103B78000020FFF7BBFF3220FFF74CFF232107206F
:103B8800FFF7B4FF3220FFF745FF00211020FFF7B1
:103B9800ADFF41F28830FFF73DFF33210720FFF7E3
:103BA800A5FF3220FFF736FF112046F63001FFF758
:103BB8009DFF3220FFF72EFF4FF4C0610220FFF770
:103BC80095FF3220FFF726FF122046F6EB41FFF75C
:103BD8008DFF3220FFF71EFF03204AF6A401FFF7EE
:103BE80085FF3220FFF716FF00210C20FFF77EFF2C
:103BF8003220FFF70FFF0D2040F60C01FFF776FF8C
:103C08003220FFF707FF0E204FF42C51FFF76EFF0D
:103C18003220FFF7FFFEB0211E20FFF767FF32209A
:103C2800FFF7F8FE012042F63F31FFF75FFF322031
:103C3800FFF7F0FE05200021FFF758FF3220FFF7BD
:103C4800E9FE00210620FFF751FF3220FFF7E2FED0
:103C580016204EF61C71FFF749FF3220FFF7DAFEF7
:103C6800172040F20311FFF741FF3220FFF7D2FE81
:103C780000210B20FFF73AFF3220FFF7CBFE00218F
:103C88000F20FFF733FF3220FFF7C4FE4120002149
:103C9800FFF72CFF3220FFF7BDFE42200021FFF77F
:103CA80025FF3220FFF7B6FE00214820FFF71EFF50
:103CB80040F23F143220FFF7ADFE21464920FFF7BE
:103CC80015FF3220FFF7A6FE00214A20FFF70EFF5E
:103CD8003220FFF79FFE00214B20FFF707FF32201D
:103CE800FFF798FE44204FF46F41FFF7FFFE3220A4
:103CF800FFF790FE00214520FFF7F8FE3220FFF77E
:103D080089FE21464620FFF7F1FE3220FFF782FEAA
:103D1800302040F20771FFF7E9FE3220FFF77AFE04
:103D280031204FF40171FFF7E1FE3220FFF772FEF8
:103D380032204FF40171FFF7D9FE40F202543220CD
:103D4800FFF768FE21463320FFF7D0FE3220FFF749
:103D580061FE342040F20751FFF7C8FE3220FFF71A
:103D680059FE35204FF40171FFF7C0FE3220FFF7EE
:103D780051FE36204FF40171FFF7B8FE3220FFF7ED
:103D880049FE21463720FFF7B1FEA4F50074322022
:103D9800FFF740FE21463A20FFF7A8FE3220FFF742
:103DA80039FE2F2041F2BE21FFF7A0FE3220FFF797
:103DB80031FE21463B20FFF799FE3220FFF72AFE0D
:103DC80000212320FFF792FE3220FFF723FE002177
:103DD8002420FFF78BFE3220FFF71CFE25204FF42E
:103DE8000041FFF783FE3220FFF714FE00214F2029
:103DF800FFF77CFE3220FFF70DFE4E200021FFF773
:103E080075FE3220BDE8104004E608B5124B93F861
:103E180029202AB11148124A124B40F222310FE0F0
:103E2800012283F82920222166234FF0C042013B5A
:103E3800DBB2118033B90948094A0B4B40F23B31D8
:103E4800FFF7ACFD108880B22228F0D1024B002287
:103E580083F8292008BD00BF840D0020D8A50508D7
:103E68004563040824A60508FAA4050810B51E4BE6
:103E7800032826D8DFE800F0021A080E1C8841F251
:103E8800280246F628000AE01C8841F2080246F695
:103E9800080004E01C8841F2300246F6300049F27E
:103EA80041318C4214BF014611460BE0188846F692
:103EB800200249F24131884214BF11464FF4815122
:103EC80000E000211B8848F68912934205D049F288
:103ED8002032934204D1032000E01120FFF706FEB0
:103EE800BDE8104091E700BF86010020014B188013
:103EF8000A208FE5000002604FF0C043188003F5E8
:103F080000331A881A88188880B270474FF0C04367
:103F180022221A8003F5003382B01A8892B2ADF8D3
:103F280006201B889BB2ADF80630BDF8060080B2AB
:103F380002B07047072040F27311D7E5072000212F
:103F4800D4E582B0044BADF80600BDF8062092B265
:103F58005A8502B0704700BF840D002082B0044B20
:103F6800ADF80600BDF8062092B25A8002B070473C
:103F780086010020014B80B2188070470000026063
:103F88004FF0C04380B218807047024B80B218804F
:103F9800704700BF000002604FF0C04380B2188035
:103FA8007047024B80B21880704700BF0000026063
:103FB80082B0044B0190019ADA62DA6A002AFCD1D5
:103FC80002B07047840D002070B54FF0C0452A2418
:103FD8002C800A4C060AC0B226802080100AD2B271
:103FE800208022802B222A800A0A2280C9B21A0A3B
:103FF800DBB221802280238070BD00BF00000260F8
:1040080010B50B4614460246FFF7DEFF4FF0C043DB
:104018002C22A0B21A80BDE8104067E7114B1B881C
:1040280048F68912934210B504460BD049F2203263
:10403800934212D1C1F1EF01202089B2FFF756FD5A
:10404800212006E0C1F1EF014E2089B2FFF74EFDB5
:104058004F202146BDE8104048E502460B46BDE822
:104068001040B1E78601002008B5FFF7D7FF0F4BD6
:104078001B78012B4FF0C0420D4B0FD12E21118020
:104088001A881A881B8892B202F0FC0002F478425F
:1040980042EAC000C3F3C423184308BD222111809B
:1040A8001A881A88188880B208BD00BFF417002043
:1040B8000000026070B5074D0646012421463046CF
:1040C800FFF7D2FF0134A4B2C82C25F8020FF5D1AE
:1040D80070BD00BF4646002010B5084B1B78012B69
:1040E800144602D1BDE810408AE7FFF797FFFFF7B3
:1040F8008CFE2046BDE81040F8E600BFF41700200B
:1041080070B5074D064601242146013435F8022FC3
:104118003046A4B2FFF7E0FFC82CF5D170BD00BF50
:104128004646002070B505460E46FFF7C3FF01243A
:104138002146013428463246A4B2FFF7CDFFC82CE9
:10414800F6D170BD2DE9F04104460D461646BDF87E
:104158001880032B39D8DFE803F00B3519273819F5
:1041680080B2294642460137FFF7B6FFBFB200E0EA
:104178000027B742F3D1BDE8F081E01B80B22946A1
:1041880042460137FFF7A8FFBFB200E00027B74259
:10419800F3D1BDE8F081E91B89B2204642460137D8
:1041A800FFF79AFFBFB200E00027B742F3D1BDE89E
:1041B800F081791989B2204642460137FFF78CFF12
:1041C800BFB200E00027B742F3D1BDE8F08170B577
:1041D800194B1A4A598E92F9004064180025A4B266
:1041E8008AB0AC4208BF0124C62C28BFC62415706B
:1041F8000F264FF6FF721E865C865A8519202B46BD
:10420800009221460A22FFF79DFF21463046FFF71C
:104218002BFF224603460A4902A80FF083FF02AA91
:1042280006A808490FF07EFF3220D22106AA2B46A5
:1042380000F002FF0AB070BD840D0020E42D0020BC
:1042480039A6050841A605082DE9F341BDF8205017
:104258000C4690461F461A46002306460095FFF76F
:1042680071FF611E414430463A46002389B20095E9
:10427800FFF768FF30462146424601230095013E7C
:10428800FFF760FFBF19B8B22146424601230895DF
:1042980002B0BDE8F04155E72DE9F0410D46C5F102
:1042A800F008411E5E18C2EB0802C5F1EF039BB28D
:1042B80092B2B6B29A422CBF904698469A4234BF00
:1042C80011461946864234BF3746074640F23F1327
:1042D800864238BF06469E4228BF1E46174B1B889B
:1042E80048F68912B8F1EF0F28BF4FF0EF08934254
:1042F800044610D049F2203293421AD15020FFF7D9
:10430800F5FB51204146FFF7F1FB52203946FFF7F4
:10431800EDFB53200AE041EA082189B24420FFF767
:10432800E5FB45203946FFF7E1FB46203146FFF71C
:10433800DDFB20462946BDE8F0416FE686010020F6
:1043480000200146F0224FF4A073A5E770B580B2B3
:1043580002FB03F489B292B29BB2FFF79DFF0020E3
:10436800FFF784FD0025064E04E0708D80B2FFF74C
:10437800BDFD0135A542F8DBBDE87040E0E700BFB0
:10438800840D002070B54FF0C0452A242C80094CBC
:10439800060A26802080080A208021802B21298077
:1043A800110A218022801A0A228023802C232B8044
:1043B80070BD00BF0000026070B5114B1B78012B67
:1043C800044607D1002040F23F110246EF23FFF7D1
:1043D800D9FF04E0FFF7B4FF0020FFF747FDF02501
:1043E80009E0013E2046B6B2FFF780FD002EF8D165
:1043F800013DADB215B14FF4A076F2E770BD00BF34
:10440800F41700202DE9F04F1C463E4B87B01B786F
:10441800039183469DF8441010980591012B039B46
:10442800049092461FFA8BF09AB208D1411E531E8F
:104438000919534489B29BB2FFF7A4FF09E01FFA98
:104448008AF51146A3B22A46FFF726FF0020FFF798
:104458000DFD0027DDF80C803E4640F23F1CA146CA
:1044680039E0BBF1000F2EDB65452CDC03980028F2
:1044780029DBB8F1EF0F26DC220702D1002CC8BFD8
:10448800013621492140002903DA013961F00F0181
:104498000131059A0AB1C1F10F01049830F81620CC
:1044A80003FA01F10A4012B26AB118494A8D02931F
:1044B80092B2A8B21FFA88F1CDF804C0FFF70CFE3B
:1044C800DDF804C0029B013401354C45C9DB0136D7
:1044D800013708F10108574503DA5D460024012336
:1044E800F3E7084B1B78012B08D1002040F23F115D
:1044F8000246EF2307B0BDE8F04F43E707B0BDE839
:10450800F04F1DE7F41700200F000080840D0020F5
:104518002DE9F74F1F463B4BDDF830801B781646D8
:104528009DF83420012B044601920D4680B28AB2D0
:1045380008D1411E531EC9199B1989B29BB2FFF7B6
:1045480021FF09E01FFA86FE1146BBB27246FFF74B
:10455800A3FE0020FFF78AFC4FF0000BDA463DE08F
:10456800002C30DB09EB040340F23F1293422ADCB3
:10457800002D28DB0BEB0503EF2B24DC19F00F0FC4
:1045880004D1B9F1000FC8BF0AF1010A1E4B09EAAC
:104598000303002B03DA013B63F00F030133019A95
:1045A8000AB1C3F10F03012202FA03F338F81A2003
:1045B80013401BB213B1154B588D01E0144A5088B3
:1045C80080B2FFF793FC09F1010901E04FF00009FF
:1045D800B945C5DB0AF1010A0BF1010BB345F5DB5F
:1045E800084B1B78012B08D1002040F23F110246EE
:1045F800EF2303B0BDE8F04FC4E603B0BDE8F04FC9
:104608009EE600BFF41700200F000080840D0020F4
:10461800860100202DE9F0411C4F069C3F789DF84B
:104628001C60012F02FB03F580B28FB209D1411E35
:10463800CB1899B27B1E9A1893B23A46FFF7A2FE9E
:1046480007E092B29BB23946FFF726FE0020FFF73B
:104658000DFC002709E034F8020B1EB1030A43EAF7
:10466800002080B2FFF742FC0137AF42F3DB074B73
:104678001B78012B07D1002040F23F110246EF239F
:10468800BDE8F0417EE6BDE8F04159E6F4170020A8
:104698002DE9F0431F2093B0FFF78EFE4FF47840CA
:1046A800FFF78AFE4FF6E0754FF4FC60FFF784FED3
:1046B8002846FFF781FE0020514CFFF77DFE0020C1
:1046C8004FF6FF79014664220346A4F82A90CDF8F4
:1046D8000090FFF737FD00200A2164220346CDF839
:1046E8000090FFF72FFD00200146642201234FF4BC
:1046F800784765850095FFF725FD7720EF21C822CB
:1047080000234FF4FC6667850097FFF71BFDBD216A
:104718003222012340F23F1066850096FFF712FD12
:10472800A02032220023782167850097FFF70AFD31
:10473800A0207821322201234FF01F0866850096B9
:10474800FFF700FDA020782132220223A4F82A8056
:10475800CDF80080FFF7F6FCA02078213222032351
:1047680065850095FFF7EEFC264B2749A3F80280E4
:1047780002AD3C2228460FF013FCEB20C321052292
:10478800302300950025A4F82A900195FFF7C0FE74
:1047980032210A2096220B4667850097FFF754FDC1
:1047A80032213C2096220B4666850096FFF74CFD89
:1047B80032210B4696226E20A4F82A80CDF800807C
:1047C800FFF742FDFFF7BAFBFFF7B4FB3220FFF714
:1047D8006DF92846FFF76AF96420FFF767F90B4B74
:1047E80003F110028DE8240028465A681B68294600
:1047F800FFF710FF1195119B01331193FBE700BFE1
:10480800840D0020860100205A630408E08701080F
:104818002DE9F14FFFF750F84FF0C0456420FFF73E
:1048280045F90127FFF72EF94FF028096D48FFF7E2
:10483800F1F82F800520A5F8009002F025FECF237F
:104848002B80694B002683221E801A8030221A8012
:10485800ED222A804FF064080322A3F800801A8012
:1048680012221A8081221A80E8222A8085221A8040
:1048780079221F801A80CB222A8039221A804FF091
:10488800340C02242C21F72219801E80A3F800C0C2
:104898001C802A8020221A80EA222A80C0221E80B8
:1048A800C1211E802A8026221A8029801121198080
:1048B800C5212980352119803E211980C7212980E9
:1048C800BE211980362129803A205521A3F800906D
:1048D80028801980B12129804FF0100BF2211E8009
:1048E800A3F800B02980082119802A80E0221F80BF
:1048F8004FF01F092A801A22A3F800904FF0180AD7
:104908001A800F210A22A3F800A01A801980062114
:1049180019804521198087211980322119800721A2
:104928001A804FF0E10E19801C80052419801C8024
:104938001E80A5F800E04FF0250E1E80A3F800E0C9
:104948004FF0270EA3F800E01C80A3F800B04FF04A
:10495800090BA3F800B04FF0780B1880A3F800B04B
:104968004FF04D0BA3F800B01C800D24A3F800A055
:104978001C8038241C8018802A20A3F80090EF247B
:1049880028802B201E801E801E801C8028803F20AF
:104998001E801E801F801880B720A5F800C02880C0
:1049A8001980B62129801A8082221A801122A3F840
:1049B80000E040461E8029272A8002F065FD404617
:1049C8002F8002F061FD0948FFF724F82C232F807F
:1049D80030462B8040F23F113246234601B0BDE8F5
:1049E800F04FCFE4400D03000000026040420F008A
:1049F8002DE9F041022098B00121002409F088FA3D
:104A0800012502268048169616A98DF85D408DF876
:104A18005E408DF85F408DF85C5008F0D1FE18209C
:104A2800294609F075FA2846294609F089FA2146E7
:104A38000C22764808F044FF0C227448294608F0F6
:104A48003FFF04210C22714808F03AFF05210C228F
:104A58006E4808F035FF07210C226C4808F030FF3B
:104A680008210C22694808F02BFF09210C2267480D
:104A780008F026FF0A2165480C2208F021FF0B21C7
:104A880062480C2208F01CFF0E210C225F4808F037
:104A980017FF0F210C225D4808F012FF07210C2296
:104AA8005B4808F00DFF08210C22594808F008FF60
:104AB80009210C22564808F003FF0A210C22544809
:104AC80008F0FEFE0B210C22514808F0F9FE0C21DB
:104AD8000A464F4808F0F4FE0D210C224C4808F015
:104AE800EFFE0E210C224A4808F0EAFE0C22484844
:104AF8000F2108F0E5FE4CF6B3734448169316A947
:104B08008DF85C608DF85E408DF85F408DF85D50E3
:104B180008F056FE16A94FF680733D4816938DF897
:104B28005C608DF85E408DF85F408DF85D5008F050
:104B380047FE40F6B830FEF76DFFFEF7A3FF40F6DC
:104B4800B830FEF767FF0F2311934FF480531027F7
:104B58000DF13C08099368464FF400231094129411
:104B68001494159400940194029403970494069461
:104B7800079408940A9405940B940C93CDF8348008
:104B88000F95139508F095FB0523684611930F962A
:104B98001094129414941594CDF83880139508F055
:104BA80088FB2946204608F004FC40F6B830FEF79A
:104BB80031FF2046FFF7A0F904461649164E38463D
:104BC800224607F00BFE41F289239C4248F68918D9
:104BD800124F01D044450ED1FEF7BCFF00233B70B5
:104BE800A6F8008010200E4948F6891241F2892360
:104BF80007F0F4FD05E0FFF70BFE49F241333D7085
:104C0800338018B0BDE8F08100040240000C024077
:104C18000010024046A6050886010020F41700206F
:104C28005DA605084FF0C04336221A8003F500330D
:104C3800012814BF682048201880704770B5244B9D
:104C480001228CB01A7000240AE0A9B21F22304653
:104C58000135FFF741FA642DF7D10134642C02D0F5
:104C68000025A6B2F1E73220014602460346FFF7C7
:104C7800ABF94FF0C0432E221A8003F50033002011
:104C88001A881C881D88A4B200F09CF8ADB20023D5
:104C9800224600930F492B4603A80FF043FA00233E
:104CA8000A20C82103AA00F0C7F904F0FC0204F4A2
:104CB800784444EAC20242EAD522074903A80FF021
:104CC80031FA0A20DC2103AA002300F0B5F9FEE737
:104CD800F41700209CA60508B4A605082DE9F04F96
:104CE80040F23F19484534BF04464C46EF2B34BFC9
:104CF80098464FF0EF084A4538BF9146EF2934BF30
:104D08000D46EF25C4EB090AC5EB080785B0BAF1D3
:104D1800000FB8BFCAF1000A002FB8BF7F424FF694
:104D2800FF734C452CBF1A4601221FFA8AFA4545E3
:104D380038BF0123BFB202930FFA8AF63BB29E42F4
:104D4800BDF838B0019202DDC6F34F0607E002262F
:104D580093FBF6F67642B6B201E01E4603E00FFA80
:104D68008AF35B420393144A1378022B20462946A0
:104D78005A4602D1FDF7FDFC01E0FFF7ADF94C45BD
:104D880001D1454514D0039A33B2934205DD019A07
:104D9800F31BA4189BB2A4B200E0334636B23AB271
:104DA8009642DADA029A5344AD189BB2ADB2D4E710
:104DB80005B0BDE8F08F00BFC04400200048704730
:104DC800FC17002082B0064BADF80600BDF806209F
:104DD80092B21A80188880B202B0FFF7B2B800BF4A
:104DE800F8170020014B188880B27047F817002088
:104DF80082B0064BADF80600BDF8062092B21A80C4
:104E0800188880B202B0FFF7A9B800BFFA170020CF
:104E1800014B188880B27047FA170020FFF7CCBA08
:104E2800FFF73ABA10B5BDF808400294BDE8104043
:104E3800FFF788B910B5BDF808400294BDE81040E6
:104E4800FFF702BAFFF782BA2DE9F04F4FEA42089E
:104E580000253D4C85B082468B46C8F103081746AD
:104E68002E461FFA87F909EB0B0C228805EB0A037B
:104E78001FFA8CFC9BB26146184692B2CDF804C06A
:104E88000293FFF729F9C9EB0B0292B20392029B36
:104E980022880399184692B2FFF71EF9DDF804C07C
:104EA8002288C5EB0A039BB26146184692B2029368
:104EB800FFF712F9029B22880399184692B2FFF76E
:104EC8000BF905EB0B0292B2039209EB0A03228855
:104ED80003999BB2184692B20293FFF7FDF8029B22
:104EE8002288C5EB0B0C1FFA8CFC1846614692B25F
:104EF800CDF804C0C9EB0A09FFF7EEF82288039938
:104F08001FFA89F992B24846FFF7E6F82288DDF8D9
:104F180004C092B248466146FFF7DEF8B8F1000FC8
:104F280004DA08EB860808F1060805E0F31B08F127
:104F38000A0808EB8308013F01360135BE42ADB2CD
:104F48008FD905B0BDE8F08FF817002008B9FEF733
:104F5800F5BF012801D1FEF7EDBF7047704700206B
:104F68000146F0224FF4A073FFF796B9704708B5D1
:104F780005280CD8DFE800F01214030507090948D2
:104F880008BD094808BD094808BD094808BD0948C1
:104F9800094A0A4B40F24111FEF700FD084808BDD6
:104FA800084808BD74010020640100205C0100204D
:104FB80054010020BFA6050896630408FAA4050852
:104FC8007C0100206C01002010B50446FFF7CFFFDC
:104FD800014B18601C7110BD8C010020014B187921
:104FE800704700BF8C01002008B5FFF7C0FF80881C
:104FF80008BD08B5FFF7BBFFC08808BDF7B51F4659
:105008000B4B0C4E1D681446EA882B68203C544311
:10501800A4B2AE1B03EB440418BF0126AB888DE88D
:10502800500017B1FFF7EEF901E0FFF771FAFEBD86
:105038008C0100207C0100202DE9F0410F469846A4
:1050480015460446084E08E0204643463946FFF711
:10505800D5FF33689B88E418A4B215F8012B002A01
:10506800F2D1BDE8F08100BF8C01002010B50446E4
:1050780008462146BDE81040DEE7094B70B50446F6
:1050880018790E461546FFF7B4FFC6F1F001091A64
:1050980089B220462A460023BDE87040CCE700BF0D
:1050A8008C010020704700BF044B1A680AB9044AF3
:1050B8001A601A681018186010467047B80D00205A
:1050C800045300204FF0FF30704708B50248034AE8
:1050D800034B3721FEF762FCDEA60508AC63040823
:1050E800FAA405080120704710B504460A480221B1
:1050F80009F094F90028F9D00748214609F057F932
:105108000548012109F08AF90028F9D00248BDE8CC
:10511800104009F049B900BF0038004010B51948DF
:10512800022109F07BF90028F9D01648002109F07E
:105138003EF91448012109F071F90028F9D0114805
:1051480009F032F90402A4B2002301E001339BB252
:10515800002BFBD00B48022109F060F90028F9D098
:105168000848002109F023F90648012109F056F9F9
:105178000028F9D0034809F017F92043C0F3CB0001
:1051880010BD00BF003800402DE9F0478AB00AAFD3
:105198000A20012108F0BCFE4FF4604347F8143D93
:1051A800474EDFF824A1012400254FF002083046BD
:1051B80039468DF81A508DF818808DF819808DF8B9
:1051C8001B4008F0FDFA30460D21052208F078FB57
:1051D80030460E21052208F073FB052230460F21C8
:1051E80008F06EFB21464FF4804008F0B5FE5046AB
:1051F80008F090FF4FF48273ADF802304FF400735B
:10520800ADF80A303823ADF80C305046072369460C
:10521800ADF81030ADF80050ADF80450ADF80650B8
:10522800ADF80850ADF80E5008F0A6FF50462146DC
:1052380009F03DF8A9468DF81A5030464FF48055CC
:10524800394605958DF818408DF819808DF81B4062
:1052580008F0B6FA3046294608F023FB40253946BF
:1052680018488DF818908DF819808DF81A908DF8D7
:105278001B40059508F0A4FA21464FF4804008F039
:1052880077FE0621032009F001F90C2307A88DF801
:10529800213007958DF820908DF8224007F084FF83
:1052A80017238DF8243009A80F238DF825308DF8A1
:1052B80026308DF8274002F06BFB0AB0BDE8F08776
:1052C80000040240000C024000380040014B1878EE
:1052D800704700BFBC0D0020024B5A889B88028093
:1052E8000B807047BC0D0020014B00221A707047DC
:1052F800BC0D0020F0B593B06846002148220EF09E
:1053080091FE6D46002464484FF4805108F0CBFAB2
:10531800002301E001339BB2002BFBD09020FFF764
:10532800E3FE002301E001339BB2002BFBD0FFF723
:10533800F5FE4FF480510746574808F0B2FA0023AB
:1053480001E001339BB2002BFBD053484FF480514E
:1053580008F0A9FA002301E001339BB2002BFBD02F
:10536800D020FFF7C1FE002301E001339BB2002BE0
:10537800FBD0FFF7D3FE4FF480510646464808F0AD
:1053880090FA45F8047B01342E6244484021E4B287
:1053980008F075FA10B9092CB5D101E0092C78D1BB
:1053A8009DE80C00D218029B03980699D218049B1A
:1053B800C018059BC018079BCB180899032490FBBD
:1053C800F4F092FBF4F25B1893FBF4F3151AC11A8C
:1053D8009C1A002DB8BF6D420029B8BF4942002C65
:1053E800B8BF6442502D03DD502909DD502C50DC34
:1053F8008D4205DAAC424FF0020405DB111806E0D5
:105408008C424FF0020401DAD11800E0C1180A9B5F
:10541800099A0C980F9DD2180B9BD2180D9BC01897
:105428000E9BC018109BEB18119D91FBF4F10324FF
:1054380092FBF4F290FBF4F05B1993FBF4F3161A69
:10544800C41A9D1A002EB8BF7642002CB8BF644219
:10545800002DB8BF6D42502E89B203DD502C09DDF6
:10546800502D16DCA64205DAB5424FF0020405DBE2
:10547800131806E0A5424FF0020401DAD31800E041
:10548800C318074A93FBF4F39BB29380012351801E
:10549800137013B0F0BD00BF00040240000C0240BE
:1054A800BC0D002000000000FFF710BFF7B505464F
:1054B8000C4601A80DF10601FFF70EFF1B4BBDF8C6
:1054C8000660BDF8040093E80600724301FB002261
:1054D80099685218164992FBF1F207EE102AF8EE75
:1054E800C77A40F23F17FCEEE77A17EE902A92B29D
:1054F800B2F5207F28BF3A462A801D69DA685B69C1
:105508006E4302FB0060C01890FBF1F107EE101A21
:10551800F8EEC77AFCEEE77A17EE903A9BB2B3F54D
:10552800F07F28BFEF232380FEBD00BFC40D0020FD
:1055380040420F00FFF7D8BE014B187E704700BFEE
:10554800C40D0020FFF7C8BE042808B505D90748D0
:10555800074A084B7D21FEF721FA054B03EB800033
:10556800038B0B80438B138008BD00BFFFA6050883
:10557800B26304081DA7050808B5082001F094F9CE
:1055880042F69643C31A584240EB030008BD10B5D3
:105598000A2001F0B1F90C4C20600E2001F0ACF9A2
:1055A8006060122001F0A8F9A060162001F0A4F9AB
:1055B800E0601A2001F0A0F920611E2001F09CF99A
:1055C80001236061237610BDC40D002010B5FFF7DC
:1055D800DBFD01F033FA044601F03CFA07490346C3
:1055E8002246202007F0FAF8FFF7C6FF28B101F09D
:1055F8003FFA10B9BDE81040C9E710BD59A7050822
:1056080010B5104C0A20216801F05DF961680E2080
:1056180001F059F9A168122001F055F9E168162046
:1056280001F051F921691A2001F04DF961691E2034
:1056380001F049F9082042F69641BDE8104001F012
:1056480025B900BFC40D00202DE9F04F0346A7B0CF
:10565800B0F800C01C898688DF885D89CDF810C045
:10566800B249B0F802C0B3F80C90B3F80E80CDF888
:1056780024C00FFA84FB30B201220FFA87FE0BEB2D
:10568800000C0A7629B20FFA89FACDF888C001EB26
:105698000E0C0FFA88F2CDF890C00AEB0B0CCDF87F
:1056A80030C002EB010CCDF858C0B3F810C05B8ACB
:1056B800CDF800C00FFA8CFC06910CEB00010A91A2
:1056C80002930CEB0A011BB2239103EB0E010E911E
:1056D80099182591049900FA81F05844504460447F
:1056E800DDF824C006990EFA8CFEDDF810C01FFA0A
:1056F80080FB1CFB0CF08E4416FB0600964414FB42
:105708000400009A19FB09009E4412FB02001FFACC
:105718008EFA09F08DFFDDF824C0029ACDE9120156
:105728001CFB0CF017FB070015FB050018FB080015
:1057380012FB020009F07CFFDDF824C0029ACDE9D3
:10574800140104991CFB01F317FB063615FB0466CC
:10575800009B18FB096612FB036009F069FFDDE98D
:105768001423CDE90001DDE9120109F0D7FF044651
:105778000D46DDE9000102460B4609F0CFFF02465F
:105788000B462046294609F015FECDE91801584672
:1057980009F05EFFCDE91001DDE91023DDE9000124
:1057A80009F0BCFFCDE90601504609F051FF8046DB
:1057B80089464246DDE912014B4609F0AFFFDDE9B3
:1057C8001023CDE91C01DDE9140109F0A7FF00222F
:1057D80006460F46564BDDE9180109F09FFF424681
:1057E80004460D464B46DDE9060109F097FF0246DF
:1057F8000B4609F0E1FD02460B462046294609F012
:10580800DBFD424604460D464B46DDE91C0109F026
:1058180085FF02460B462046294609F0CBFDDDE907
:10582800102304460D463046394609F077FF0246F4
:105838000B462046294609F0BDFDDDF828C0CDE914
:1058480002014FEA8C10DDF830C000EB0C20DDF8C7
:1058580010C0A0241CFB040009F0EAFEDDF838C0E3
:10586800CDE90A014FEA8C10DDF858C000EB0C2096
:10587800DDF824C01CFB040009F0DAFECDE90C01B8
:10588800504609F0D5FEDDE91023CDE91601DDE922
:105898000C0109F043FF4246CDE91E014B46DDE904
:1058A8000A0109F03BFF4246CDE920014B46DDE9FC
:1058B800000109F033FF32463B4609F07BFDCDE994
:1058C8000E01584609F0B4FEDDE91C23CDE91A01A2
:1058D800DDE9060109F06EFDDDF88CC0C024CDE9D4
:1058E800060104FB0CF0DDF888C0302505FB0C0030
:1058F800DDF810C078261CFB060009F099FEDDF8DB
:1059080094C0824604FB0CF0DDF890C005FB0C0047
:10591800DDF824C01CFB06008B4609F089FEDDE992
:10592800102306460F4609F0F9FE03E0C40D0020D7
:10593800000014404246CDE904014B465046594602
:1059480009F0ECFEDDE9142380468946DDE90A0109
:1059580009F0E4FEDDE9002304460D46DDE90C010B
:1059680009F0DCFE02460B462046294609F022FDD6
:105978000022A14B09F0D2FEDDE9202304460D46A2
:10598800DDE91E0109F016FD02460B46DDE91601A8
:1059980009F0C4FE02460B462046294609F00CFDD4
:1059A800002204460D46954BDDE90E0109F0B6FECE
:1059B80002460B462046294609F0FEFCDDE9022393
:1059C80009F0D6FF88A3D3E9002309F0A7FE0AF05F
:1059D8003FF98B490860DDE91223DDE90C0109F084
:1059E8009DFEDDE9002304460D46DDE90A0109F0C4
:1059F80095FE02460B462046294609F0DBFC0022AC
:105A08007D4B09F08BFEDDE91E2304460D46DDE9DA
:105A1800200109F0CFFC02460B46DDE91A0109F026
:105A28007DFE02460B462046294609F0C5FC0022A9
:105A380004460D46714BDDE9060109F06FFE02468A
:105A48000B462046294609F0B7FCDDE9022309F098
:105A58008FFF65A3D3E9002309F060FE0AF0F8F888
:105A6800674A5060DDE90E23DDE90A0109F056FEB8
:105A7800DDE9062304460D46DDE90C0109F04EFE7A
:105A880002460B462046294609F096FC00220446A9
:105A98000D465A4BDDE9180109F040FE02460B4657
:105AA8002046294609F088FCDDE9022309F060FF59
:105AB8004DA3D3E9002309F031FE0AF0C9F8504B91
:105AC80059469860DDE91423504609F027FEDDE9C0
:105AD800002304460D463046394609F01FFE0246AB
:105AE8000B462046294609F065FC0022424B09F086
:105AF80015FE424604460D464B46DDE9040109F011
:105B080059FC02460B46DDE9160109F007FE02467C
:105B18000B462046294609F04FFC35A3D3E900235C
:105B280004460D46DDE90E0109F0F8FD02460B4674
:105B38002046294609F040FCDDE9022309F018FF58
:105B480029A3D3E9002309F0E9FD0AF081F8DFF879
:105B5800B0C0DDE91223CCF80C003946304609F014
:105B6800DDFDDDE9002304460D465046594609F09F
:105B7800D5FD02460B462046294609F01BFC0022AB
:105B88001D4B09F0CBFDDDE9042304460D464046D4
:105B9800494609F00FFC02460B46DDE91A0109F0F7
:105BA800BDFD02460B462046294609F005FC10A318
:105BB800D3E9002304460D46DDE9060109F0AEFDF0
:105BC80002460B462046294609F0F6FBDDE902238A
:105BD80009F0CEFE04A3D3E9002309F09FFD0AF0E3
:105BE80037F8074908610DE00000000080842E4165
:105BF8000000000000C082400000144000008940FE
:105C0800C40D0020DDE90E235046594609F086FDF3
:105C1800DDE9062304460D463046394609F07EFD87
:105C280002460B462046294609F0C6FB11A3D3E9D4
:105C3800002304460D46DDE9180109F06FFD024610
:105C48000B462046294609F0B7FBDDE9022309F097
:105C58008FFE0AA3D3E9002309F060FD09F0F8FFDD
:105C6800034A506127B0BDE8F04FC9E4AFF30080A4
:105C7800C40D00200000000000C0824000000000A9
:105C880080842E41AFF30080064B074A59681160A3
:105C98001969064A1160D969054A11609A6A054B63
:105CA8001A60704794010020B03E0020CC440020C8
:105CB800A4440020603E0020014B1878704700BFC4
:105CC800E00D0020032808B505D90548054A064B0C
:105CD8007321FDF763FE0C235843044B185808BD85
:105CE80094A70508DE630408AEA705089401002000
:105CF800032808B505D90648064A074B7821FDF759
:105D08004DFE064B0C2202FB0030406808BD00BF68
:105D180094A70508EE630408AEA7050894010020BF
:105D2800034B044A1B780C2101FB03239868704736
:105D3800E00D002094010020034B044A1B780C203E
:105D480000FB032399607047E00D002094010020B8
:105D5800144B1B78012B10B5134B144C0ED119683A
:105D6800C82000F0B0FD2168CC2000F0ACFD104B3D
:105D7800D020196800F0A7FDD4200DE01968D820BC
:105D880000F0A1FD2168DC2000F09DFD084BE0201B
:105D9800196800F098FDE420064B1968BDE810402A
:105DA80000F091BD2C0F0020B03E0020CC44002014
:105DB800A4440020603E0020144B1B78012B10B532
:105DC800134C0FD1C82000F097FD2060CC2000F0C4
:105DD80093FD104B1860D02000F08EFD0E4B18601C
:105DE800D4200EE0D82000F087FD2060DC2000F0F1
:105DF80083FD084B1860E02000F07EFD064B18601C
:105E0800E42000F079FD054B186010BD2C0F002030
:105E1800B03E0020CC440020A4440020603E002076
:105E280008B502F071FB10B1BDE80840C4E7BDE851
:105E3800084029E70148FBF7CCBB00BFD815002074
:105E48000148FBF7C6BB00BFD81500200148FBF787
:105E5800C0BB00BFD81500200148FBF7BABB00BF84
:105E6800D8150020032808B505D91648164A174B37
:105E78004F21FDF793FD164B1870164B1870164BF3
:105E8800012202281A70154B0FD0032813D0904214
:105E980005D0134A12681A60BDE80840CAE7114ADB
:105EA80012681A60BDE80840CAE70F4A12681A600B
:105EB800BDE80840CAE70D4A12681A60BDE8084004
:105EC800CAE700BF94A70508FF630408D8A7050818
:105ED800E00D0020A63E00200C0E0020EC02002061
:105EE800E4020020E0020020DC020020D8020020AA
:105EF800064B07495960C021002219721E211A70E9
:105F0800D9601A745A611A76DA6170472818002025
:105F180040787D0110B50321FF22C02001F094F8DC
:105F28001F4C102120608022C02001F08DF8112123
:105F380020608022C02001F087F812212060802292
:105F4800C02001F081F8132120608022C02001F0D8
:105F58007BF8142120608022C02001F075F81521FB
:105F680020608022C02001F06FF880222060162176
:105F7800C02001F069F82060C0201721802201F0BC
:105F880063F82060074CC020227AB72101F05CF842
:105F98000023237463612376E3610123237010BD1A
:105FA800843E00202818002038B5C0200321FF2295
:105FB80001F04AF80B4D00242B19615D5A78C02076
:105FC800023401F041F8C82CF6D1B121AC22C0202E
:105FD80001F03AF8C0200321002201F035F8002032
:105FE80038BD00BF136404082DE9F34706460F4681
:105FF80092461D461AB90C1FE401914635E005EE9C
:10600800902A06EE903AB8EE657AF8EE667AFC01C8
:10601800C7EE277AA4F500749FED5C7A67EE877A5D
:1060280017EE900A09F026FB41EC100B0BF070FB01
:1060380059EC108B4946404609F032FE24184FEAC5
:10604800CA1009F0F5FACDE90001284609F0F0FA7E
:106058004B46424609F062FB02460B46DDE9000169
:1060680009F0A8F909F01CFE8146002E14BF4FF074
:1060780022084FF01A08C5F307224146C02000F055
:10608800E3FF08F10101EAB2C02000F0DDFFC4F32C
:10609800014208F10201C02000F0D6FFC4F3072234
:1060A80008F10301C02000F0CFFFE2B208F10401BB
:1060B800C02000F0C9FFC9F3034305F4702243EA86
:1060C800123208F10501C02000F0BEFF08F10601F8
:1060D800C9F30722C02000F0B7FF08F107015FFAF3
:1060E80089F2C02000F0B0FFC020B121A02200F04A
:1060F800ABFF07EE107A264CF8EEC77A0EBBD4ED4C
:10610800015A06EE90AAB8EE657A05EE905AB8EEF6
:10611800666AF8EE656A0123C6EE266A237477EE8E
:10612800A67A67EE277A17EE900A09F0A3FA41ECEF
:10613800100B0BF0EDFA51EC100B09F0B1FD60619A
:1061480020E005EE90AAD4ED016AB8EE656A05EE86
:10615800905AB8EE667AF8EE656A0123C6EE266AAA
:10616800237677EEA67A67EE277A17EE900A09F07B
:1061780081FA41EC100B0BF0CBFA51EC100B09F043
:106188008FFDE0610020BDE8FC8700BF00000043F0
:10619800281800200022012326E7012838B50D46DB
:1061A80004D002280CBF3C242C2400E034242146CF
:1061B800C02000F0C3FF05F0070200F00F0040EA1E
:1061C80002122146C020BDE8384000F03DBF2DE94D
:1061D800F3470A9C1D4607468A461646524B01E07D
:1061E8006D0864089C42FBD82DB906F10076043E80
:1061F800F601A94634E006EE905AB8EE667A06EE45
:10620800904AF8EE667AF601C7EE277AA6F5007688
:106218009FED467A67EE877A17EE900A09F02AFA18
:1062280041EC100B0BF074FA59EC108B49464046C0
:1062380009F036FD3618E80109F0FAF9CDE9000150
:10624800204609F0F5F94B46424609F067FA02463E
:106258000B46DDE9000109F0ADF809F021FD8146A2
:10626800022F9BBF324BDB194FF0000893F8C88010
:10627800C4F307224146C02000F0E6FE08F1010100
:10628800E2B2C9B2C02000F0DFFE08F10201C9B2D3
:10629800C6F30142C02000F0D7FE08F10301C9B2DD
:1062A800C6F30722C02000F0CFFE08F10401C9B2EE
:1062B800F2B2C02000F0C8FE04F47024C9F303430E
:1062C80008F1050143EA1432C9B2C02000F0BCFE4F
:1062D80008F10601C9B2C9F30722C02008F107086E
:1062E80000F0B2FE5FFA89F25FFA88F1C02000F090
:1062F800ABFEBAF1010F0CBF2F220F220DB942F0ED
:106308004002012F06D002D3022F0AD105E0C02097
:10631800102104E0C020112101E0C020122100F06A
:1063280093FE0020BDE8FC87FFFF0F00000000433C
:106338001364040807B5012300930023FFF747FF00
:106348000EBD00280CBFFF22002208B5C020032183
:1063580000F07AFE002008BD08B5C020B121AC22AB
:1063680000F072FE002008BD08B50420012107F0E6
:10637800CFFD4FF480700121BDE8084007F0F8BD5B
:1063880007B50223009303238DF804300348002344
:1063980069468DF8073007F013FA0EBD0008024071
:1063A80030B5124D8BB0002406A8069407940894C3
:1063B800099406F0D3FB00948DF804408DF805404D
:1063C8000294039404942846012469468DF81440E5
:1063D80006F095FB28460B212246062306F00AFC08
:1063E8002846214606F0D4FB0BB030BD0020014002
:1063F80010B5002104460122302000F025FEC0B966
:10640800012001F041F8002CB8BF4034E4B210215B
:106418002246302000F018FE012001F035F8302027
:106428001121224600F010FE0120BDE8104001F0C5
:106438002BB810BD10B5002104460122302000F011
:1064480003FEC0B9012001F01FF8002CB8BF40348A
:10645800E4B212212246302000F0F6FD012001F0BE
:1064680013F830201321224600F0EEFD0120BDE88C
:10647800104001F009B810BD38B5012205460C4698
:106488003020002100F0E0FDF0B9012000F0FCFF11
:1064980025EAE5725F2AA8BF5F223B21D2B23020ED
:1064A80000F0D2FD012000F0EFFF24EAE4725F2A39
:1064B800A8BF5F22D2B230203C2100F0C5FD0120E8
:1064C800BDE8384000F0E0BF38BD302810B50446BC
:1064D8000ADC10F17F0F02DB002802DB05E06FF019
:1064E8007E0404F5807400E03024002130200A4640
:1064F80000F0AAFDA8B90120E4B200F0C5FF4121CF
:106508002246302000F0A0FD012000F0BDFF302021
:106518004221224600F098FD0120BDE8104000F01D
:10652800B3BF10BD282810B5044609DC10F1180FB8
:1065380002DB002802DB04E06FF017047F3400E080
:106548002824002130200A4600F07EFDA8B9012049
:10655800E4B200F099FF53212246302000F074FD88
:10656800012000F091FF30205421224600F06CFDFC
:106578000120BDE8104000F087BF10BD08B53020ED
:106588000021012200F060FD60B9012000F07CFFCD
:1065980030203321402200F057FD0120BDE808409B
:1065A80000F072BF08BD10B530200021012200F0B4
:1065B8004BFD044660B9012000F066FF302033210E
:1065C800224600F041FD0120BDE8104000F05CBF0C
:1065D80010BD10B530200021012200F035FD044621
:1065E800A0B9012000F050FF34212246302000F0ED
:1065F8002BFD012000F048FF30203721224600F013
:1066080023FD0120BDE8104000F03EBF10BD402032
:10661800EEE640200EE708B500210122302000F008
:1066280013FD012000F030FF30203421024600F035
:106638000BFD012000F028FF30203721024600F032
:1066480003FD0120BDE8084000F01EBF08B5002189
:106658000122302000F0F8FC012000F015FF302066
:1066680034210C2200F0F0FC0120BDE8084000F0C5
:106678000BBF000000000000184B1949D3ED006A59
:1066880093ED017A00231A469FED166A03E0F0EEB7
:10669800476AB0EE677A505E05EE900AF8EEE57A42
:1066A8000133C7EE867A9BB218B204327F2877EEA0
:1066B800E67AECDD27EE077A07EEA77A0A49074A59
:1066C8000B80BDEEC77A002313605360C2ED027AD7
:1066D80017EE102A054B92001A607047E40D00204F
:1066E800E42900200000FA45143E0020B01A0020DA
:1066F8002DE9F84F2E4B2F4A19682F4B19B92F49FE
:1067080011602F4A02E02F4911602F4A1A602F4B5F
:10671800DFF8BCA0DFF8BC90DFF8BCB000221A801C
:10672800244A9846176830E007EB84036500B3F9FC
:10673800023007EE103AF8EEC77A013617EE900AE3
:1067480008F098FF18A3D3E9002308F0E7FF09F041
:106758007FFA29F815002AF8140037F9243007EED3
:10676800103AF8EEC77A013517EE900A08F082FF62
:106778000DA3D3E9002308F0D1FF09F069FA2BF83B
:10678800140029F81500A8F80060B8F8006034B2C1
:10679800FF2CC9DD00F05EF800F06AF801F09CF902
:1067A800BDE8F84F68E700BF9A9999999999E93F28
:1067B800A41A0020981A0020D0180020E6310020E2
:1067C800E62D0020E6390020E6350020143E0020A2
:1067D800E4250020E4290020E427002010B50B4C14
:1067E800204606F03AFC0A4B18600A4806F035FCC9
:1067F800094B1860FFF77CFF084B09490122204626
:106808009A81BDE8104006F0A9BC00BF10600240A4
:10681800A41A002088600240C01A0020E40D00205D
:1068280020800010014B1868704700BFB01A002084
:1068380008B5054B054819880022012309F05AFFBD
:10684800034B187008BD00BFC4010020CC250020F0
:10685800E820002003480449044A4FF4807309F0F3
:10686800C1BF00BFC8010020E4250020CA230020C2
:1068780003480449044A4FF4807309F0B3BF00BFCA
:10688800D4010020E4270020041C002038B5054668
:106898000C460135C1F3072100F004FEA8B2E1B2AD
:1068A80000F000FE00B238BD38B5044600F00EFD19
:1068B80001340546A0B200F009FDEDB2C0B240EACD
:1068C800052000B238BD37B50B0E8DF804300B0C1F
:1068D8008DF805300B0A8DF806308DF80710002466
:1068E80000E0284601AB451CE15C013400F0DAFD0C
:1068F800042CADB2F5D13EBD37B5002400E02846E2
:10690800451C00F0E3FC01ABADB2E0540134042CAB
:10691800F5D19DF805009DF80430000440EA0360B5
:106928009DF8073018439DF8063040EA03203EBD25
:1069380038B50446642000F0A7FD25786068AD00EE
:10694800EDB2257006F0A1FF237A40FA03F000F0BB
:1069580003000543104B257005F00F055A5D637859
:10696800D218D2B2D3B20132D2B2022A637001D89D
:106978000022A2705BB2012B03DD0123A370002368
:10698800637094F90130013303DAFF23A370002305
:10699800637094F9020038BDDE640408F7B504207A
:1069A8000121234F07F0B4FA02AD01214FF48040D2
:1069B800012407F0DDFA00264FF4B0733846694623
:1069C80045F8083D8DF804608DF8074006F0F8FE9C
:1069D8001020214607F09CFA782369461548009351
:1069E8008DF804608DF8074006F0EAFE0420214681
:1069F80007F08EFA21464FF4804007F0B9FA1C23BD
:106A08003846694600938DF804608DF8074006F013
:106A1800D7FE0220214607F07BFAB02306488DF8FE
:106A2800046069468DF80740009306F0C9FEFEBD74
:106A3800000802400010024000040240802108B50E
:106A4800034806F01CFFD0F1010038BF002008BD44
:106A58000004024008B54FF48071044806F00FFFA7
:106A6800D0F1010038BF002008BD00BF0008024077
:106A780008B5FFF7E3FF08B1FFF7ECFFC0B208BDA8
:106A880010B5642000F000FD1D48FFF751FF0446D3
:106A980010B91C4B187009E0FFF7DCFF30B9002C67
:106AA800184B01DD012200E0FF221A701648FFF79B
:106AB8003FFF164B1B78042B16D100281FD0144B10
:106AC8001A7806DD0132D2B20F2A1A7008D91022BC
:106AD80005E0013AD2B2102A1A7001D900221A70C0
:106AE800BDE81040FAF768BE00280A4B01D11870BB
:106AF80010BD02DD01221A7010BDFF221A7010BDF0
:106B080014020020A844002020020020483E002053
:106B1800AE3E0020E42D002007B50220012107F039
:106B2800F7F9012300938DF8043002238DF805301E
:106B38000448002369468DF806308DF8073006F0C2
:106B48003FFE0EBD0004024010B5084C0121002292
:106B5800204606F0AAFE40F2FF4000F095FC012115
:106B680020460A46BDE8104006F09FBE00040240D9
:106B780008B5FFF7E9FF00210A46302000F064FA63
:106B8800012000F081FC01210A46302000F05CFA67
:106B9800012000F079FC00210122302000F054FA95
:106BA800012000F071FC01210822302000F04CFA8D
:106BB800012000F069FC02210122302000F044FA93
:106BC800012000F061FC00210A46302000F03CFA68
:106BD800012000F059FC1B21CD22302000F034FAAE
:106BE800012000F051FC04210322302000F02CFA8F
:106BF800012000F049FC06210822302000F024FA88
:106C0800012000F041FC07210A46302000F01CFA60
:106C1800012000F039FC08218022302000F014FA0D
:106C2800012000F031FC1E21B022302000F00CFAC7
:106C3800012000F029FC05219122302000F004FAFF
:106C4800012000F021FC0D210322302000F0FCF986
:106C5800012000F019FC0E210022302000F0F4F988
:106C6800012000F011FC14218022302000F0ECF902
:106C7800012000F009FC0B218822302000F0E4F903
:106C8800012000F001FC30200C21822200F0DCF908
:106C9800012000F0F9FB12218822302000F0D4F9FD
:106CA800012000F0F1FB13218C22302000F0CCF9F8
:106CB800012000F0E9FB00210122302000F0C4F996
:106CC800012000F0E1FB0C210822302000F0BCF983
:106CD800012000F0D9FB0D210822302000F0B4F982
:106CE800012000F0D1FB0E210822302000F0ACF981
:106CF800012000F0C9FB0F210822302000F0A4F980
:106D0800012000F0C1FB00210A46302000F09CF968
:106D1800012000F0B9FB40210222302000F094F954
:106D2800012000F0B1FB00224121302000F08CF955
:106D3800012000F0A9FB30203F21D42200F084F983
:106D4800012000F0A1FB00210122302000F07CF995
:106D5800012000F099FB10210F22302000F074F977
:106D6800012000F091FB11210F22302000F06CF976
:106D7800012000F089FB12210022302000F064F984
:106D8800012000F081FB13210022302000F05CF983
:106D9800012000F079FB09213C22302000F054F951
:106DA800012000F071FB00210122302000F04CF995
:106DB800012000F069FB30203421024600F044F93C
:106DC800012000F061FB30203721024600F03CF939
:106DD800012000F059FB36210322302000F034F95D
:106DE800012000F051FB39210322302000F02CF95A
:106DF800012000F049FB3B213C22302000F024F91F
:106E0800012000F041FB3C210A46302000F01CF92B
:106E1800012000F039FB00210A46302000F014F967
:106E2800012000F031FB5121C022302000F00CF984
:106E3800012000F029FB30205221002200F004F943
:106E48000120BDE8084000F01FBB00BF2DE9F04F4E
:106E5800454E464D93B001214FF4001007F058F805
:106E6800304605F0FBFF4FF0C0630293404B03939D
:106E7800404B002404934FF400794FF400334FF44F
:106E880080684FF400674FF4005A4FF4807B304617
:106E980002A90C9301930997CDF8189005940794CB
:106EA800CDF82080CDF828A0CDF82CB00D9406F0B0
:106EB80061F822463046304906F0B7F830460121DD
:106EC80006F0BDF801210A464FF0402007F08EFA7F
:106ED800284605F0C3FF294A019B0392284A0C93D0
:106EE80004922846402202A9059209970294CDF8F7
:106EF80018900794CDF82080CDF828A0CDF82CB0B4
:106F08000D9406F037F8224628461E4906F08DF8FB
:106F18002846012106F093F842F210770122022157
:106F2800194807F063FA384600F0AEFA30460121F6
:106F380006F05BF80121284606F057F8384600F0BD
:106F4800A3FA0B238DF8443011A801238DF845408E
:106F58008DF846408DF8473000F01AFD384600F0AD
:106F680093FA13B0BDE8F08F1060024088600240C9
:106F78000C400040E6390020E63100200C3C00407F
:106F8800E6350020E62D0020003C00400248102194
:106F9800012206F0A1B800BF1060024013B502201C
:106FA800012106F0B5FF4FF410730E4C0093022335
:106FB8008DF804308DF8053001238DF80630204611
:106FC800002369468DF8073006F0FAFB20460621B3
:106FD800042206F075FC20460921042206F070FC04
:106FE8001CBD00BF0004024030B5154D85B001211D
:106FF8004FF4001006F0B0FF284606F077FC002397
:10700800ADF804304BF6FF73ADF806303323ADF816
:1070180008304FF48063ADF80A304FF48043ADF880
:107028000C3004AC074B2846012144F8103D06F00B
:10703800FFFC2846694606F087FC05B030BD00BF56
:1070480000540040801A060073B54FF496130646A4
:107058000D461446019304E0019B5A1E0192002B31
:1070680057D031484FF4003106F0FAFD0028F3D12B
:107078002D48012106F0E8FC4FF48053019304E009
:10708800019B5A1E0192002B45D02748274906F03C
:10709800D2FD0028F4D024483146002206F0ECFC4A
:1070A8004FF48053019304E0019B5A1E0192002B78
:1070B80033D01D481E4906F0BEFD0028F4D01A48FA
:1070C800294606F05CFD4FF48053019303E0019BD1
:1070D8005A1E01921BB31448164906F0ACFD00284D
:1070E800F5D01148214606F04AFD4FF49613019356
:1070F80003E0019B5A1E01929BB10B480E4906F012
:10710800AFFD0028F5D00848012106F0A9FC0020B1
:1071180008E0012006E0022004E0032002E0042049
:1071280000E005207CBD00BF0054004001000300C2
:1071380082000700800007000400001037B54FF4F4
:10714800961304460D46019305E0019B5A1E0192D1
:10715800002B00F09B8056484FF4003106F080FD6C
:107168000028F2D15248012106F06EFC4FF48053FA
:10717800019305E0019B5A1E0192002B00F08880C4
:107188004B484C4906F057FD0028F3D048482146A3
:10719800002206F071FC4FF48053019304E0019B38
:1071A8005A1E0192002B75D04148434906F043FD11
:1071B8000028F4D03E48294606F0E1FC4FF48053FD
:1071C800019304E0019B5A1E0192002B64D03848B9
:1071D8003A4906F045FD0028F4D03548012106F06B
:1071E80033FC4FF48053019304E0019B5A1E019233
:1071F800002B53D02E482F4906F01DFD0028F4D04F
:107208002B482146012206F037FC4FF480530193A6
:1072180004E0019B5A1E0192002B41D0244C2849BE
:10722800204606F01DFD0028F3D02046002106F078
:107238002BFC20460121238B06F012FC4FF48053CF
:10724800019304E0019B5A1E0192002B2AD0184892
:107258001C4906F005FD0028F4D0154806F091FCFD
:107268004FF480530193124A03E0019B591E019188
:10727800D3B113889B05F8D4012104460C4806F0C5
:1072880003FC0B48104906F005FD0EE001240CE054
:1072980002240AE0032408E0042406E0052404E0AC
:1072A800062402E0072400E0082420463EBD00BF73
:1072B8000054004001000300820007000400001091
:1072C80002000010400000100004001013B54FF435
:1072D80096130446019305E0019B5A1E0192002B68
:1072E80000F0B08061484FF4003106F0B9FC002886
:1072F800F2D15E48012106F0A7FB4FF480530193B9
:1073080005E0019B5A1E0192002B00F09D80574812
:10731800574906F090FC0028F3D05448A0210022D9
:1073280006F0AAFB4FF48053019305E0019B5A1E17
:107338000192002B00F08A804C484E4906F07BFCF5
:107348000028F3D0C4F30521484806F018FC4FF490
:107358008053019304E0019B5A1E0192002B77D0C1
:107368004248454906F07CFC0028F4D0E1B23F4889
:1073780006F005FC4FF48053019304E0019B5A1E6C
:107388000192002B66D039483B4906F069FC002879
:10739800F4D03648012106F057FB4FF4805301938F
:1073A80004E0019B5A1E0192002B55D02F4830490A
:1073B80006F041FC0028F4D02C48A121012206F057
:1073C8005BFB4FF48053019304E0019B5A1E01922A
:1073D800002B43D0254C2949204606F041FC0028C3
:1073E800F3D02046002106F04FFB20460121238BD5
:1073F80006F036FB4FF48053019304E0019B5A1EBC
:107408000192002B2CD019481D4906F029FC0028B0
:10741800F4D0164806F0B5FB4FF480530193134A95
:1074280003E0019B591E0191E3B113889905F8D433
:10743800012104460D4806F027FB0C48114906F0C7
:1074480029FC10E001240EE002240CE003240AE0E9
:10745800042408E0052406E0062404E0072402E0EA
:10746800082400E0092420461CBD00BF0054004049
:107478000100030082000700040000100200001051
:10748800400000100004001082B0002304E0019BBB
:1074980001330193009B01330093009B8342F6D391
:1074A80002B0704737B54FF4805304460D46019338
:1074B80004E0019B5A1E0192002B6ED03D484FF408
:1074C800003106F0CDFB0028F3D13A48012106F03F
:1074D800BBFA4FF48053019304E0019B5A1E0192BA
:1074E800002B5CD03348344906F0A5FB0028F4D0C3
:1074F8003048A021002206F0BFFA4FF480530193D0
:1075080004E0019B5A1E0192002B4AD029482B49BE
:1075180006F091FB0028F4D0C4F30521254806F0B5
:107528002EFB4FF48053019304E0019B5A1E0192F5
:10753800002B38D01F48224906F07DFB0028F4D0E4
:10754800E1B21C4806F01BFB4FF48053019303E0A3
:10755800019B5A1E019243B31648194906F06BFB6A
:107568000028F5D01348294606F009FB4FF4961376
:10757800019303E0019B5A1E0192C3B10D481149C2
:1075880006F06EFB0028F5D00A48012106F068FADB
:107598000D48FFF779FF00200AE0012008E00220EB
:1075A80006E0032004E0042002E0052000E00620B5
:1075B8003EBD00BF005400400100030082000700E8
:1075C8008000070004000010A0860100F7B54FF402
:1075D800805304460D461646019304E0019B5A1E4B
:1075E8000192002B75D041484FF4003106F038FB6A
:1075F8000028F3D13D48012106F026FA4FF48053C4
:10760800019304E0019B5A1E0192002B63D0374876
:10761800374906F010FB0028F4D03448A021002296
:1076280006F02AFA4FF48053019304E0019B5A1E96
:107638000192002B51D02D482E4906F0FCFA002863
:10764800F4D0C4F30521294806F099FA4FF4805381
:10765800019304E0019B5A1E0192002B3FD023485E
:10766800254906F0E8FA0028F4D0E1B21F4806F0F0
:1076780086FA4FF48053019304E0019B5A1E01924D
:10768800002B2ED019481C4906F0D5FA0028F4D052
:1076980000244FF4961710E0295D144806F06FFA9D
:1076A800019703E0019B5A1E0192E3B10F48134969
:1076B80006F0D6FA0028F5D00134E3B2B342EBD392
:1076C8000A48012106F0CCF90D48FFF7DDFE00203D
:1076D8000AE0012008E0022006E0032004E004207C
:1076E80002E0052000E00620FEBD00BF0054004077
:1076F800010003008200070080000700040000105A
:10770800A086010013B50520012106F001FC184CE4
:107718004FF4E053009302238DF804308DF80530C0
:107728002046002369468DF806308DF8073006F0AC
:1077380047F820460A21062206F0C2F820460C2106
:10774800062206F0BDF8062220460B21A4F50064A7
:1077580006F0B6F84FF4004320466946009306F059
:107768002FF820460F21062206F0AAF81CBD00BFFC
:10777800000802401FB50446FFF7CEF9FFF734FCB6
:10778800FFF7F6F9FFF7BEFF01214FF4004006F0BE
:10779800E3FB02940F4C1023ADF80230204600237F
:1077A8006946ADF80430ADF80C30ADF80030ADF8EE
:1077B800063006F000FD69464FF0402006F0CFFD88
:1077C8002046012106F07FFD4FF04020012106F000
:1077D8007AFD1FBD003C0040014B1860704700BF98
:1077E800000E0020704710B50A4A1379262B04D8DA
:1077F8000949C8540133137110BD074A0123591EA2
:10780800D45C0133272B5454F9D1034B83F8260059
:1078180010BD00BF000E0020E83D0020704710B5E5
:1078280004462078FFF7DFFF14F8013F002BF8D15A
:1078380010BD38B504460D46013D14F8010BEDB2F4
:10784800FFF7D1FF002DF7D138BD00BF014B1878E5
:10785800704700BF080E0020014B5878704700BFE2
:10786800080E0020024B187880F00100704700BF16
:10787800080E0020024B00221A705A70704700BF91
:10788800080E0020014B01221A707047080E0020D4
:10789800014B01225A707047080E002082B0002365
:1078A80004E0019B01330193009B01330093009B8B
:1078B8008342F6D302B0704707B50420012106F0D1
:1078C80027FB01214FF4804006F052FB4FF4007370
:1078D800009300238DF804300348012369468DF88E
:1078E800073005F06DFF0EBD000802400D4B07B5CF
:1078F8001A680D484FF47A73B2FBF3F20B4B013A56
:107908005A600B4AF02182F8231000229A6007225D
:107918001A60084B084A00930121084B04F07EFCCA
:107928000EBD00BFF0020020B43E002010E000E0D1
:1079380000ED00E00C040020F003002058030020B4
:10794800054B1A6812B11A68013A1A60034B1A6893
:1079580001321A60704700BF703E0020883E002048
:1079680082B0044B0190019A1A601A68002AFCD16F
:1079780002B07047703E0020704700BF40F0BE6004
:10798800024B40F42020D860704700BF00ED00E0B3
:10799800C37810B503B3164B4278DB688478DB43B1
:1079A800C3F30223C3F10401C9B202FA01F10F22A1
:1079B80042FA03F2C9B222400A430E4B017812017F
:1079C800CB18D2B283F8002303780122590903F0B7
:1079D8001F0302FA03F307E003780122590903F0B1
:1079E8001F0302FA03F32031024A42F8213010BD86
:1079F80000ED00E000E100E021F0604121F07F01AE
:107A0800014B08439860704700ED00E0044B1A6989
:107A180009B1104301E022EA00001861704700BF75
:107A280000ED00E0044B1A6804280CBF42F0040281
:107A380022F004021A60704710E000E00000000025
:107A4800034A044B1A60044A044B1A60704700BF8B
:107A58000000FA45B81A0020DB0FC93FB41A00200D
:107A6800034B00221A60034A034B1A60E8E700BF81
:107A7800E84400200000FA45B019002007EE100A7B
:107A8800024BF8EEC77AC3ED007A7047B0190020B0
:107A980038B510EE100A07F0EDFD0DA3D3E9002369
:107AA80007F03CFE084B044618680D4607F0E2FD57
:107AB8000B4602462946204607F05AFF08F010F9FF
:107AC800024B186038BD00BFB81A0020B41A002055
:107AD800182D4454FB2119402DE9F04F2DED048B4E
:107AE8009D4C89B04FF00008A1469C4B38F80350D4
:107AF8009B4B258038F803609A4B6680186807F01E
:107B0800B9FD8DA3D3E9002307F008FE08F0A0F81B
:107B18006368954AC018011101F580610905090DCE
:107B28006060C0F30B1008AF32F8203032F8212023
:107B3800616A238115FB02F0628115FB03F516FBD0
:107B480002F216FB03F607EB4103E0602561C0F380
:107B5800CF30C5F3CF356261A661C2F3CF32C6F329
:107B6800CF3623F8200C23F8105C23F8182C23F8C0
:107B7800086C7E4BA08301310B40002BE5832284E7
:107B8800668403DA013B63F003030133C9F8243048
:107B9800002B40F0C5807648764A774E774D694687
:107BA800042309F0DFF87648764A04A9042309F08B
:107BB800D9F87548754A02A9042309F0D3F8744A1C
:107BC800744806A9042309F0CDF8B4F9283007EE63
:107BD800903AB4F92A30B8EEE79A07EE903AB4F939
:107BE8002C30B8EEE78A07EE903AB4F92E30F8EE6A
:107BF800E79A07EE903AF8EEE78A68EE087A49EED7
:107C0800097A17EE900A07F035FD41EC100B09F0E0
:107C180039FF51EC100B08F063F868EEA87A49EECA
:107C2800A97A306017EE900A07F024FD41EC100B9A
:107C380009F028FF51EC100B08F052F868EE897A29
:107C480058EE297A28EE288A286009EE298A17EE44
:107C5800900A07F00FFD824618EE100A8B4607F0CF
:107C680009FD4BEC10AB41EC110B09F083FE51EC14
:107C7800100B08F035F8484B1860286807F0FAFC34
:107C88002FA3D3E9002307F0BBFF08B1434B2B60B8
:107C980096ED000AD5ED007A80EE270A404F87ED71
:107CA800000A09F039FE00B9FEE73B4E3D4D306849
:107CB80007F0E0FC24A3D3E9002307F02FFD824658
:107CC80028688B4607F0D6FC21A3D3E9002307F0E8
:107CD80025FD02460B465046594607F06DFB07F056
:107CE800FFFF2860306038682F4D07F0C3FC16A3EB
:107CF800D3E9002307F012FD824628688B4607F077
:107D0800B9FC13A3D3E9002307F008FD02460B468C
:107D18005046594607F050FB07F0E2FF28603860EC
:107D280008F10208B8F5007F7FF4DFAE09B0BDECBA
:107D3800048BBDE8F08F00BF39D6C56D305FC440F5
:107D48008DEDB5A0F7C6B03E9A9999999999B93F22
:107D5800CDCCCCCCCCCCEC3F1C0E0020CA230020D0
:107D6800041C0020B41A0020F864040803000080F2
:107D780008020020440E0020F0440020E4440020C3
:107D8800FC010020460E0020F0010020480E0020D3
:107D98004A0E0020E4010020D4440020BD37863577
:107DA800DC440020D8440020EC440020014B93ED33
:107DB800000A7047DC440020014B93ED000A70472D
:107DC800D4440020014B93ED000A7047EC44002096
:107DD800014B93ED000A7047D8440020014B93ED06
:107DE800000A7047F0440020014B93ED000A7047E9
:107DF800E4440020AFF3008010B5FEF78BF80020B4
:107E0800012324210246FEF7EFF8114B1C780020CD
:107E1800012C05D10146FEF7C0F92046002104E0F7
:107E28000721FEF7BAF901200721FEF7B6F9632208
:107E38001221C020FFF708F902200121FEF7ADF951
:107E4800FEF78AFA0120BDE81040FEF77ABA00BFB3
:107E58002C0F00200D4B1B78012B05D10C4B0D4A24
:107E6800196812688A181A600B4B1B78012B084B8B
:107E7800196805D1094A914207DD01321A60704735
:107E8800074A914201DD01321A607047483E0020DE
:107E9800AC440020443E00202C0F00207FD1F00885
:107EA800FF1FA1070E4B1B78012B05D10D4B0E4A66
:107EB800196812688A1A1A600C4B1B78012B094B37
:107EC80005D10B4A1968914208DC1A6070471A6894
:107ED800B2F57A2FDCBF4FF47A221A60704700BFE0
:107EE800483E0020AC440020443E00202C0F0020D7
:107EF80040420F00024B1A68024B1A60704700BFDD
:107F0800A83E0020AC4400202DE9F04F8246584896
:107F18008BB0B0FBF1F00C4607F08AFB41EC100B7C
:107F280009F0F6FB51EC100B07F0BAFEC307074641
:107F380048BF471E04FB07F007F07AFB46A3D3E9C6
:107F4800002307F015FD04460D4645EC104B09F0DB
:107F5800DFFB59EC108B204642464B46294607F07A
:107F680029FACDE904014946404607F099FE3CA3A9
:107F7800D3E900230990DDE9040107F04BFE00284E
:107F88003DD1002401234FF015092246984620468A
:107F9800DFF8E4B003E0234642462C46B04600FB37
:107FA80004355D452ED800FB0826DDE904012EA323
:107FB800D3E9002307F02EFE30BBDDE904230020BF
:107FC8002C4907F0D5FC41EC100B0390029109F005
:107FD8009FFB0398029953EC102B8DED060B07F0CD
:107FE800E9F909F1FF39CDE904015FFA89F9DDE919
:107FF800060107F055FEB9F1000FCCD104E00125C8
:10800800002601E025464646099BD9B2BAF1000F81
:108018000BD132462B465046FDF7E6FF012300936D
:10802800504651463A46534609E032462B4601200F
:10803800FDF7DAFF0120009001463A460023FEF7DB
:10804800C6F8FEF789F901200BB0BDE8F04FFEF73E
:1080580078B900BFAFF300800000000084D77741F3
:10806800956479E17FFDA53DBBBDD7D9DF7CDB3DBC
:1080780000E9A4350000F03FFFFF0F0038B5384B8A
:108088001B78022B374B03D1374A12681A6038BD68
:108098001968364B364A1B68364CCB189342236016
:1080A80018DC0020FFF730FF01202168FFF72CFFC4
:1080B800314B1C780020012C05D10146FEF76DF8E4
:1080C8002046002104E00721FEF767F80120072178
:1080D800FEF763F8294B1B78022B14D1284B294D46
:1080E8001A68204C2B68D31822689A420BDA264B60
:1080F8001B78012B07D1254B186800F0A9F82268D6
:108108002B68D31823601D4B1B78012B0FD11C4BF8
:108118001A681C4B1B68D318124A12689A4206DA6E
:10812800194B1B78012B02D10A2000F091F80C4A58
:108138001378012B13D116490888164909888842F3
:108148000DD902211170144A12788A4204D1134AB7
:108158001370134B00221A80124B00221A6038BD8C
:1081680044460020AC440020A83E0020C44400201F
:1081780080D1F008C84400202C0F0020483E002081
:10818800983E0020443E0020903E0020603E0020A3
:10819800244500200C480020C0440020600E002028
:1081A800620E0020AC0E002008B5FEF747FC094B14
:1081B8005A78187002435A701AB19A7801329A7034
:1081C80030B99B78034A012B02D90023537093706E
:1081D80008BD00BF4C0E002007B50420012105F0A2
:1081E80097FE4FF46043009301238DF80430022377
:1081F8008DF805300448002369468DF806308DF85F
:10820800073005F0DDFA0EBD00080240084B1A6879
:108218004FF47A73B2FBF3F2064B013A5A60064AFE
:10822800F02182F8231000229A6007221A60704712
:10823800F002002010E000E000ED00E0034B5A6877
:1082480012B15A68013A5A60704700BF4C0E0020BC
:10825800024B58605A68002AFCD170474C0E002027
:1082680030B585B004460D4601A85C490A220BF0DA
:1082780097FE5B4B1B78032B10D8DFE803F0020551
:10828800080B01A8574907E001A8574904E001A8CD
:10829800564901E0564901A80BF06CFF04AA1319CE
:1082A80013F80C3C5D19EDB22F2D01D80A3502E008
:1082B800392D01D90A3DEDB204AB1C194FF6FF70F8
:1082C80004F80C5CFCF77EFD0020FCF77DFE0DF148
:1082D80003050F24204623345A21002315F8012FC3
:1082E800A4B2FCF78BFEB4F5A57FF3D164205A2124
:1082F8002C220023FCF782FE0023CD205A212C22B9
:10830800FCF77CFE0020FCF75DFD354B1B78032B4A
:1083180062D8DFE803F002284B5601A931480BF078
:1083280029FF0A2200212F480CF0C8F8314A324BA5
:1083380012781860012A06D1304A904201DC0132D5
:108348001A602F4A06E0B0F5FA5FBCBF4FF4FA5244
:108358001A602C4A1B689342C4BF274B1A602A4BE9
:108368001A682A4B20E001A91F480BF003FF0A22D4
:1083780000211D480CF0A2F81E4A254B12781860FF
:10838800012A06D11D4A904201DC01321A601C4ABA
:1083980006E0B0F5FA5FBCBF4FF4FA521A60194A0A
:1083A8001B68934218DD1A4B1A6015E001A90F48A3
:1083B8000BF0E0FE0D4800210A220CF07FF8154B67
:1083C80009E001A90A480BF0D5FE094800210A2254
:1083D8000CF074F8104B186005B030BDD5A805082E
:1083E800A63E0020743E00209C3E0020B1440020A0
:1083F800643E00202C0F0020B03E00203F420F00BA
:1084080080D1F00840420F00A83E0020AC44002074
:10841800CC440020A4440020603E002010B50D4B41
:108428000D4C1A680D4821460BF07CFE0C4B0D488C
:108438001A6821460BF076FE0B4B0C481A68214649
:108448000BF070FE0A4B0B481A682146BDE8104035
:108458000BF068BEB03E0020DFA80508743E00207F
:10846800CC4400209C3E0020A4440020B1440020BD
:10847800603E0020643E00209FED010A704700BF67
:10848800000000009FED010A704700BF00000000D7
:108498009FED010A704700BF000000007047704759
:1084A800044B18B1012801D1034A00E0034A1268BD
:1084B8001A607047AC440020983E0020A83E002077
:1084C80010B9034B18687047024B1868704700BF13
:1084D800B03E0020A83E002010B9034B1868704732
:1084E800024B1868704700BFCC440020983E00201B
:1084F80008B54FF49570FEF7D7F940F26523C31A13
:10850800584240EB030008BD08B5C620FEF7CCF979
:1085180040F28D13C21A504240EB020008BD4FF4DE
:10852800957040F26521FEF7B1B9C62040F28D1171
:10853800FEF7ACB9704760EEA00AB7EE007AF0EE2D
:10854800606A70EE077A40EE006A47EEA70A36EED8
:10855800C77A08B5C7EE200A10EE900A07F08AF825
:108568000022084B07F0DAF80022074B06F024FF38
:1085780007F0B6FB07EE900AFDEEE77A17EE900AD1
:108588009F3008BD000059400000E03F38B52DED90
:10859800028BF7EE008AB0EE608A70EE288A10EE41
:1085A800900A28EE088A07F065F808EEA88A0022E3
:1085B8000F4B07F0B3F8044618EE100A0D4607F003
:1085C80059F802460B462046294607F0D1F9002201
:1085D800084B06F0F1FE07F083FB07EE900AFDEE6C
:1085E800E77A17EE900A7730BDEC028B38BD00BFF2
:1085F800000069400000E03FF0B5694D2DED068BA5
:1086080095E80F008DB008AE103586E80F000FCD45
:1086180001AC0FC495E807004FF6FF7384E8070024
:108628009F2077216422FAF772F8A020772164222C
:108638004FF6FF73FAF76BF89E20772164224FF606
:10864800FF73FAF764F89F20762164224FF6FF73D0
:10865800FAF75DF84FF6FF73782164229F20FAF746
:1086680056F80020FBF76DFC9F2077216522FCF768
:10867800EBFB9F2077216422FCF7E6FB07AD0C3665
:10868800F7EE009A0435F7EE008A95ED009A4FF45C
:108698009674B0EE68AA18EE900A06F0EBFF3EA3B7
:1086A800D3E9002307F03AF807F01AFB08EE900A1E
:1086B80038EEE98AB0EE490AF0EE480AFFF73BFFC8
:1086C800B0EE490AF0EE480A0746FFF75FFFBFB26F
:1086D80081B20F223846FBF7FFFC013CDBD14FF497
:1086E8009674F7EE008A18EE900A06F0C3FF2AA3E4
:1086F800D3E9002307F012F807F0F2FA08EE900A1F
:1087080039EEE88AB0EE490AF0EE480AFFF713FF9F
:10871800B0EE490AF0EE480A0746FFF737FFBFB246
:1087280081B20F223846FBF7D7FC013CDBD1B542BA
:10873800A8D16C4607AE043494ED009A4FF4C8757E
:10874800F7EE008A18EE900A06F094FF12A3D3E918
:10875800002306F0E3FF07F0C3FA08EE900A38EEAC
:10876800CA8AF0EE490AB0EE480AFFF7E4FEB0EE16
:10877800480AF0EE490A0746FFF708FFBFB281B280
:1087880000223846FBF7A8FC013DDBD1B442D2D128
:108798000DB0BDEC068BF0BD295C8FC2F528F03F0B
:1087A800F8A40408121A06EE902A081AB8EEE67A17
:1087B80006EE900AF8EEE67AC7EE277A9FED047A7D
:1087C80067EE877AFDEEE77A17EE900A704700BFEA
:1087D8000000A0438A1A06EE902A081AB8EEE67A34
:1087E80006EE900AF8EEE67AC7EE277A9FED047A4D
:1087F80067EE877AFDEEE77A17EE900A704700BFBA
:108808000000484370B506460D460024610704D5AC
:10881800A0B231462A46FBF75FFC0134B4F5A07FCD
:10882800F4D170BD70B506460D460024600704D526
:10883800A1B230462A46FBF74FFC0134C82CF5D1CB
:1088480070BD114B11481B781149124A0068012B61
:10885800114B09D1126808601A60104B1A68104B46
:108868001A60104B1A680CE01268D2011A600B4BA0
:108878001A680B4BD2011A600A4B1A68C0010860CB
:10888800D201094B1A6070472C0F0020B03E00201F
:10889800A83E0020CC440020983E0020A44400209C
:1088A800443E0020803E0020C4440020024B1A6849
:1088B800024B1A60704700BFA83E0020AC4400205D
:1088C80008B5FFF7BEFFBDE80840EFE770B5002127
:1088D8000A222A482A4D2B4E2B4C0BF0EFFD002183
:1088E8000A22286029480BF0E9FD00210A2230609D
:1088F80027480BF0E3FD00210A22206025480BF0F1
:10890800DDFD254B326818602B68D31A06EE903AC5
:108918002368B8EEE67A06EE903AF8EEE67AC7EE05
:10892800277A17EE900A06F0A5FE00221B4B06F0E8
:1089380043FD07F0B5F983B207EE903AB8EE677ACF
:10894800F4EE007A67EE277A154A164B1080FCEE93
:10895800E76A16EE901A8AB206EE902AB8EEE67A20
:10896800198077EEC77AF5EEC07AF1EE10FA01DDDC
:1089780001321A80BDE87040A2E700BF743E0020B3
:10898800B03E0020CC440020A44400209C3E00209F
:10899800B1440020643E0020603E00200000E03F1B
:1089A8000C4800208C4800200022F0B513462026F1
:1089B80003254FF02C0C00E02646303EF6B2174651
:1089C8000132092E10F8014B0AD897FBF5F605FB82
:1089D80016772FB9CE1801F803C07470023301E07E
:1089E800CC540133092AE7D12022CA54CB18482293
:1089F8005A707A229A700022DA70F0BDF0B51F46DC
:108A0800144B1E788DB005460C4606B3A6F1040C2F
:108A1800DCF1000646EB0C06CEB90F4908A80BF0AE
:108A280081FB08A86946FFF7BFFF0C496A4604A8FE
:108A38000BF078FBBDF84800FCF7C4F93846FCF7A2
:108A4800D7F92846214604AA3346FCF7F5FA0DB0B3
:108A5800F0BD00BF483E0020F69F050841A6050866
:108A68002DE9F04F7E4B2DED068B93ED008A78EEC5
:108A7800087A7C4B85B017EE900A1C6806F0FAFD60
:108A880080462046894606F0F5FD68EE088A41ECE6
:108A9800100BF7EE009ACDE9020108F0E1FD78EE3F
:108AA800A97A57EC106B17EE900A06F0E3FD3246F0
:108AB8003B4682468B464046494606F02FFE024614
:108AC8000B465046594606F075FC07F009F979EE51
:108AD800E88A09EE100AC8EE898ADFED637A9DED0F
:108AE800020B68EEA78A08F0BBFE404653EC102B39
:108AF800494606F013FE064619EE100A0F4606F020
:108B0800B9FD02460B463046394606F031FF574B51
:108B1800002206F003FE07F0E3F809EE100A69EEFA
:108B2800097A48EEA87AB1EE49AA88EEA77A504B9E
:108B38005C60D8608AEE27AA83ED008AC3ED028ABA
:108B480083ED047A83ED05AA4A4B1B78033B042B7B
:108B58006ED8DFE803F00312254E3C0018EE900AA9
:108B680006F088FD044619EE100A0D4606F082FD4F
:108B7800CDE90001404841490DE017EE100A06F022
:108B880079FD04461AEE100A0D4606F073FDCDE98C
:108B9800000139483A4922462B460BF0C3FA47E010
:108BA80018EE100A06F066FD41EC100B08F0E4FE22
:108BB8000022344B51EC100B06F0B0FD07F090F892
:108BC80006F058FD02460B462B482F492EE018EEBA
:108BD800100A06F04FFD1EA3D3E9002304460D46F4
:108BE800DDE9020106F09AFDCDE900012248274996
:108BF800D1E718EE100A06F03DFD17A3D3E90023CC
:108C080007F01CF8DFED227A002818BFB0EE678A5B
:108C180078EE297A79EEC89AC7EEA99A19EE900AE1
:108C280006F028FD02460B4613481A490BF07AFA5B
:108C3800114C00230220CA212246FCF7FDF900232B
:108C4800237005B0BDEC068BBDE8F08FAFF3008054
:108C5800F6285C8FC2A54C40AE47E17A14AEEF3FD0
:108C6800284500202C4500200000484200004940CB
:108C7800EC470020C0440020FA440020E5A805087D
:108C8800F5A80508000034C005A9050817A90508B6
:108C9800A4707D3F33A905082DE9F0434FF47F7098
:108CA8008DB0FDF701FE00271FFA80F86BE04FEA50
:108CB800C7091FFA89F909F580691FFA89F0FEF7D3
:108CC80005FB60F3070409F1010080B2FEF7FEFA24
:108CD80060F30F2409F1020080B2FEF7F7FA60F39F
:108CE800174409F1030080B2FEF7F0FA60F31F643D
:108CF80009F1040080B2FEF7E9FA60F3070609F10A
:108D0800050080B2FEF7E2FA60F30F2609F10600CB
:108D180080B2FEF7DBFA09F1070960F307051FFACD
:108D280089F0FEF7D3FA60F30F25B0B206F090FC95
:108D380000221B4B06F0F2FC06F0D2FF06F09AFC6C
:108D4800CDE90001A8B206F083FC11A3D3E9002302
:108D580006F030FB10A3D3E9002306F009FE06F065
:108D6800BFFF06F087FC2246CDE902010D4905A8A0
:108D78000BF0D8F9C1B205A803F0FAF80120FFF703
:108D880067FA0137BFB2B84591DA0DB0BDE8F08394
:108D980000000000C0FFDF40E17A14AE47C1664022
:108DA8000000F03E3EA9050808B50021C620FDF7E1
:108DB8006DFD4FF495700021BDE80840FDF766BDD4
:108DC800024B4FF6FF721A80704700BFF84400202C
:108DD80000200146C82240F23F13FBF7B7BA07B597
:108DE8000DF1070003F0C5F89DF807000EBD08B5A2
:108DF800FFF7F5FF0028FBD108BD30B5044687B062
:108E080010EE100A0D4606F035FC02460B4601A886
:108E180005490BF087F92046294601AA0023FCF7EB
:108E28000BF907B030BD00BF51A9050808B50848BF
:108E380003F028FF0648022103F0F5FF0028F9D0C7
:108E4800034803F04BFF07EE900AB8EE670A08BD27
:108E58000020014010B50C4C00232DED028B23801F
:108E68009FED0A8A06E0FFF7E1FF238838EE008AC3
:108E7800013323802388182BF5D99FED050A28EEA6
:108E8800000ABDEC028B10BD143E0020000000005B
:108E9800ACC8683910B54FF4C770FDF705FDDB287D
:108EA80005D14FF4C870FDF7FFFC84B219E041F218
:108EB800E104214644F20100FDF7E8FC44F2010018
:108EC800FDF7F2FCA04214BF80244FF4007421B2D5
:108ED8004FF4C870FDF7DAFC4FF4C770DB21FDF7DB
:108EE800D5FC204610BD024B00221A70704700BF07
:108EF8002C480020014B01221A7070472C48002092
:108F0800014B00221A60704724450020014B187855
:108F1800704700BF2C4800200030024B18BF0120CA
:108F2800187070472D4800200E4B1A680E4B1A60B7
:108F38000E4A002313700E4A13700E4A0121117055
:108F48000D4A4FF6FF7010800C4A13700C4B1A78BC
:108F58000C4B002A14BF052204224FF080401A70DF
:108F680005F037BCA83E0020AC440020903E00200D
:108F78002C4800200E0E0020F84400204446002013
:108F8800180E0020190E002070EEA10A88B030EEED
:108F9800010A08B0704770EEE10A88B030EE410A65
:108FA80008B07047F0EE407A20EEA10A60EE810A20
:108FB80047EEA10A88B017EE810A08B07047D0B50D
:108FC80061EEA17A41EE017A2DED048B17EE900A3D
:108FD80088B0B0EE409AF0EE609AF0EE418AB0EEBA
:108FE800618A06F047FB0022002306460F4606F07A
:108FF800FDFDE8B969EE887A49EE287A29EE088AF3
:1090080017EE900A06F036FB32463B4606F0B0FCF7
:1090180019EEA88A06F064FE044618EE100A06F057
:1090280029FB32463B4606F0A3FC06F059FE01E058
:109038000448044600EE900A00EE104A08B0BDEC61
:10904800048BD0BD0050C347F0EE407A86B020EEC6
:10905800200A67EE810A06B07047064B93E80300C2
:1090680084B004AB03E90300DDED030A9DED020AB9
:1090780004B0704790480020F7EE007A77EEC07A87
:1090880020EE022A20EE210A07EEA00AF0EE420A9C
:1090980047EE810A88B008B0704770B56D4B2DED6A
:1090A800068B1A786C4B94B00E468DED020ACDED06
:1090B800030A22B91A68802392FBF3F200E01A68C7
:1090C800664C012E236C616CDFED659AB7EE00AA41
:1090D80051D002D3022E60D154E0D21A07EE102AE2
:1090E800CB1AB8EEC79A07EE103AF8EEC77AD4ED65
:1090F800000A89EE279A94ED011AD4ED021A94ED2C
:10910800032AB0EE490AFFF7B7FF8DED000ACDED4F
:10911800010A9DE8030006ABD4ED040A94ED051A94
:10912800D4ED061A94ED072A83E80300B0EE490A45
:10913800FFF7A2FF8DED000ACDED010A9DE80300BF
:1091480008AB83E80300D4ED0C0A94ED0D1AD4EDB6
:109158000E1A94ED0F2AB0EE490AFFF78DFF8DED38
:10916800000ACDED010ADDED068A9DED078A04AB04
:109178009DE803000EE0D4ED008A94ED018A08AB67
:10918800103405E0D4ED028A94ED038A08AB183454
:1091980094E8030083E8030003E0B0EE698AF0EE88
:1091A8004A8ADDED030A9DED020A30EEC88A70EEA8
:1091B800688A9DED081ADDED091ACDED0C8A8DED52
:1091C8000D8AFFF7EFFE8DED000ACDED010A9DE84F
:1091D800030010AB83E80300DDED111A9DED101AB2
:1091E80079EEE11A3AEE411AB0EE680AF0EE480A52
:1091F8008DED0E1ACDED0F1AFFF7E1FE8DED000A89
:10920800CDED010A9DE803000AAD6C4685E8030030
:109218008EB99DED040ADDED050A9DED0A1ADDED16
:109228000B1AFFF7BFFE8DED000ACDED010A9DE890
:10923800030085E803000AAB93E8030014AB03E9D5
:109248000300DDED130A9DED120A14B0BDEC068B88
:1092580070BD00BF2C0F0020AC4400204048002007
:109268000000000010B5244C4FF496702168FDF7FB
:109278002AFB61684FF49870FDF725FBA1684FF44D
:109288009A70FDF720FBE1684FF49C70FDF71BFB1B
:1092980021694FF49E70FDF716FB61694FF4A070C9
:1092A800FDF711FBA1694FF4A270FDF70CFBE16912
:1092B8004FF4A470FDF707FB216B4FF4A670FDF780
:1092C80002FB616B4FF4A870FDF7FDFAA16B4FF438
:1092D800AA70FDF7F8FAE16B4FF4AC70FDF7F3FAFA
:1092E800216C4FF4AE70FDF7EEFA616C4FF4B0707C
:1092F800BDE81040FDF7E7BA4048002010B54FF42C
:109308009670FDF7F9FA224C20604FF49870FDF73B
:10931800F3FA60604FF49A70FDF7EEFAA0604FF42C
:109328009C70FDF7E9FAE0604FF49E70FDF7E4FAEF
:1093380020614FF4A070FDF7DFFA60614FF4A2706E
:10934800FDF7DAFAA0614FF4A470FDF7D5FAE061F1
:109358004FF4A670FDF7D0FA20634FF4A870FDF71C
:10936800CBFA60634FF4AA70FDF7C6FAA0634FF416
:10937800AC70FDF7C1FAE0634FF4AE70FDF7BCFACC
:1093880020644FF4B070FDF7B7FA606410BD00BFF9
:109398004048002008B5FFF7ABF810B1BDE8084019
:1093A800ACE708BD70B500F58065A8B2FDF78EFF83
:1093B800294C2070681C80B2FDF788FF6070A81CDB
:1093C80080B2FDF783FFA070E81C80B2FDF77EFF36
:1093D800E070281D80B2FDF779FF002660F30706CC
:1093E800681D80B2FDF772FF60F30F26B6B207EE74
:1093F800906AB8EE677ADFED197A194B67EE277A2B
:10940800A81DC3ED007A80B2FDF760FF002607357E
:1094180060F30706A8B2FDF759FF60F30F26B6B24E
:10942800A6F5FE46FF3E07EE106AF8EEC77A17EE7D
:10943800900A06F01FF906A3D3E9002306F098FA6C
:1094480006F04EFC074B22681860074B9A6170BD06
:10945800CDCCCCCC0C5FC440304600200000803717
:10946800284500202C450020EC47002013B5044671
:10947800002844D0264B18880419A4B222B2002A26
:1094880005DB40F23F139A42C8BF1C4600E00024A7
:10949800FAF736FEA0B24EF29C71FAF743FE1C4B67
:1094A8001C801C4B188824B2604306F0D1F816A320
:1094B800D3E9002306F05CFA0022174B05F07CFF85
:1094C80006F00EFC07EE900AFCEEE77A17EE900A1B
:1094D800C00080B2FFF766FF4FF6FF7300930F4B93
:1094E8000520DC219A690023FFF788FA0C4B0D4808
:1094F8001A780D4902B0BDE81040FFF7B1BA02B0C2
:1095080010BD00BFAFF300800000000000F0734002
:10951800F84400200C4800200000E03FEC47002001
:10952800C0440020284500202C4500202DE9F04F9C
:10953800354D2DED088B2B78022BBDB009D1334B5F
:109548001A68334B42F210701A60FDF79DFF00F065
:1095580028BE304B1B78B7EE00AADFED2FBA002BE0
:1095680049D02E4E2E4C3068C00080B2FFF71AFF4B
:1095780022782C482C49FFF773FA2C4B2C49D3F846
:109588001880D3F804A00988306893ED009A79EE22
:109598000A8A7AEE497AD3ED029AC8EEA78A00229F
:1095A80093ED038A93ED04BAD3ED05AA214BF4EEAB
:1095B8006B8A9A60DA600022F1EE10FAC8BFF0EE0A
:1095C8006B8AF4EE4A8AF1EE10FA48BFF0EE4A8A46
:1095D80088421A610ADD022129702178022902D104
:1095E80001211975DA820D4B00221A600B4B1A689B
:1095F80001321A6017E2104B1A78054BF2B91A6853
:10960800802392FBF3F81BE044460020A83E00208C
:10961800AC440020180E0020003C1C4624450020C5
:10962800C0440020284500202C450020EC4700209D
:109638000C4800204C0E00202C0F0020D3F800808E
:10964800FEF7B4FBCE4D85ED060AFEF7B5FBA8691B
:1096580085ED070A10EE104A06F00CF8064620467B
:109668000F4606F007F841EC100B41EC180B07F019
:10967800F7FF5BEC10ABB0EE480AF0EE680A08F0B2
:10968800EFF852465B46304639468DED040B06F03E
:1096980045F806F025FBDFEDBB8A07EE900A9FED43
:1096A800BA8A17EEA88AB94CDDE9042384ED008A4A
:1096B8003046394606F032F806F012FB00EE900A02
:1096C80060EEA80AB0EE480A0021B148C4ED010ACC
:1096D800FFF7E3FC8DED0A0ACDED0B0A0AAA92E822
:1096E8000300AC4B83E8030093ED018ADFEDAA7A0F
:1096F800B4EE6B8AF1EE10FAC8BFB0EE678ADFED00
:10970800A77AB4EE678AF1EE10FA48BFB0EE678A1E
:10971800FDEE007AB4EEE78AF1EE10FAD3ED009A86
:1097280008DDB5EE408ADFED9E7AF1EE10FA48BF0B
:10973800B0EE678A68EE088ADFED9A7AB0EE68BA0A
:1097480009EEA9BA19EE900AB5EE40BAF1EE10FA90
:1097580008BFB0EE67BA05F08DFF0022924B0646AF
:109768000F4605F027FE044618EE900A0D4605F050
:1097780081FF224682468B462B462046294605F025
:10978800CDFF52465B4605F017FE41EC100B08F082
:1097980079F9002230463946834B8DED040B05F0EC
:1097A8000BFE02460B4605F0B9FF52465B4605F034
:1097B80003FE41EC100B08F065F9DDE9040155ECF6
:1097C800104B06F08DFA294608EE900A204606F05E
:1097D80087FA09EE100A88EE899A744CF1EE48AAC5
:1097E800CAEE8BAA89EE8BBA19EE100A05F042FF71
:1097F8005DA3D3E9002306F003FADFED6D7A0028B4
:1098080018BFB0EE679ADFED6B7A6AEEA77AB4EE0E
:109818004A9ADFED698AF1EE10FA17EE900AC8BF8E
:10982800B0EE689A05F026FFDFED647A4BEE4B7ACE
:109838004AEEEA7A06460F4617EE900AC4E902672E
:1098480005F018FF47EC106B41EC110BC4E900015F
:1098580008F090F851EC100B06F042FAB4EE4A9A70
:10986800F1EE10FAA8BFB0EE689A7AEE497A79EE6E
:109878000A8A534BC8EEA78A1B78DFED477AF4EEC5
:109888006B8AF1EE10FAC8BFF0EE678AF4EE4A8AE6
:10989800F1EE10FAF7EE007A48BFF0EE678A022B75
:1098A80080F0004A40F0B380464B1B78002B00F054
:1098B800AE80454B454C1D682C40002C03DA013C1A
:1098C80064F00704013419EE100A05F0D3FE0022F3
:1098D8003F4B05F023FF06F0E3F906468146504664
:1098E80005F0C8FE22A3D3E9002305F017FF22A341
:1098F800D3E9002305F060FD06F0D2F9354B204985
:10990800C3F8008001EBC403C8F3072283F82120C1
:10991800C8F3074283F8222083F8246083F82600DE
:109928004FEA1862C6F30726C0F3072083F82080A1
:1099380083F8232083F8256083F82700264B08271F
:109948001B8895FBF7F7BF019D42BFB250DD07F5B5
:10995800806080B220314022FDF738FE0546E8B32A
:10996800FEE700BFAFF300802D431CEBE2361A3F41
:10997800CDCCCCCC0C5FC44000000000C0FFDF4061
:109988004C0E00200000F04200008C42904800205D
:10999800404800203C460020003C1C46003C1CC6B9
:1099A800CDCC4C3D5F7089300000494018480020FC
:1099B80017B7D1380AD7233D72F97F3F17B7D13986
:1099C800483E00202C480020244500200700008045
:1099D8000000F040304600200C4800209E4E4FF416
:1099E8007F70B6F90010FCF751FF9C4B35601D7075
:1099F800072C08D107F58067B8B299494022FDF7CE
:109A0800E5FD00B1FEE7944B1A6801321A60FEF7D3
:109A1800E5F9944C84ED020AFEF7E6F984ED030AB1
:109A2800FCF700FF20618F4C8F49424634A80AF0AA
:109A380079FBA06805F01EFE02460B4624A88B4958
:109A48000AF070FBE06805F015FE02460B4628A8F0
:109A580087490AF067FB1BEE100A05F00BFECDE9FB
:109A68000601DDE9062383492CA80AF05BFB1AEE00
:109A7800900A05F0FFFDCDE90401DDE904237E49E4
:109A880030A80AF04FFB19EE900A05F0F3FD0246E4
:109A98000B4610A879490AF045FB18EE100A05F0A4
:109AA800E9FD06460F4632463B46754914A80AF0BA
:109AB80039FB19EE100A05F0DDFDCDE90801DDE9F5
:109AC8000823704918A80AF02DFB504605F0D2FD6E
:109AD80082468B4652465B466B491CA80AF022FB1D
:109AE80018EE900A05F0C6FD02460B4620A8674905
:109AF8000AF018FB0CA8664922690AF013FBB5EEB8
:109B0800C08AF1EE10FADFED63AA37D5404605F0BA
:109B18009FFD4BA3D3E9002305F000FEF1EE487A40
:109B2800044617EE900A0D4605F0A4FD02460B46C2
:109B38002046294605F0F2FD02460B4642A1D1E92E
:109B4800000105F015FF06F0CBF89FED537A07EEFC
:109B5800900AF4EEC77AF1EE10FAC6BFC7EEAA7AF9
:109B68004E4C4F4CF4EEEA7AF1EE10FA36DD9FEDEA
:109B7800497A4C4D4C4CC7EE877A32E034A3D3E98E
:109B880000233046394605F0C9FD044640460D46D7
:109B980005F05EFD2AA3D3E9002305F0BFFD0246C8
:109BA8000B462046294605F0E3FE06F099F807EE35
:109BB800900AF4EECA7AF1EE10FA46BF67EEAA7A76
:109BC8003A4C3B4CF4EEEA7AF1EE10FA08DD9FEDE0
:109BD800317A384D384CC7EE877A02E0314D00E0D3
:109BE800344D17EE900A05F045FD2A46CDE90001EF
:109BF80038A8324902940AF095FA314B1C68314B67
:109C08001D68184BA845CCBF00260126A045D8BF23
:109C180000261E662C4B1B78013BDBB2012B00F2A1
:109C2800B2822A4B1B78072B00F2AD82DFE813F0D3
:109C38005000AB02E2003201B8010D026E022802A8
:109C48001F85EB51B81E1940000000A2941A6D42FE
:109C58000000000080842E41244500202C4800206C
:109C68006C0E00204C0E00206BA9050875A905088C
:109C780080A905088BA9050895A905089FA90508C5
:109C8800AAA90508B5A90508C0A90508CBA905080A
:109C9800D7A9050800007A44002474495CA905087E
:109CA80059A9050870AA050865A9050862A9050843
:109CB8005FA905088FA1050868A90508E4A9050892
:109CC800B03E0020CC440020483E0020C044002084
:109CD800A54B1C78002C40F056820220FBF774F943
:109CE8004FF6FF70FBF784F81F20FBF76BF819217C
:109CF8009E4A23462D20FBF79FF94FF6FF70FBF78E
:109D080077F82046FBF75EF80F20B42142464FF65D
:109D1800FF730094FEF772FE0F206E2124AA2346DB
:109D2800FBF78AF9A0206E210DEB00022346FBF712
:109D380083F90F20382118AA2346FBF77DF9A020C4
:109D480038211CAA2346FBF777F90F205C212CAA9F
:109D58002346FBF771F9A0205C2130AA2346FBF7C4
:109D68006BF90F204A2110AA2346FBF765F9A020BA
:109D78004A2114AA2346FBF75FF90F209B212346AB
:109D880020AAFBF759F97A4B1B78012B05D10F2034
:109D9800842138AA2346FBF74FF9764B1B69B3F5A4
:109DA8007A7FCCBF4FF4FC604FF47840FBF720F883
:109DB8000023A0209B210CAAFBF73EF96E4B1B78D1
:109DC800012B08D14FF4FC60FBF712F84FF48C70AC
:109DD80002216A4A07E04FF6E070FBF709F8684A83
:109DE8004FF48C7002210023FBF726F91F20FAF7A5
:109DF800FFFFC8E1DFED637A29EE279A19EE100A12
:109E080005F038FC4BEC10AB06460F4607F028FC73
:109E1800304653EC102B394605F080FC4EA3D3E9AD
:109E2800002305F0C9FA05F013FF4BEC10AB04460C
:109E380007F016FD304653EC102B394605F06EFC42
:109E480002460B4646A1D1E9000105F0B3FA05F038
:109E5800FFFE4FF6E0730093054600230520DC2142
:109E68004246FEF7CBFD434B1B6E53B1464B188859
:109E7800464B4FF4784619880096A2B2ABB2FAF76F
:109E88002DFF414B1C60414B4FF6E0701D60FAF707
:109E980099FF78E1DFED3E8A204629464246FEF7E3
:109EA80081FCF4EE689AF1EE10FAC8BFF0EE689AF9
:109EB800F5EE409ADFED377AF1EE10FA48BFF0EE92
:109EC800679AF4EEE89AF1EE10FA04461CD8F4EE1C
:109ED800E79AF1EE10FA17DBFDEEE99A002019EE89
:109EE800902A4FF4FA71FEF775FC054656B1264BD9
:109EF8001888264B4FF6FF7619880096A2B2ABB2A7
:109F0800FAF7ECFE214B1D60B4EE688ADFED207A8B
:109F1800F1EE10FAC8BFB0EE678ADFED1F7AB4EE33
:109F2800678AF1EE10FA48BFB0EE678AB4EEE88AA5
:109F3800F1EE10FA00F22781B4EEE78AF1EE10FA9A
:109F4800C0F22181BDEEC88A144818EE102A4FF4D9
:109F5800FA71C8E0AFF300800000000000E0634041
:109F68000000000000C05D40180E0020F1A905089F
:109F7800483E00204C0E00202C0F002010AA050897
:109F880014AA05080000C842384600209848002056
:109F98000000FA43000000000000FAC30CFEFFFFB7
:109FA800204629464246FEF7FDFBB5EEC0BAF1EE63
:109FB80010FA044625DDDDE906017FA3D3E9002375
:109FC80005F01EFEE8B190A3D3E90023DDE9060100
:109FD80005F0A4FB02460B460020814905F0EAF98A
:109FE80005F036FE054656B17E4B18887E4B4FF677
:109FF800FF7619880096A2B2ABB2FAF76FFE7A4BD9
:10A008001D60DDE904016AA3D3E9002305F016FE0B
:10A01800002800F0B880DDE9040167A3D3E9002334
:10A0280005F0EEFD002800F0AE8065A3D3E900231B
:10A03800DDE9040105F072FB02460B4600206B497E
:10A0480005F0B8F905F004FE4FE0204629464246DF
:10A05800FEF7A8FB5CA3D3E900230446DDE9080169
:10A0680005F0ECFD50B19DED080B07F085FC0022D2
:10A0780051EC100B5E4B05F051FB6FE0C82570E00A
:10A0880053A3D3E900235046594605F047FB52A392
:10A09800D3E9002305F06CFC05F022FE294608EE02
:10A0A800100A42462046FEF77DFBDFED527A49EE64
:10A0B800677A0446FDEEE77A17EE905A56B1494B97
:10A0C8001888494B4FF6FF7619880096A2B2ABB2B2
:10A0D800FAF704FEBDEEC88A434B18EE102A1D603D
:10A0E8006FF0B300B421FEF775FB434B1B6E0546BA
:10A0F80053B13C4B1888414B4FF4FC6619880096C5
:10A10800A2B2ABB2FAF7EAFD3C4B39E0DFED3C7A9C
:10A11800F4EE678AF1EE10FAC8BFF0EE678AF4EE43
:10A12800E78AF1EE10FA2ED8424620462946FEF775
:10A1380039FB044618EE900A05F09CFA41EC100B26
:10A1480007F01AFC0022294B51EC100B05F0E6FA37
:10A1580002460B460020224905F02CF905F078FD4F
:10A168000546254B1B6E53B11E4B18881E4B4FF6E8
:10A17800FF7619880096A2B2ABB2FAF7AFFD1A4B78
:10A188001D60184B1C601F4B1B78022B09D043B174
:10A198004FF6FF7300930520DC2142460023FEF7AB
:10A1A8002DFC3DB0BDEC088BBDE8F08FAFF300800F
:10A1B8009A9999999999B9BF9A9999999999B93FF9
:10A1C8000000000000408F4089B5F81400E3693FA3
:10A1D80000000000008076401F85EB51B81E194032
:10A1E8000000694038460020984800200000594087
:10A1F800000054C0000048434C0E002018450020C1
:10A208000000C842C04400200000000000409F40F9
:10A218002DE9F843461F8846B6B200250D4F12E0D7
:10A2280008EB040189B23046F9F71EFF29F814003B
:10A238000A200134FDF728F9062CF1D1163501362C
:10A24800F22DB6B204D06FF0040407EB0509E7E776
:10A25800BDE8F8832E4800202DE9F04F85B00B1A91
:10A268000193431E9BB20293431C441F00F106094D
:10A2780001F1FF3A01F1010B9BB20F461646A4B259
:10A288001FFA89F91FFA8AFA1FFA8BFB0393804693
:10A29800204651463246F9F71FFF204639463246D6
:10A2A800F9F71AFF204659463246F9F715FF019B80
:10A2B8000298E518ADB229463246F9F70DFF404637
:10A2C80029463246F9F708FF0134039829463246F1
:10A2D800F9F702FFA4B20A20FDF7D6F84C45D7D10A
:10A2E80005B0BDE8F08F2DE9F843461F8846B6B2A1
:10A2F80000250E4F12E008EB040139F8142089B24A
:10A308003046F9F7E9FE01340A20FDF7BDF8062CBE
:10A31800F1D116350136F22DB6B204D06FF004042F
:10A3280007EB0509E7E7BDE8F88300BF2E480020E2
:10A338002DE9F0432DED068B70EE007A8DB017EE07
:10A34800900AB0EE408A10EE904A20EE009A05F08E
:10A3580091F9064620460F4605F08CF9F7EE008A7B
:10A3680041EC100B41EC1A0B07F07AF979EE287AD8
:10A3780055EC104B17EE900A05F07CF92246804602
:10A3880089462B463046394605F0C8F902460B4641
:10A398004046494605F00EF805F0A2FCB0EE4A0A20
:10A3A800F0EE6A0A09EE900A38EEC99ADFED377ABC
:10A3B80089EE299A29EE279A07F052FA304653EC8B
:10A3C800102B394605F0AAF9044619EE900A0D46F5
:10A3D80005F050F902460B462046294605F0C8FA12
:10A3E80000222B4B05F09AF905F07AFCB4EE688A46
:10A3F800DFED287A284BF1EE10FA044619EE100A20
:10A4080008BFB0EE678A1D6805F034F902460B46AE
:10A4180003A8224909F086FE204605F02BF90246DA
:10A428000B4606A81E4909F07DFE78EE287A38EE1C
:10A43800C88A87EE888A18EE100A05F01BF90246CA
:10A448000B4609A8174909F06DFE0520014603AA25
:10A458000023FAF7F1FD0520142106AA0023FAF7D4
:10A46800EBFDC820052109AA0023FAF7E5FD4FF600
:10A47800E07300930520DC212A460023FEF7BEFA8C
:10A488000DB0BDEC068BBDE8F08300BF000048426C
:10A4980000004940A4707D3F3046002018AA0508F6
:10A4A800EDA8050820AA05082DE9F84F444F3B7888
:10A4B800022B2DED048B804674D1424C424EE08A2B
:10A4C800424DC00080B2FEF76DFF3A78304629460B
:10A4D800FEF7C6FA96ED008ADFED3D7A68EE277A38
:10A4E8002F6817EE900A05F0C5F8824638468B4665
:10A4F80005F0C0F841EC100B41EC190B07F0B0F86F
:10A50800504653EC102B594605F008F928A3D3E917
:10A51800002304F051FF05F0C3FBB0EE490AF0EE4A
:10A52800690A064685B207F09BF9504653EC102B92
:10A53800594605F0F3F80B4602461FA1D1E9000180
:10A5480004F038FF05F0ACFB237D81461FFA80FA42
:10A558002BB9B4F86400B4F86610FFF7C4FE002302
:10A56800284651462375FFF753FE1F2228465146B9
:10A57800FFF772FEB0EE480A00EE907AFFF7D8FEB9
:10A58800E38A9844134B1B881FFA88F8984528BF1C
:10A598000C4AA4F8168028BFD3820A4BA3F864603B
:10A5A800A3F86690BDEC048BBDE8F88FAFF300808C
:10A5B8000000000000E063400000000000C05D40B3
:10A5C800C04400204C0E0020284500202C450020C7
:10A5D8000000C8420C480020174B1B78022B13B50B
:10A5E8000AD1164B1B78022B06D1154C207808B3DC
:10A5F80040B2FFF759FF1BE0124CB4F86830ADF8D1
:10A608000630BDF806309BB24BB1BDF806004EF2DD
:10A618009C7180B2F9F786FD0023A4F86830074BD7
:10A628001B78022B06D1064C94F90000FEF71EFF9A
:10A63800002323701CBD00BFC044002044460020F6
:10A64800E42D00204C0E0020064B00201860064B1D
:10A658001870064B1870064B1870064B1870FDF7EB
:10A668001FBF00BF24450020903E00204446002024
:10A67800180E00202C480020074B10B500241C6041
:10A68800064B02221A702046FDF70AFF044B1C7085
:10A69800044B1C7010BD00BF244500204446002018
:10A6A800180E0020903E00207047FEE7FEE7FEE708
:10A6B800FEE7704770477047FDF7C0BD10B5094CFD
:10A6C800A37A4BB1084B1A6822F006021A6000F010
:10A6D80013F8204600F07FFE4FF48020BDE81040BC
:10A6E80002F0CABDB43E002010ED00E0014801F0C0
:10A6F80041B800BFB43E0020364BD3F8882042F45E
:10A708007002C3F88820344B1A6842F001021A60BC
:10A7180000229A60196821F0847121F4803119604F
:10A728002E495960196882B021F480211960DA60D5
:10A73800009201921A6842F480321A601A6802F490
:10A7480000320192009A01320092019A1AB9009AD5
:10A75800B2F5A06FF2D1204B1B6813F4003318BF79
:10A7680001230193019B012B2ED11B4B1A6C42F044
:10A7780080521A641A4A116841F4804111609A683B
:10A788009A609A6842F400429A609A6842F4A05229
:10A798009A60144A5A601A6842F080721A601968FE
:10A7A8000D4A8901FBD5104B40F205611960936889
:10A7B80023F003039360936843F002039360936864
:10A7C80003F00C03082BFAD1024B4FF000629A6099
:10A7D80002B0704700ED00E000380240103000245D
:10A7E8000070004008544007003C0240184B194ACA
:10A7F800996801F00C01042903D0082903D0164BED
:10A8080019E0164B17E059685A6811F4800F596817
:10A8180014BF124B104B02F03F02B3FBF2F30C4A89
:10A828005268C2F30142C1F38811013252004B430E
:10A83800B3FBF2F3074A1360054B9A68054BC2F362
:10A8480003129A181968127921FA02F21A607047ED
:10A8580000380240F00200200024F40000127A00C0
:10A8680037B51C230124002501A88DF804308DF884
:10A8780005508DF806408DF80740FDF789F8204609
:10A88800214603F069FB0A494CF24F334B60A3F5AC
:10A8980042430B800D814D804FF0804003F004FF50
:10A8A8004FF080402146224604F0C3FA3EBD00BF67
:10A8B8009049002038B54FF08040012104F0CEFACD
:10A8C800002843D04FF080400121214D04F0D1FAF7
:10A8D8004FF08040002103F07CFF2B78013B042BD4
:10A8E80034D8DFE803F003070B102200BDE8384036
:10A8F800F5F75EBFBDE83840F5F78CBFF6F7DEF830
:10A9080000232B7038BD134B00242C7001251D70BB
:10A91800FEF7F0FAFEF7F4FA0F4B1D700F4B18789C
:10A92800F6F7BAF90E4B1C7038BD0A4B0122002409
:10A938001A702C70FEF7D7FAFEF7E2FA064B1C7075
:10A94800064B1878F6F7A8F9054B1C7038BD00BF00
:10A95800190E002044460020903E0020C0440020EC
:10A968000E0E002008B5402002F078FC30B1FAF74E
:10A97800C1FC4020BDE8084002F07EBC08BD0000D4
:10A98800014608B5044804F033FC0348402104F0AC
:10A99800DCFC0028F9D008BD00440040F0B589B0BF
:10A9A8004FF4E1330120019300232B4CADF808301C
:10A9B8001E460146ADF80A30ADF80C30ADF810303F
:10A9C8000C23ADF80E3003F0A3FA4FF40030012148
:10A9D80003F0C2FA20680221072202F071FF072261
:10A9E8006068032102F06CFF012502270423206818
:10A9F800059305A98DF81A608DF81B508DF818700D
:10AA08008DF8197002F0DCFE08236068059305A92B
:10AA18008DF8187002F0D4FEA06801A904F03EFB7E
:10AA28002A4640F225510D4804F076FC262307A853
:10AA38008DF81C308DF81D608DF81E608DF81F5044
:10AA4800FCF7A6FFA068294604F0A5FB044A054BBD
:10AA58001A6009B0F0BD00BF0403002000440040A4
:10AA680089A90008FC520020024B9868002104F0D4
:10AA780092BB00BF0403002010B5094C40F22551D9
:10AA8800204604F06CFC50B1A288D2B2112A02D13F
:10AA9800044B01211970044B19884A401A8010BDD3
:10AAA80000440040120E0020B80E00207047704786
:10AAB80073B50120014603F02BFA264C4FF4D85306
:10AAC8000093022303268DF80430204600236946AC
:10AAD8008DF806308DF807308DF8056002F070FEAD
:10AAE800204608210A2202F0EBFE204609210A220C
:10AAF80002F0E6FE20460B210A2202F0E1FE0A22BD
:10AB080020460C2102F0DCFE01254FF4806320462C
:10AB1800694600938DF806508DF807508DF805604A
:10AB280002F04EFE0A210A46204602F0C9FE2946D6
:10AB38004FF4804003F01CFA8020294603F0F4F912
:10AB48004FF08050294603F043FA284602F094FB60
:10AB58007CBD00BF0000024007B54FF4C060FCF7A1
:10AB68000DFF43238DF804300322012301A88DF83B
:10AB780005308DF806208DF80730FCF709FF0EBD6B
:10AB8800782358430723B0FBF3F0002301338342B3
:10AB9800FCD970474FF47A735843F1E737B500236F
:10ABA800104C019305460320FFF7EAFFEB681A698A
:10ABB800013C019213D0019A002AF4DA019A42F07A
:10ABC80001020192019A1A61064A1969013A019132
:10ABD80002D00199C907F8D40320FFF7D1FF00205C
:10ABE8003EBD00BF410D030010B5C47874B900EB39
:10ABF800820003339B10D0F8D000224603E051F8BE
:10AC0800044C0132046004319A42F8D1002010BD8E
:10AC1800033230B59210D0F8D0400B46002003E044
:10AC28002568013043F8045C04339042F8D101EB05
:10AC3800800030BD0122F0B5002382704022012936
:10AC4800C37082800CD108230370042343704FF42F
:10AC5800A073C38002230372C1724FF0A04309E0BE
:10AC680041B90C230370062343704FF4A063C380DB
:10AC78001F4BC17203F500620261C3604678044647
:10AC880001461A46002508E002F5106C02F530620C
:10AC98000A65C1F814C001353A460431B54202F1DB
:10ACA8002007F1D303F58062426103F58862C0F89A
:10ACB800CC20067803F5A0650146002203E0C1F820
:10ACC8008C50013220350431B242F8D319460022A3
:10ACD80002E0C4F8CC1001320434B24201F58051CC
:10ACE800F7D303F56063C0F80C310020F0BD00BF56
:10ACF8000000044038B5037AC2680025012B0446D9
:10AD080025D1936B417A65F3104309B143F480135D
:10AD18009363D36823F4800323F0500343F01003B4
:10AD28006FF3C3036FF3C7136FF351436FF3D34349
:10AD3800D3602046FFF732FFE378012B3ED105238D
:10AD480063F34405E36845F020059D6036E0D36869
:10AD580043F04003D360FFF721FF237A627A032B85
:10AD680014BF4FF434134FF43C130AB143F4801367
:10AD7800E26814209363FFF70DFFE268217AD36835
:10AD8800032908BF43F48033D360237A032B15D1FA
:10AD9800156B012363F39B656FF3D7552D2345F09E
:10ADA800805563F316451563C820FFF7F3FEE36883
:10ADB80045F400051D63C820FFF7ECFEE378012B7E
:10ADC80007D1E3689D68052262F3440545F0200534
:10ADD8009D60002038BDC3689A6842F001029A60FD
:10ADE80000207047C3689A6822F001029A60002028
:10ADF800704707B500230193019B43F0200301939B
:10AE0800019B61F38A130193019BC2681361064B8E
:10AE18001169013B019102D001998806F8D40320F9
:10AE2800FFF7AEFE00200EBD410D030007B500235D
:10AE38000193019B43F010030193019BC2681361C6
:10AE4800064B1169013B019102D00199C906F8D45A
:10AE58000320FFF795FE00200EBD00BF410D030043
:10AE680008B5C268D36801296FF35D736FF39E73E9
:10AE780002D143F0005302E009B943F08043322085
:10AE8800D360FFF787FE002008BDC368586900F04B
:10AE980001007047C3685B6913F0010F14BF0020FD
:10AEA80001207047C368586900F001007047C36803
:10AEB8005A69986910407047C368586870470369B1
:10AEC8001A6861F301021A607047C268002393612F
:10AED8004FF0FF335361536053610B4B9361C37859
:10AEE8009169002B14BF4FF400634FF4016343F4DE
:10AEF800701343F4405343F0080321EA03010B4362
:10AF080093610020704700BF00080080F8B5D0F8B2
:10AF18000C3100221A60036915461A6865F3CC22C1
:10AF28001A60C37A012B04461BD10321FFF7C7FF20
:10AF3800E36880214FF4800261F30F0259629A623C
:10AF4800C02262F30F0561F31F454FF4A072C3F8E6
:10AF5800045162F30F056FF31F45C3F80851C3F896
:10AF68000C5110212046FFF744FF2046FFF75EFFF3
:10AF7800226900234FF0FF311361204653611E46BA
:10AF88009161FF25D361214610E082691768C7F3F4
:10AF9800076707F08007FFB2002F14BF4FF09047F4
:10AFA8000027176001331661043095606278934278
:10AFB800EBD300231D46FF2010E04A6D1668C6F348
:10AFC800076606F08006F6B2002E14BF4FF09046D2
:10AFD800002616600133156104319060627893424F
:10AFE800EBD323691A6942F480721A61E278012A64
:10AFF80004D1054A402161F359421A632046FFF7FC
:10B0080064FF0020F8BD00BF0301010003699B68CD
:10B01800C3F34103013B022B9ABF024AD05C0320D1
:10B02800704700BF40A5040810B5036981699C6892
:10B038000A68C4F34100022802D06FF30A0202E052
:10B04800032060F30A020A605A6842F480725A6068
:10B05800002010BD30B54D780B780022012D00EB93
:10B06800830405D105FA03F3A46963F30F0205E02D
:10B07800012505FA03F3646D63F31F422368C3F3E4
:10B08800072505F08005EDB26DB98D6865F30A03F3
:10B09800CD78C98865F3934361F3995343F080539E
:10B0A80043F4004323600369D9690A43DA61002045
:10B0B80030BD30B54D780B780024012D224600EBC9
:10B0C800830105D105FA03F3896963F30F0205E0EB
:10B0D800012505FA03F3496D63F31F4203696FF312
:10B0E800CF340C60D96921EA0202DA61002030BD50
:10B0F800F8B54F780B78012F00EB830349D19E698F
:10B108004C69356833692A4664F3120314B967F346
:10B11800DC430BE08F68E419013CB4FBF7F7CC780B
:10B1280067F3DC43012C08BF64F35E733361C378B3
:10B13800012B06D10B780C6900EB83039B695C61DA
:10B148000CE0CB78012B09D04B693BB103690C7833
:10B158005E6B012707FA04F434435C63CB78012B58
:10B1680007D103699B68DB0554BF45F0005245F0E1
:10B1780080520B7800EB830342F004429B691A600B
:10B18800CB78012B38D10A788B8AC968FFF72CFD58
:10B1980032E05E6D4F6935688C6833692A462FB98D
:10B1A80064F31203012464F3DC430AE03F19013F0E
:10B1B800B7FBF4F7BF05BF0D67F3DC437C4364F3CB
:10B1C80012033361C378012B05D10B780C6900EBAE
:10B1D80083035B6D5C61CB78012B06D14B7913B18E
:10B1E80045F0005201E045F080520B7800EB8300F7
:10B1F80042F00442436D1A600020F8BD73B54D78E3
:10B20800012D3DD183694A691E681C690094E4B226
:10B2180042B962F306048DF800409DF8024065F3D8
:10B22800C4040EE08D68AA4286BF4D6165F306042A
:10B2380062F306048DF800409DF80240012262F393
:10B24800C4048DF80240009A1A61C278012A05D117
:10B258000A780C6900EB82029269546146F0044254
:10B268001A60C378002B34D14B69002B31D00369A5
:10B278000A78586B012101FA02F202435A6328E066
:10B288000B784E698C6800EB83035B6D1A681D6947
:10B298000095EDB206B14C6164F306059DF80240D5
:10B2A8008DF80050012565F3C4048DF80240009C18
:10B2B8001C61C378012B05D10B780C6900EB830363
:10B2C8005B6D5C610B7800EB830042F00442436DD8
:10B2D8001A6000207CBD4B78012B0B7800EB8300B3
:10B2E8000AD182691368C3F3076101F08001C9B20A
:10B2F80021B143F0804301E0426D136843F4001329
:10B308001360002070474B78012B0B78C97800EB4D
:10B3180083000CBF8269426D02391368C9B26FF3AA
:10B328005553012998BF43F080531360002070479C
:10B3380003699A69D8691040000C704700EB8101D5
:10B3480002694B6D9B68506918407047036998699A
:10B35800DB69184080B2704782B000230093C02395
:10B368008DF803300122002362F3C4038DF8023004
:10B3780018238DF80030009A436D1A61C278012AAB
:10B3880006D100F5B96058611A684FF080221A603A
:10B3980002B07047D0F8143110B50446D3B1036930
:10B3A8009A68D20716D5827A42B1D0F80C21D0F823
:10B3B8000C116FF341026FF300020A605A6842F001
:10B3C80001025A600520FFF7E5FB23695A6822F05D
:10B3D80001025A6010BD837A63B103699B68D9077B
:10B3E80008D5D0F80C31D0F80C216FF341036FF376
:10B3F800000313607047012310B5002280F8123152
:10B4080004460346FF2104E058698160186D013243
:10B418008160607804338242F6D3236900221A617E
:10B428005A61DA614FF0FF329A612046FFF7FEFC5D
:10B4380020461021BDE81040DBE44B78012B0B7847
:10B4480000EB83000FD183691868C0F3074000F050
:10B458002003DBB2CBB900F00200C0B200280CBF59
:10B46800302020207047436D1868C0F3074000F073
:10B478002003DBB25BB900F00200C0B200280CBFA9
:10B488004FF440504FF400507047102070474FF46D
:10B49800805070474B78012B0B7810B500EB830375
:10B4A8000AD19C69102A236802D1BDE8104012E72E
:10B4B800202A0CD0302A0FE05C6DB2F5805F23683B
:10B4C80002D143F400131BE0B2F5005F02D143F050
:10B4D800006315E0B2F5405F0FD1C3F3074202F0F5
:10B4E8002002D2B222B100234B71BDE810400AE716
:10B4F80043F0806343F0802302E00AB962F3CF335C
:10B50800236010BDF8B50446FFF794FB0122002321
:10B5180084F8122184F81331282716461946402545
:10B528000CE007FB03F000F58C7022182354D3803D
:10B538005670D1709560D160516101336278934241
:10B54800EFD300232826194640250CE006FB03F01C
:10B5580000F55C7022182354D3805170D170956027
:10B56800D1605161013362789342EFD32046FFF7EF
:10B5780039FC2046FFF7BEFB00212046FFF770FC90
:10B588002046FFF7C3FC2046BDE8F840FFF723BC80
:10B5980070B5CDB20C464FF0280601F07F0106FBCE
:10B5A800010115F0800F14BF01F58C7101F55C7174
:10B5B80004F07F04ED090C704D708A60CB7005B102
:10B5C800CC80022B01D100230B71FFF743FD002033
:10B5D80070BD10B5CAB201F07F034FF0280404FB18
:10B5E800030312F0800F14BF03F58C7303F55C732B
:10B5F80001F07F01D20919705A701946FFF759FDF9
:10B60800002010BD38B501F07F0528246C4304F5EF
:10B618005C7401194B6100238B614B70EBB20355CD
:10B62800CA60C478012C08BF0A6113B9FFF7E6FDA8
:10B6380001E0FFF75DFD002038BD70B501F07F0423
:10B648002825654305F58C7541190126E4B2CA60C1
:10B658000A6100224E7044558A614B6114B9FFF7A4
:10B66800CDFD01E0FFF744FD002070BDCAB212F025
:10B67800800F10B54FF0280306D001F07F0403FBBC
:10B68800040303F58C7303E003FB010303F55C7308
:10B69800D209012401F07F0119709C705A70194673
:10B6A800FFF719FE002010BDCAB212F0800F10B5C6
:10B6B8004FF0280306D001F07F0403FB040303F5D1
:10B6C8008C7303E003FB010303F55C730024D209C8
:10B6D80001F07F0119709C705A701946FFF713FE2C
:10B6E800204610BD08B50B0604D501F07F01FFF711
:10B6F80080FB01E0FFF79AFB002008BD03690022E8
:10B7080061F30A1219680A431A60704703695A6894
:10B7180003206FF341025A60FFF73CBA03695A6885
:10B72800032042F002025A60FFF734BA11F0800F8A
:10B738004FF0280306D001F07F0103FB010101F55A
:10B748008C7103E003FB010101F55C71FFF775BE25
:10B7580011F0800F4FF0280306D001F07F0103FBA2
:10B76800010101F58C7103E003FB010101F55C7136
:10B77800FFF790BE2DE9F74F0446FFF78BFB002833
:10B7880000F03F822046FFF792FB0546002800F0B4
:10B798003882C0F3074000F00800C0B2002861D02A
:10B7A8002046FFF7C5FDA146824627464FF0000810
:10B7B800DFF86CB32E4650E01AF0010F46D05FFA5E
:10B7C80088F2114620460092FFF7B8FD10F0010FED
:10B7D8000546009A20D07B6D01259D60E178A9423D
:10B7E80007D11B69D9F87813C3F31203CB1AC9F828
:10B7F8008833DBF8003020461B6811469847E37809
:10B80800012B09D1B8F1000F06D194F81131052B9D
:10B8180002D12046FFF7A0FD05F00203DBB213B109
:10B828007B6D02259D6005F00403DBB213B17B6DCF
:10B8380004259D6005F00805EDB23DB1DBF8003048
:10B8480020469B6898477B6D0820986008F101089E
:10B858004FEA5A0A043709F12809BAF1000FABD1A7
:10B8680035460120C5F3074303F00403DBB2002B80
:10B8780000F0AF802046FFF769FD264683464FF06B
:10B88800000801959FE01BF0010F00F097802369E5
:10B898005FFA88F919695D6B04EB890225FA09F5E5
:10B8A8009269ED019268EDB20D431540EA071CD587
:10B8B8005A6B012000FA08F122EA01025A63B369BF
:10B8C800974A9860136805465B682046494698473A
:10B8D800E378AB4209D1B8F1000F06D194F81131E1
:10B8E800042B02D12046FFF737FD05F00403DBB235
:10B8F80013B1B36904259D6005F00803DBB213B1E9
:10B90800B36908259D6005F01003DBB213B1B36974
:10B9180010259D6005F02003DBB213B1B369202523
:10B928009D6005F04003DBB213B1B36940259D600B
:10B9380005F00203DBB213B1B36902259D6025F05F
:10B948007F0515F0FF0F39D0282505FB084505F5BB
:10B958008C75C246AB696A69C3EB020CAB689C453F
:10B9680028BF9C460CF1030CB3694FEA9C0C9B69F9
:10B978006746A04614E0AA68E9681C1B944228BFE1
:10B988001446A3B240464A46FFF72EF9EB681B1946
:10B99800EB60AB69E71C1C19AC61B3699B69BF0814
:10B9A8009BB2BB4205D9AC696B699C4201D2002BA2
:10B9B800E1D1B369802544469D60D04608F101086D
:10B9C8004FEA5B0B0436BBF1000F7FF45CAF019DBF
:10B9D800012005F00203DBB213B1E36802225A61C9
:10B9E800C5F3076303F08003DBB2CBB1A37A43B19D
:10B9F800D4F80C31D4F80C216FF341036FF3000332
:10BA0800136023695A6822F001025A60444B1B688C
:10BA180020469B699847E3684FF000425A6101202D
:10BA2800C5F3072303F00803DBB2F3B13C4B1B68F3
:10BA380020465B6998472369E2689B684FF4006178
:10BA48005161A27A82B1DB070ED5D4F80C311A689D
:10BA580042F001021A601A6842F003021A60314B80
:10BA68001A6942F006021A61012005F00803DBB2E8
:10BA780043B12B4B1B682046DB689847E3680822D4
:10BA88005A61012005F01003DBB2002B33D0E368C4
:10BA98009A6922F010029A611F6A282607F00F039C
:10BAA80006FB0346C7F34343022B06F55C7602D038
:10BAB800062B1AD10EE047F6F0733B40ABB1C7F343
:10BAC8000A172046F1683A46FFF7A2F8F368DB192F
:10BAD800F36007E004F5B96120460822FFF798F8FB
:10BAE800C7F30A17B369DF19B761E3689A6942F0C7
:10BAF80010029A610120C5F3072303F01003DBB29B
:10BB0800002B39D023695A68002622F001025A60B6
:10BB180031462046FFF76DF923463246FF2108E0FB
:10BB2800A003002000ED00E058698160186D013223
:10BB38008160607804338242F6D3236901274FF08D
:10BB4800FF3267F30F069A6167F31F460F22DE6123
:10BB58005A612F221A611A686FF30A121A60204676
:10BB6800FFF7FAFBE3684FF480525A61264B1B68D3
:10BB780020461B6998473846C5F3072303F020037E
:10BB8800DBB2EBB12046FFF74FFAE3682046DE68E8
:10BB9800FFF73CFA032806D10023A3704FF4007383
:10BBA800A380092304E00123A3704023A380052375
:10BBB80063F38D26E3684FF40052DE6001205A617A
:10BBC800C5F3074303F01003DBB24BB10E4B1B6800
:10BBD8002046DB699847E3684FF480125A610120D8
:10BBE800C5F3074505F02005EDB255B1064B1B68B6
:10BBF80020461B6A9847E3684FF400125A610120F7
:10BC0800FFE7BDE8FE8F00BFA003002043230B80A1
:10BC1800004870471003002038B51F4B1A68511CA4
:10BC2800052A196035D11979002201291A6030D006
:10BC38009968B1F5006F08BF9A60174B9968DC687E
:10BC4800A1421A4602D100221A7122E086BFC1F52C
:10BC580000631361C1EB0404D0F8EC3598BF14619C
:10BC68001569B3F839300C4C9D428AB204D9591879
:10BC7800ED1AA160256104E06918A1600021ABB24A
:10BC88002161054901240C7104498A188121FFF7B3
:10BC9800D4FC002038BD00BFBC0E00202F4A002075
:10BCA80038B528230A4D03FB01010A4BB1F8881364
:10BCB8001B69044628469847D4F8EC352046B3F863
:10BCC800403001212A46FFF79DFC002038BD00BF07
:10BCD800E74900208C03002070B50B7813F060054D
:10BCE80006460C4625D0202D1FD1CD88B5B113F0BE
:10BCF800800F487808D0214B21499B682A469847ED
:10BD0800E2881F49304625E01E4B1D4958641E4BEA
:10BD180030465D612A4600F022FB1DE0174B48784B
:10BD28009B6829462A46984725E000F077FB0225BC
:10BD380021E04B780A2B11D00B2B14D0062B1AD1EB
:10BD48004B881B0A212B03D1CA883A2A28BF3A22DA
:10BD58000E49304600F0EAFA00250CE00C490122B1
:10BD680000F0E4FA07E08B781BB9074A1D46936197
:10BD780001E000F053FB284670BD00BF8C03002093
:10BD8800274A002010030020BC0E002022030020B8
:10BD9800D40E002010B581210446FFF71AFC0121BA
:10BDA8002046FFF716FC82212046FFF712FC024BC3
:10BDB8005B689847002010BD8C03002038B5D0F888
:10BDC800EC350446B3F8392081210223FFF7E0FB64
:10BDD800D4F8EC350121B3F8402020460223FFF7C0
:10BDE800D7FB8221082203232046FFF7D1FB094B0A
:10BDF800022200251A715D71074B1B689847D4F819
:10BE0800EC35064AB3F8403020460121FFF7FAFB2B
:10BE1800284638BDD00300208C030020E7490020C5
:10BE280010B5074C606CFF2807D0064B064A9B6884
:10BE3800064952699847FF236364002010BD00BF7C
:10BE4800100300208C030020BC0E0020274A00208D
:10BE580038B510490B79012B19D10C690CB90C7143
:10BE680015E0D0F8EC358D68B3F839309C42AAB2A9
:10BE780003D95D198D60E41A03E0A3B22C198C6014
:10BE880000240C61044952188121FFF7D6FB0020D9
:10BE980038BD00BFBC0E00202F4A0020002070478C
:10BEA800002070470023F0B5084A094E1D4609E0F6
:10BEB8001468C75C375501340133B4F5006F14605A
:10BEC80008BF15608B42F3D10020F0BDC80E0020DA
:10BED8002F4A0020104B114AD3F800C000232DE947
:10BEE800F0410F4F16461D460DE0146810F8038008
:10BEF80007F804800134802C08BF2C46146034688D
:10BF0800644505D001338B42EFD10020BDE8F081B4
:10BF18000220BDE8F08100BFB0520020C4520020CA
:10BF28003052002021280FD1084B1A680A701A686D
:10BF3800120A4A705A888A70DA78CA701A790A71AD
:10BF48005A794A719B798B710020704784030020CD
:10BF580007B502AB012103F8010D1846FFF7A2FF50
:10BF68000EBD002100E00131435C002BFBD199E7B5
:10BF780098E70B4B0B491A68096891420BD00A499C
:10BF88008A5C02701A680132802A1A6005D1002280
:10BF98001A6001207047002070470120704700BFD9
:10BFA800B0520020C452002030520020204B1A68A2
:10BFB800204B1B689A42F0B509D135E00133802B3C
:10BFC80008BF00239A4203D11A4B1A602CE01A4C7E
:10BFD800E15C0029F2D00A29F0D00D29EED0154CE9
:10BFE8001549134D23600E460023CF182268BA5C0A
:10BFF800C254226801339F18802F08BF53422F680C
:10C008009A18974210D0B25C1AB10A2A01D00D2AA8
:10C01800EBD10022C254074A116859187F291160D0
:10C0280003D98039116000E000231846F0BD00BF35
:10C03800C4520020B052002030520020704700BF88
:10C04800D0F8E43510B51B6904469847032384F8F3
:10C058001231002010BD08B5042380F81231D0F841
:10C06800E435DB689847002008BD08B5D0F8E0350E
:10C07800DB6903B19847002008BD08B5D0F8E03562
:10C088001B6A9847002008BD08B5D0F8E0355B6A00
:10C098009847002008BD002110B5402204460B46F1
:10C0A800FFF776FA8021402200232046FFF770FA36
:10C0B800012384F81231D4F8E435A0785B689847F6
:10C0C800002010BD13B56946044600F085F99DF8B7
:10C0D800001001F01F03012B07D0022B0AD073B9FF
:10C0E8002046694600F026FA0FE02046694600F02F
:10C0F80007FA0AE02046694600F0A2F905E021F0B7
:10C108007F01C9B22046FFF7B1FA00201CBD38B53F
:10C11800044600293DD190F81131022B42D1D0F8C4
:10C128003421D0F820319A4211D9C178D21A012984
:10C13800C0F8342104D1D0F82411CB18C0F8243128
:10C1480092B22046D4F8241100F000F92AE0D0F881
:10C158003821B2FBF3F503FB152565B99A420AD3DA
:10C16800D0F83C319A4206D229462A4600F0EEF829
:10C17800C4F83C5116E0D4F8E035DB682BB194F8EC
:10C188001221032A01D120469847204600F00FF9D2
:10C1980008E0D0F8E0355B6923B190F81221032A52
:10C1A80000D19847002038BD10B5044659BB90F817
:10C1B8001131032B30D1D0F88C23D0F878339A4240
:10C1C80014D9C178D21A0129C0F88C2304D1D0F827
:10C1D8007C13C918C0F87C139A4228BF1A4692B239
:10C1E8002046D4F87C1300F0CAF815E0D0F8E03502
:10C1F8001B6923B190F81221032A00D198472046E1
:10C2080000F0C6F808E0D0F8E0359B6923B190F853
:10C218001221032A00D19847002010BD2DE9F041D2
:10C22800069F0446164698460D46FEF741FC2046F2
:10C238002946C4F8E085C4F8E475C4F8E865FFF752
:10C2480061F9D4F8E4351B6898472046BDE8F04109
:10C25800FEF782BC00207047D0F8E03510B50446E0
:10C268001B689847D4F8E4359B689847002010BDB0
:10C2780008B5D0F8E0355B689847002008BD000095
:10C2880012230B8000487047D003002004230B8042
:10C2980000487047E203002010B5044C04480A46E1
:10C2A800214600F075FA204610BD00BFC852002094
:10C2B8002CAA05080A4608B50248034900F068FA9E
:10C2C800014808BD3FAA0508C85200200A4608B51B
:10C2D8000248034900F05CFA014808BD4DAA050868
:10C2E800C852002008B50A4608B9044800E00448C6
:10C2F800044900F04DFA034808BD00BF58AA0508D4
:10C3080065AA0508C852002008B50A4608B90448B5
:10C3180000E00448044900F03BFA034808BD00BFA8
:10C3280072AA050893AA0508C852002010B513463A
:10C338000C46C0F83821C0F83421022280F81121B7
:10C3480000212246FFF779F9002010BD10B50C46F0
:10C35800134600212246FFF770F9002010BD10B5E2
:10C3680013460C46C0F89023C0F88C23032280F8AB
:10C37800112100212246FFF745F9002010BD10B514
:10C388000C46134600212246FFF73CF9002010BD59
:10C398000021042310B50A46044680F811310B46E3
:10C3A800FFF74BF92046FEF7D7FF002010BD00210C
:10C3B800052310B50A46044680F811310B46FFF7ED
:10C3C80021F92046FEF7C8FF002010BD282303FBF3
:10C3D8000100B0F88803704790F8C8350B7090F8E2
:10C3E800C9354B7090F8CB2590F8CA3503EB02237A
:10C3F8004B8090F8CD2590F8CC3503EB02238B8049
:10C4080090F8CF2590F8CE3503EB02239BB2CB8072
:10C41800C0F83C31012380F81131704710B591F90B
:10C428000030002B044601DBCB880BB9802100E0EB
:10C438000021FFF71BF92046BDE81040FEF78CBF2E
:10C4480038B50D4604466B780979012B10D027D3EF
:10C45800032B51D190F81231022B28D0032B47D14E
:10C468006B889BB991B1802910D0FFF7FFF80DE0D8
:10C4780090F81231022B1AD0032B39D16B88002B7C
:10C488003AD149B1802907D0FFF70EF9D4F8E03541
:10C4980020469B68294698472046FFF779FF2BE0FE
:10C4A80090F81231022B02D0032B21D106E019B3E8
:10C4B800802921D02046FFF7D9F81DE011F0800F20
:10C4C8004FF0280306D001F07F0103FB010393F826
:10C4D8001A2103E003FB010191F87223074B02B113
:10C4E80001221A60204605490222FFF71FFF03E0D8
:10C4F80020462946FFF792FF002038BDD80E0020BD
:10C5080038B590F81231032B04460D460CD10B793F
:10C51800012B09D8D0F8E0359B689847EB883BB9E0
:10C528002046FFF735FF03E020462946FFF776FF50
:10C53800002038BD73B54B7804460D46092B00F230
:10C548001C81DFE813F0D10008011A01E4001A0188
:10C5580072000A001A01C00092004B881A0A013AB8
:10C56800062A00F20A81DFE812F007001A00270005
:10C578000801080108010801D4F8E835A0781B680B
:10C588000DF106019847EB88402B014603D094F83B
:10C598001231012B3AD10823ADF8063036E0D4F831
:10C5A800E035A0789B6A0DF1060198470223437095
:10C5B8000146C4F8EC0529E0DBB2052B00F2DD806A
:10C5C800DFE803F003080D12171CD4F8E835A0784B
:10C5D8005B6817E0D4F8E835A0789B6812E0D4F8D7
:10C5E800E835A078DB680DE0D4F8E835A0781B6959
:10C5F80008E0D4F8E835A0785B6903E0D4F8E835BA
:10C60800A0789B690DF1060198470146BDF80630F0
:10C61800002B00F0B680EA88002A00F0B2809A4227
:10C6280028BF1A46ADF806205CE08B88002B40F046
:10C63800A480CB88002B40F0A08094F812214B886E
:10C64800032A00F09A8003F07F05204684F81351EE
:10C658002946FFF753F82046FFF79AFE0DB102234B
:10C6680000E0012384F812318BE08978464E0129D5
:10C67800317100F2828094F81231022B02D0032B20
:10C688007BD108E0002962D00121032384F810112E
:10C6980084F8123113E041B9022384F8123184F886
:10C6A80010112046FFF7E4FD51E094F8101101291C
:10C6B80020464DD0FFF7DCFD317984F81011204673
:10C6C800FFF7CAFD43E0CA88012A56D194F812310F
:10C6D800022B02D0032B50D102E020462B4913E055
:10C6E80004F5887120460FE094F81231023B012BC3
:10C6F80043D8D4F814312449002B0CBF0123032359
:10C7080041F80C3F20460122FFF710FE39E04B8824
:10C71800012B29D0022B34D18B8813F0FF0F30D195
:10C7280021691B0A013B4A68042B0FD8DFE803F094
:10C73800030507090B00012306E0022304E0032395
:10C7480002E0042300E0052363F306124A60204652
:10C75800FFF71EFE15E094F81231023B012B0CD8AE
:10C768004B88012B0DD10023C4F81431D4F8E035DF
:10C7780020469B6829469847E9E720462946FFF75F
:10C788004DFE00207CBD00BFD80E0020E00E00202A
:10C7980030B5C8B10023DDB20133C41814F8014C18
:10C7A800002CF8D16B1C5B0013800B7003234B70BB
:10C7B800022305E0CA545A1CD2B202338C54DBB2AD
:10C7C80010F8012B002AF5D130BD00BF7047704723
:10C7D8007047704770477047704700000EB403B049
:10C7E80070470A2810B5044602D10D20FFF7F9FF5B
:10C7F800064A13681BB103F8014B136010BD044BC4
:10C808001B680BB12046984710BD00BFE80E0020FA
:10C81800FC52002010B5044601E0FFF7E2FF14F8CF
:10C82800010B0028F9D110BD2DE9F04F044685B061
:10C838000D464FF00A0A00E035462078002800F03F
:10C84800C480252801D0013467E06078302803D1FE
:10C85800A0780123033407E02D2802D002340023F6
:10C8680002E0A078022303344FF0000805E00AFB39
:10C87800080814F8010BA8F13008A0F13002D2B270
:10C88800092AF4D96C2801D04C2803D114F8010BDB
:10C8980043F00403002800F09880602886BFA0F1C8
:10C8A8002002D2B202464F2A3DD006D8432A2DD0C4
:10C8B800442A09D0422A30D133E0552A04D0582AD4
:10C8C80029D0532A29D101E00A272DE02E1D2F68EF
:10C8D800002500E001357A5D002AFBD104E0202024
:10C8E800FFF77FFF4D4601E0980704D4454505F161
:10C8F8000109F4D34D463846FFF78CFF03E02020AA
:10C90800FFF76FFF01354545F9D395E728782E1DC8
:10C91800FFF767FF90E7102706E0FFF762FF2E4654
:10C928008AE7022700E008272E1D442A296804D137
:10C93800002902DA494243F00803002200E02A46AF
:10C94800B1FBF7FE07FB1E11CDB2092D714607D9C1
:10C95800782814BF4FF0070C4FF0270C6544EDB250
:10C9680030350DF80250551CBEF1000F02D0102DC5
:10C97800E5D10F22190705D504A94D192D2105F870
:10C98800101C951C13F0010F0CBF4FF0200B4FF03B
:10C99800300B9B072F4604D508E05846FFF721FFC8
:10C9A8004F46474507F10109F7D34F46013D1DF8AA
:10C9B8000500FFF716FF002DF8D103E02020FFF750
:10C9C80010FF01374745F9D336E705B0BDE8F08FCA
:10C9D80070B5064D0C462E68286001E0FFF701FF90
:10C9E80014F8010B0028F9D12E6070BDFC5200200C
:10C9F8000FB407B504A951F8040B0191FFF714FF10
:10CA0800BDE80E4004B070470EB417B505A9084C30
:10CA180051F8043B206018460191FFF705FF226892
:10CA2800002313702360BDE81E4003B0704700BFA9
:10CA3800E80E00200EB433B505A9074C51F8043BA5
:10CA48002568206018460191FFF7EEFE2560BDE8D5
:10CA58003C4003B0704700BFFC52002070B51E4632
:10CA680004461C481546FFF7C3FF022E1FD0042EAC
:10CA780025D0012E2AD105E0A15D1748FFF7B8FFA0
:10CA8800013600E00026AE42F6DB2020FFF7A9FEC3
:10CA9800002609E0A05DA0F12003DBB25E2B88BF71
:10CAA8002E20FFF79EFE0136AE42F3DB0EE034F88F
:10CAB800021B0A48FFF79CFF013DF8D106E054F835
:10CAC800041B0748FFF794FF013DF8D10A20BDE891
:10CAD800704086E6B4AA0508BBAA0508C1AA0508DD
:10CAE800C7AA050808B501214FF4807001F07CFA47
:10CAF8004FF480700021BDE8084001F075BA436822
:10CB08000A6823F0407323F4807313430A7943EAD5
:10CB180002234360CA680B6930B51A4384688D687C
:10CB2800084B2A43234013434A7943EA420383606C
:10CB38000B7DC26A013B22F47002DBB242EA035366
:10CB4800C36230BDFDF7FFC000230360037143716A
:10CB58008360C3600361012303757047074A084B6C
:10CB6800516810B50B4090E8120021438468C068F2
:10CB7800214301430B43536010BD00BF0023014014
:10CB8800E030FCFF0023036043608360C3607047AC
:10CB9800836811B143F0010301E023F001038360CE
:10CBA8007047436823F4400323F400730B43436046
:10CBB8007047416282627047436823F01F030B434A
:10CBC80043607047044B5A6810B142F4000201E018
:10CBD80022F400025A60704700230140044B5A684F
:10CBE80010B142F4800201E022F480025A607047DA
:10CBF80000230140092970B50CB20CD904EB440498
:10CC08001E3CC6680725A54026EA0505A34045EA57
:10CC18000304C4600AE0066904EB44040725A54040
:10CC280026EA050513FA04F42C430461062A0CD8F5
:10CC38000523013A5A43446B1F23934024EA030314
:10CC4800914043EA0102426370BD0C2A12B20CD82B
:10CC580002EB8202233A046B1F23934024EA030366
:10CC6800914043EA0102026370BD02EB8202413A3D
:10CC7800C46A1F23934024EA0303914043EA010254
:10CC8800C26270BD836843F08043836070478068E8
:10CC9800C0F380507047836811B143F4806301E0AA
:10CCA80023F4806383607047836811B143F0020303
:10CCB80001E023F00203836070474368013923F4DD
:10CCC800604343EA413343607047436811B143F41A
:10CCD800006301E023F4006343607047C06C80B2D6
:10CCE8007047014B1868704708230140836811B1E9
:10CCF80043F4807301E023F4807383607047836892
:10CD080011B143F4007301E023F4007383607047AA
:10CD1800044B5A6810B142F4005201E022F4005268
:10CD28005A60704700230140092970B50CB20CD92C
:10CD380004EB44041E3CC6680725A54026EA050501
:10CD4800A34045EA0304C4600AE0066904EB44040E
:10CD58000725A54026EA050513FA04F42C430461C7
:10CD6800836BC3F30154121B0232D2B202EB82026C
:10CD78001F24944023EA040391400B43836370BD4E
:10CD8800836B013923F4401343EA015383637047EB
:10CD980082B0002301930190019BCB180193019B62
:10CDA8001A6002B07047836823F470230B438360D2
:10CDB8007047836823F440130B438360704783688C
:10CDC80043F48003836070478068C0F380507047E5
:10CDD800436811B143F4806301E023F48063436046
:10CDE8007047436811B143F4805301E023F4805342
:10CDF8004360704782B0002301930190019B283360
:10CE08005B180193019B186880B202B07047012338
:10CE1800C9B213FA01F143680AB1194301E023EAE0
:10CE2800010141607047036819420CBF00200120CE
:10CE38007047C943016070474368006810EA1120D1
:10CE480007D00122C9B212FA01F119420CBF002021
:10CE5800012070476FEA112101607047036823F0D1
:10CE6800010303600023036043608360C3600361C0
:10CE7800212343612C4B98421CD02C4B984220D044
:10CE88002B4B984225D02B4B98422AD02A4B9842BC
:10CE98002FD02A4B984233D0294B984237D0294B70
:10CEA800984204D14FF03D5243F8AC2C7047264BC2
:10CEB800984203D13D2243F8082C7047234B9842EF
:10CEC80004D14FF4746243F8202C7047204B9842E9
:10CED80004D14FF4741243F8382C70471D4B984214
:10CEE80004D14FF0746243F8502C70471A4B9842A3
:10CEF80003D11A4A43F8642C7047194B984203D15E
:10CF0800184A43F87C2C7047174B984203D1174AAC
:10CF180043F8942C7047164B984204BF4FF03D528B
:10CF280043F8AC2C704700BF1060024028600240F4
:10CF380040600240586002407060024088600240D1
:10CF4800A0600240B86002401064024028640240B9
:10CF58004064024058640240706402403D00002072
:10CF680088640240400F0020A064024000003D2079
:10CF7800B86402400268134B10B51340CC680A68C5
:10CF880022434C6922438C692243CC6922430C6AB0
:10CF980022434C6A22438C6A22434C6B22438C6B9B
:10CFA80022431343036042690C6BCB6A22F00702E9
:10CFB8002343134343610B6943604B6883608B6869
:10CFC800C36010BD3F801CF0002303604360836092
:10CFD800C360036143618361C36103624362836227
:10CFE800C3620363436383637047036811B143F00B
:10CFF800010301E023F0010303607047036811B1E6
:10D0080043F4004301E023F40043036070470368DE
:10D0180011B143F0200301E023F0200303607047BF
:10D0280041607047406880B27047036812B143F4AA
:10D03800002301E023F400230360016170470368C3
:10D0480011B143F4802301E023F480230360704787
:10D058000AB101617047C16070470068C0F3C04001
:10D068007047006800F001007047406900F0380020
:10D0780070470A4A0A4B10B50A4CA04288BF1346AB
:10D088008A004CBF5B681B6821F0F02121F08211F7
:10D0980019420CBF0020012010BD00BF00640240EF
:10D0A800006002400F64024010B5084B084A094C62
:10D0B800A04288BF134611F0005F21F0F02121F053
:10D0C800821114BFD960996010BD00BF0060024092
:10D0D800006402400F6402400B0607D5436912B191
:10D0E80043F0800301E023F080034361802909D0E5
:10D0F80001F01E01036812B119430160704723EA69
:10D10800010101607047124B124A10B5124CA0423F
:10D118008CBF14461C4621F0F02323F0C3132BB117
:10D12800026802F01E0202EAD12202E0426902F01D
:10D13800800288004CBF6368236821F0F02121F049
:10D148008210184002D0101C18BF012010BD00BF6B
:10D1580000600240006402400F64024010B5084BB2
:10D16800084A094CA04288BF134611F0005F21F01D
:10D17800F02121F0821114BFD960996010BD00BF61
:10D1880000600240006402400F640240044B002229
:10D198001A605A609A60DA60024A5A61704700BFA2
:10D1A800003C0140FFFF7F00837910B5002B29D098
:10D1B8001A4B01681C68CA4314401C605C68224012
:10D1C8005A60027902F1804202F59E3214682143C6
:10D1D800116002689C68D1430C409C60DC68214067
:10D1E800D9604179102906D1996811439960D968A5
:10D1F8000A43DA6010BD01F1804303F59E331968D4
:10D208000A4308E00379016803F1804303F59E337C
:10D218001A6822EA01021A6010BD00BF003C0140F2
:10D2280000230C2203600371427183717047024B23
:10D238001A6902431A617047003C0140034B5B695D
:10D2480018420CBF00200120704700BF003C01407D
:10D25800014B5861704700BF003C0140054B1A68FC
:10D268005B69034004D010420CBF002001207047C6
:10D2780018467047003C0140014B5861704700BF99
:10D28800003C01404FF0204318B943F2DB021A601A
:10D2980003E043F2D20243F820204FF02042411C21
:10D2A8006FF0704342F8213002F5827242F8203064
:10D2B800704770B584684568C368C16A02682543C9
:10D2C8001D4303691D4343691D4383691D43C369A6
:10D2D8001D43036A1D43436A1D43836A1D43036B51
:10D2E8000D431D434FF02043082C43F8225005D12D
:10D2F80053F8224044F0400443F82240436B9E69AF
:10D308001D6835435E6845EA06159E6845EA0625A8
:10D31800DE6845EA06451E695B6945EA0655541C00
:10D3280045EA03654FF02043B1F5804F43F8245098
:10D3380010D1836B986919680143586841EA001154
:10D34800986841EA002118695B6941EA005141EA9D
:10D35800036101E06FF07041014B43F8221070BD8A
:10D36800040100A0022242604FF480524262416BE5
:10D378004FF4005210B5826200230F22FF2403608D
:10D388008360C360036143618361C3610362C362F5
:10D3980003630A604A608C60CA600A614A618B61F3
:10D3A800816B0A604A608C60CA600A614A618B615D
:10D3B80010BD4FF0204321B153F8202042F0010264
:10D3C80003E053F82010024A0A4043F8202070472F
:10D3D800FEFF0F0010280CBF064B074B4FF0400212
:10D3E8004FF0180119605A604FF0FC329A60DA6009
:10D3F800704700BF600000A0800000A030B58368BF
:10D4080044681C43C36844F008041C4303691C4374
:10D41800436944EA4324836944EA4334C369996805
:10D428005A68090441EA02211A68DB68114341EA93
:10D438000361036A9A685D68120442EA05221D685E
:10D44800DB682A4342EA03620368102B0CBF034BD4
:10D45800034B1C609960DA6030BD00BF600000A01B
:10D46800800000A010230360C2690023436083602A
:10D47800C360036143618361FC231360536093605D
:10D48800D360026A136053609360D360704741B100
:10D4980010280CBF074B084B1A6842F004021A60A8
:10D4A800704710280CBF034A034A044B11680B400D
:10D4B80013607047600000A0800000A0FBFF0F0011
:10D4C80041B110280CBF084B084B1A6842F04002C3
:10D4D8001A60704710280CBF034A044A044B1168AD
:10D4E8000B401360704700BF600000A0800000A0E0
:10D4F800BFFF0F00102802D1024B58697047024B3A
:10D5080058697047600000A0800000A0054B1822F1
:10D518001A6000225A604FF0FC329A60DA601A6191
:10D52800704700BFA00000A00268436842F01002E4
:10D5380042EA4322836842EA4332144B10B51A6028
:10D54800C26891685468090441EA04211468D268E1
:10D55800214341EA02629A600269916854680904A9
:10D5680041EA04211468D268214341EA0262DA6080
:10D57800426991685068090441EA00211068D2683C
:10D58800014341EA02621A6110BD00BFA00000A079
:10D59800C2680023036043608360FC231360536008
:10D5A8009360D3600269136053609360D3604269EB
:10D5B800136053609360D3607047054B18B11A68C5
:10D5C80042F0040202E01968024A0A401A607047F1
:10D5D800A00000A0FBFF0F0062B1102801D10E4B84
:10D5E80003E0B0F5807F03D10C4B5A68114311E07A
:10D5F8000B4BFAE7102804D1074B5A6822EA0101BD
:10D6080008E0B0F5807F0CBF044B054B5A686FEA01
:10D618000101114059607047600000A0800000A01F
:10D62800A00000A0102801D1064B04E0B0F5807FCF
:10D638000CBF054B054B5B680B420CBF002001205B
:10D64800704700BF600000A0800000A0A00000A0FC
:10D65800102804D1074B5A6822EA010108E0B0F506
:10D66800807F0CBF044B054B5A686FEA01011140DB
:10D6780059607047600000A0800000A0A00000A0D2
:10D68800102801D1084B04E0B0F5807F0CBF074B90
:10D69800074B5B6813EA010004D013EAD1010CBF01
:10D6A80000200120704700BF600000A0800000A09B
:10D6B800A00000A0102804D1084B5A6822EAD10122
:10D6C80009E0B0F5807F0CBF054B064B5A684FEA5E
:10D6D800D10122EA01015960704700BF600000A033
:10D6E800800000A0A00000A008B52C4B984205D1EE
:10D6F8000120014600F048FC012048E0284B9842F0
:10D7080005D10220012100F03FFC02203FE0254B1B
:10D71800984205D10420012100F036FC042036E0AF
:10D72800214B984205D10820012100F02DFC08204A
:10D738002DE01E4B984205D11020012100F024FC59
:10D74800102024E01A4B984205D12020012100F036
:10D758001BFC20201BE0174B984205D140200121DB
:10D7680000F012FC402012E0134B984205D18020B3
:10D77800012100F009FC802009E0104B98420BD1F0
:10D788004FF48070012100F0FFFB4FF480700021FE
:10D79800BDE8084000F0F8BB08BD00BF000002402B
:10D7A8000004024000080240000C02400010024041
:10D7B8000014024000180240001C024000200240F1
:10D7C8002DE9F0470023D1F800801A464FF0010CEC
:10D7D80003270CFA02F404EA0805A5422ED10668CC
:10D7E80017FA03F4E443264006600E79D0F8009057
:10D7F80006FA03FA013E4AEA0909012EC0F8009028
:10D8080014D8866891F8059026408660866809FADB
:10D8180003F949EA06068660466826EA0505456072
:10D828008D7946689540ADB235434560C5682C4052
:10D83800C460CC79C5689C402C43C4600132023373
:10D84800102AC6D1BDE8F0874FF6FF7303600023A6
:10D85800037143718371C371704782B04FF4803391
:10D868000193019B0B430193019BC361C161019B20
:10D87800C361C3690193C369019302B07047036927
:10D8880019420CBF002001207047006980B2704720
:10D89800436919420CBF002001207047406980B2DB
:10D8A800704701837047418370470AB1018370470D
:10D8B800418370474161704743694B4043617047FA
:10D8C80001F00703C908083130B59B0050F8215012
:10D8D8000F249C4025EA040440F8214050F82140D8
:10D8E80012FA03F31C4340F8214030BD08B5134B2E
:10D8F800984207D14FF40010012100F069FB4FF462
:10D90800001014E00E4B984207D14FF4800001211B
:10D9180000F05EFB4FF4800009E00A4B98420BD1FF
:10D928004FF40000012100F053FB4FF400000021E8
:10D93800BDE8084000F04CBB08BD00BF00540040E3
:10D9480000580040005C00407FB504468688684661
:10D958000D4600F06DFA02992C482B6826F03F0618
:10D968003604B1FBF0F0360C80B20643A68022885C
:10D9780022F001021204120C2280254A93420AD88E
:10D988005B00B1FBF3F301309BB280B22084032B20
:10D9980098BF042321E0EE884BF6FF72964205D12A
:10D9A80003225343B1FBF3F39BB206E0192253431E
:10D9B800B1FBF3F39BB243F480431A054FF496721C
:10D9C80008BF43F0010350434FF47A7290FBF2F022
:10D9D800013080B243F400432084A38323886989FB
:10D9E800AA889BB243F001032380238823F4816330
:10D9F80023F002031B040A431B0C13439BB223802E
:10DA08002A89AB8913439BB223817FBD40420F0013
:10DA1800A086010041F288330360002383804BF61F
:10DA2800FF72038143814FF48043C2808381704732
:10DA3800038819B19BB243F0010303E023F001030B
:10DA48001B041B0C03807047038819B19BB243F475
:10DA5800807303E023F480731B041B0C038070475E
:10DA6800038819B19BB243F4007303E023F40073F5
:10DA78001B041B0C0380704712B141F0010101E047
:10DA880001F0FE0101827047038819B19BB243F48B
:10DA9800806303E023F480631B041B0C038070473E
:10DAA80083899BB201F0FE0123F0FE030B438381BF
:10DAB8007047838919B19BB243F0010303E023F057
:10DAC80001031B041B0C83817047038819B19BB2A7
:10DAD80043F0400303E023F040031B041B0C0380C6
:10DAE8007047038829B16FEA43436FEA53439BB2F7
:10DAF80001E05B045B0C03807047038819B99BB293
:10DB080043F0800303E023F080031B041B0C038015
:10DB18007047B1F5804F838B04D023F480431B04F6
:10DB28001B0C02E09BB243F4804383837047B1F53A
:10DB3800006F038803D19BB243F4006303E023F42E
:10DB480000631B041B0C03807047B1F5005F03885A
:10DB580003D19BB243F4005303E023F400531B04A6
:10DB68001B0C03807047038819B19BB243F0100364
:10DB780003E023F010031B041B0C03807047018291
:10DB88007047008AC0B27047038819B19BB243F44A
:10DB9800805303E023F480531B041B0C038070475D
:10DBA800B1F5006F038803D19BB243F4006303E02F
:10DBB80023F400631B041B0C03807047038819B10E
:10DBC8009BB243F0200303E023F020031B041B0C4B
:10DBD80003807047008BC0F307207047838819B112
:10DBE8009BB243F4006303E023F400631B041B0CA3
:10DBF80083807047838819B19BB243F4805303E054
:10DC080023F480531B041B0C8380704782B00023CD
:10DC180001930190019BCB180193019B188880B256
:10DC280002B0704783889BB20AB1194301E023EA26
:10DC3800010181807047838A008B9BB243EA0040D0
:10DC4800084020F07F40431A584240EB03007047D9
:10DC5800838A008B9BB243EA004020F07F407047E4
:10DC680082B00023009301930B0F01900093009B57
:10DC780021F07F4113B1019B143302E0019B090C91
:10DC880018330193019B1B6819420CBF0020012027
:10DC980002B07047C94389B2818270478388808AFD
:10DCA80080B208409BB206D001F0E06113EA11414E
:10DCB8000CBF002001207047C94389B28182704798
:10DCC8000A4B1A6842F001021A6000229A60196829
:10DCD80021F0847121F4803119600549596019686F
:10DCE80021F480211960DA60704700BF00380240D3
:10DCF80010300024024B00221A701870704700BFC1
:10DD080002380240034B1A6822F0F80242EAC002C5
:10DD18001A60704700380240014B1860704700BF16
:10DD280000004742064B002201281A701A7002D0E0
:10DD3800042804D101E01870704705221A70704752
:10DD480070380240014B1860704700BF800E474290
:10DD5800014341EA821200995B08013B42EA0161F2
:10DD680041EA0341014B5960704700BF0038024047
:10DD7800014B1860704700BF600047428001034BA9
:10DD880040EA0171C3F88410704700BF00380240B0
:10DD9800014B1860704700BF68004742014B18608C
:10DDA800704700BF4C004742034B9A6822F0EC6270
:10DDB80002430A439A60704700380240034B9A684E
:10DDC80022F0784202430A439A60704700380240C2
:10DDD800034B9A6822F0030202439A60704700BF1F
:10DDE80000380240024B986800F00C00704700BFF2
:10DDF80000380240034B9A6822F0F00202439A600E
:10DE0800704700BF00380240034B9A6822F4E05282
:10DE180002439A60704700BF00380240034B9A687B
:10DE280022F4604242EAC0029A6070470038024019
:10DE38001E4B9A6802F00C02042A10B503D0082A77
:10DE480003D01B4B18E01B4B16E059685A6811F4B5
:10DE5800800F596814BF174B154B02F03F02B3FBF4
:10DE6800F2F3124A5268C2F30142C1F38811013237
:10DE78004B435200B3FBF2F30C4903608B680E4A24
:10DE88000468C3F30313D35C34FA03F343608C6868
:10DE9800C4F38224145D33FA04F484608968C1F3FE
:10DEA8004231525CD340C36010BD00BF003802400D
:10DEB8000024F40000127A002804002000F44073C3
:10DEC800B3F5407F084B08D1996820F0704221F4DF
:10DED800F81122F440720A439A601A6F000542EA68
:10DEE80010501867704700BF00380240014B186097
:10DEF800704700BF3C0E4742014B1860704700BF97
:10DF0800400E4742014B1860704700BF5C01474212
:10DF1800044B1A6B09B1104301E022EA00001863B0
:10DF2800704700BF00380240044B5A6B09B11043D8
:10DF380001E022EA00005863704700BF0038024041
:10DF4800044B9A6B09B1104301E022EA0000986380
:10DF5800704700BF00380240044B1A6C09B11043E7
:10DF680001E022EA00001864704700BF0038024050
:10DF7800044B5A6C09B1104301E022EA00005864CE
:10DF8800704700BF00380240044B1A6909B11043BA
:10DF980001E022EA00001861704700BF0038024023
:10DFA800044B5A6909B1104301E022EA00005861A4
:10DFB800704700BF00380240044B9A6909B110430A
:10DFC80001E022EA00009861704700BF0038024073
:10DFD800044B1A6A09B1104301E022EA00001862F2
:10DFE800704700BF00380240044B5A6A09B1104319
:10DFF80001E022EA00005862704700BF0038024082
:10E00800044B1A6D09B1104301E022EA00001865BB
:10E01800704700BF00380240044B5A6D09B11043E5
:10E0280001E022EA00005865704700BF003802404E
:10E03800044B9A6D09B1104301E022EA000098658B
:10E04800704700BF00380240044B1A6E09B11043F4
:10E0580001E022EA00001866704700BF003802405D
:10E06800044B5A6E09B1104301E022EA00005866D9
:10E07800704700BF00380240044B1A7809B11043BA
:10E0880001E022EA00001870704700BF0D38024016
:10E098004309012B074A01D1136803E0022B0CBF87
:10E0A800136F536F00F01F0033FA00F000F0010007
:10E0B800704700BF0038024007B5002301933120A4
:10E0C800FFF7E6FF019B01330193019BB3F5A06FB6
:10E0D80001D00028F3D03120FFF7DAFF003018BF55
:10E0E80001200EBD024B5A6F42F080725A6770478A
:10E0F80000380240034BDB6818420CBF00200120A7
:10E10800704700BF00380240014B1870704700BFCD
:10E118000E38024008B5154B98420BD101214FF437
:10E128008050FFF761FF4FF480500021BDE80840A0
:10E13800FFF75ABF0E4B984207D14FF48040012198
:10E14800FFF746FF4FF4804009E00A4B98420BD195
:10E158004FF400400121FFF73BFF4FF4004000213E
:10E16800BDE80840FFF734BF08BD00BF00300140DC
:10E1780000380040003C00400B88028810B54C88ED
:10E1880023438C882343CC8823430C8923434C891D
:10E1980023438C892343CC8902F4415223431343FC
:10E1A8009BB20380838B23F400631B041B0C8383C3
:10E1B8000B8A038210BD838B23F47B6323F00F0348
:10E1C8001B041B0C8383022303848B68F0B5858BA7
:10E1D800022BADB238D0294A8E889468002E14BF1D
:10E1E80002260126240203D5946824F400049460CE
:10E1F800D2F88440D2F884705268DFF884C002F004
:10E208003F02BCFBF2F2C4F388145443C7F3027212
:10E21800B4FBF2F4CA88B2F5007F4FF00A0201D1CC
:10E22800240A02E07601B4FBF6F46243B2FBF3F38E
:10E2380005330A229BB2B3FBF2F303F00102120288
:10E24800C3F34F0392B200E000229C1EA4B2FE2C3E
:10E2580028BF0022CC8828BF0223134323439BB244
:10E2680003840B884A882B4343F4006313438A884A
:10E2780013438A8913439BB28383F0BD003802405D
:10E2880000127A000023038043808380C3800381C7
:10E2980043818381C38107230382704700230222BD
:10E2A800038043808380C3808260838170470388B2
:10E2B80019B19BB243F0400303E023F040031B0471
:10E2C8001B0C03807047838B19B19BB243F48063A6
:10E2D80003E023F480631B041B0C838370470388CB
:10E2E80023F400631B041B0C038003889BB20B43BD
:10E2F80003807047B1F5804F038803D19BB243F484
:10E30800804303E023F480431B041B0C0380704705
:10E318004FF6FF639942038803D09BB243F480739E
:10E3280003E023F480731B041B0C0380704783886D
:10E3380019B19BB243F0040303E023F004031B0468
:10E348001B0C83807047838819B19BB243F010037C
:10E3580003E023F010031B041B0C83807047838B9E
:10E3680023F47B6323F00F031B041B0C838302231A
:10E3780003840B88828BB3F5007F10B592B205D069
:10E38800002B0CBF4FF48073002301E04FF480731F
:10E398004C8822438C88898942F4006222430A43CC
:10E3A80092B21343838310BD808980B27047818104
:10E3B8007047038819B19BB243F4005303E023F478
:10E3C80000531B041B0C0380704703889BB243F463
:10E3D800805303807047012902D0008B80B27047B8
:10E3E800808A80B27047008A80B2704783889BB267
:10E3F8000AB1194301E023EA010181807047090944
:10E4080001238B409BB21AB1828892B2134303E076
:10E41800828892B222EA03038380704703891942F3
:10E428000CBF002001207047C94389B201817047A1
:10E4380010B584880089012301F00F0280B213FA15
:10E4480002F21040A4B205D009098B401C420CBF4F
:10E458000020012010BD01F00F0101238B40DB4398
:10E468009BB20381704700BF08B501214FF480407B
:10E47800FFF7BAFD4FF480400021BDE80840FFF7E0
:10E48800B3BD014B186070470038014001F003022A
:10E4980089080A4B023130B5920053F821500F24F5
:10E4A800944025EA040443F8214053F8214010FA27
:10E4B80002F2144343F8214030BD00BF0038014048
:10E4C800014B1860704700BFDC002742014B186001
:10E4D800704700BF00042742024B186AC0F30020AF
:10E4E800704700BF0038014030B5048C24F00104A7
:10E4F8002404240C0484058B048CADB2A4B225F04A
:10E50800F305154324F00A0445EA031544F0010411
:10E51800ADB20C430583048430BD30B5048C24F0BF
:10E5280010042404240C0484048B058C24F4407403
:10E53800ADB22405240D25F0A00544EA022445F0D7
:10E54800100544EA033445EA0115A4B2ADB20483C8
:10E55800058430BD08B5474B984205D101200146D6
:10E56800FFF742FD01203DE0B0F1804F05D10120C9
:10E578000146FFF72DFD012076E03F4B984205D17B
:10E5880002200121FFF724FD02206DE03B4B984259
:10E5980005D104200121FFF71BFD042064E0384B5E
:10E5A800984205D108200121FFF712FD08205BE001
:10E5B800344B984205D110200121FFF709FD1020A6
:10E5C80052E0314B984205D120200121FFF700FD90
:10E5D800202049E02D4B984209D102200121FFF764
:10E5E80003FD02200021BDE80840FFF7FDBC284BD1
:10E5F800984207D14FF480300121FFF7F5FC4FF422
:10E608008030EFE7234B984207D14FF400300121C7
:10E61800FFF7EAFC4FF40030E4E71F4B984207D1BC
:10E628004FF480200121FFF7DFFC4FF48020D9E769
:10E638001A4B984205D140200121FFF7C9FC402020
:10E6480012E0174B984205D180200121FFF7C0FC4A
:10E65800802009E0134B98420BD14FF480700121C0
:10E66800FFF7B6FC4FF480700021BDE80840FFF7C3
:10E67800AFBC08BD00000140000400400008004095
:10E68800000C00400010004000140040000401404D
:10E69800004001400044014000480140001800408B
:10E6A800001C0040002000401C4A038890429BB296
:10E6B80012D002F5806290420ED0B0F1804F0BD09C
:10E6C800A2F58032904207D002F58062904203D0D2
:10E6D80002F58062904203D14A8823F07003134305
:10E6E8000F4A904208D002F58062904204D023F489
:10E6F80040730A899BB2134303804B68C3620B883B
:10E708000385064B984203D003F58063984201D1F4
:10E718008B7A038601238382704700BF0000014083
:10E72800001000404FF0FF33436000230380038153
:10E73800438083727047018582827047038823F083
:10E7480070031B041B0C0B43038070474162704726
:10E75800C1627047406A7047008D80B27047038875
:10E7680019B19BB243F0020303E023F002031B0438
:10E778001B0C03807047038819B19BB243F0040354
:10E7880003E023F004031B041B0C03807047038879
:10E7980019B19BB243F0800303E023F080031B040C
:10E7A8001B0C03807047038823F008031B041B0C11
:10E7B800038003889BB20B4303807047038823F4CC
:10E7C80040731B041B0C038003889BB20B4303801C
:10E7D8007047038819B19BB243F0010303E023F0AB
:10E7E80001031B041B0C03807047038C23F00103F7
:10E7F8001B041B0C038470B5038C8488028B0D8862
:10E808004E8822F073021204120C2A438D8923F0D9
:10E8180002031B0435431B0CADB22B430E4DA8421B
:10E82800A4B203D005F58065A8420ED1CD894E8AE1
:10E8380023F008032B438D8823F004032B430D8A10
:10E84800354324F44074ADB22C43848002838A6833
:10E858004263038470BD00BF00000140038C23F0B5
:10E8680010031B041B0C0384038C828830B5048BB3
:10E878000D8824F4E6442404240C23F0200344EAFD
:10E8880005241B048D891B0C43EA05134D8843EAB4
:10E898000513134DA84292B2A4B29BB203D005F55A
:10E8A8008065A84215D1CD8923F080039BB243EA45
:10E8B80005134FF6BF751D408B8845EA03130D8A73
:10E8C80022F4406242EA85024D8A42EA85029BB2FE
:10E8D80092B282808A6804838263038430BD00BF59
:10E8E80000000140038C23F480731B041B0C038479
:10E8F800038C828830B5848B0D8824F0730424043B
:10E90800240C23F400731B042C438D891B0C43EA4D
:10E9180005234D8843EA0523124DA84292B29BB2C3
:10E9280003D005F58065A84215D1CD8923F400638D
:10E938009BB243EA05234FF6FF351D408B8845EA15
:10E9480003230D8A22F4405242EA05124D8A42EA14
:10E9580005129BB292B282808A688483C263038460
:10E9680030BD00BF00000140038C23F480531B041A
:10E978001B0C0384038C30B58488828B0D8822F4A9
:10E98800E6421204120C23F4005342EA05221B0447
:10E998008D891B0C43EA05334D8843EA05330B4D3B
:10E9A800A842A4B292B29BB203D005F58065A842F2
:10E9B80005D10D8A24F4804444EA8514A4B28480E5
:10E9C80082838A680264038430BD00BF000001406E
:10E9D800002303804380838083608381C381038213
:10E9E8004382704730B5058C0124ADB28C4025EACE
:10E9F800040400F11803048409B1082907D149085F
:10EA08004FF68F70CC582040C850C8580AE00439D7
:10EA1800C1F34E0148F6FF70CC582040C85012028E
:10EA2800C85892B20243CA5030BD416370478163EF
:10EA38007047C163704701647047038B23F070030C
:10EA48001B041B0C0B4303837047038B23F4E04325
:10EA58001B041B0C43EA01239BB203837047838B7F
:10EA680023F070031B041B0C0B4383837047838BB9
:10EA780023F4E0431B041B0C43EA01239BB283836A
:10EA88007047038B23F008031B041B0C0B43038301
:10EA98007047038B23F400631B041B0C43EA012318
:10EAA8009BB203837047838B23F008031B041B0C62
:10EAB8000B4383837047838B23F400631B041B0C75
:10EAC80043EA01239BB283837047038B23F004033B
:10EAD8001B041B0C0B4303837047038B23F48063D5
:10EAE8001B041B0C43EA01239BB203837047838BEF
:10EAF80023F004031B041B0C0B4383837047838B95
:10EB080023F480631B041B0C43EA01239BB2838319
:10EB18007047038B23F080031B041B0C0B430383F8
:10EB28007047038B09025B0441EA53439BB203839A
:10EB38007047838B23F080031B041B0C0B438383D8
:10EB48007047838B09025B0441EA53439BB283837A
:10EB58007047038C23F002031B041B0C0B43038434
:10EB68007047038C23F008031B041B0C0B4303841E
:10EB78007047038C23F020031B041B0C43EA01138A
:10EB88009BB203847047038C23F080031B041B0C87
:10EB980043EA01139BB203847047038C23F4007388
:10EBA8001B041B0C43EA01239BB203847047038CAC
:10EBB80023F400631B041B0C43EA01239BB2038468
:10EBC8007047038C23F400531B041B0C43EA0133E6
:10EBD8009BB20384704710B5048C01238B40A4B208
:10EBE80024EA03030384038C12FA01F10B439BB25A
:10EBF800038410BD10B5048C04238B40A4B224EA0E
:10EC080003030384038C12FA01F10B439BB20384C0
:10EC180010BD00230122038043808280C3800381CA
:10EC28007047406B7047806B7047C06B7047006CD3
:10EC38007047038B23F00C031B041B0C0383038B0B
:10EC48009BB20B4303837047038B23F440631B047D
:10EC58001B0C0383038B9BB243EA01239BB2038300
:10EC68007047F8B50C464988A288B4F800E02389B3
:10EC7800054600290CBF02270027012A14BF0126D8
:10EC88000226BEF1000F10D1FFF72EFC2846E188BE
:10EC9800FFF7CFFF2846394632462389FFF73DFC68
:10ECA800E1882846BDE8F840CEE7FFF736FC28465D
:10ECB800E188FFF7C9FF2846394632462389FFF71E
:10ECC80013FCE1882846BDE8F840B2E7838B23F0BF
:10ECD8000C031B041B0C8383838B9BB20B43838322
:10ECE8007047838B23F440631B041B0C8383838B43
:10ECF8009BB243EA01239BB283837047F8B50D4664
:10ED08000B88AA88498804463BB92B89FFF7ECFB96
:10ED1800E9882046BDE8F8408BE7042B07D12B890A
:10ED2800FFF7FBFBE9882046BDE8F8408CE7082B95
:10ED3800B5F808C0078C1DD127F480773F043F0C35
:10ED48000784868B038CB6B29BB226F0F30623F4B5
:10ED5800206346EA0C1C43EA01211FFA8CFC89B2A5
:10ED68004CEA020241F4807182830184E988BDE89B
:10ED7800F840ABE727F480573F043F0C0784868BA5
:10ED8800038C26F4407623F4005336055B04360DD5
:10ED98005B0C46EA022243EA013342EA0C329BB298
:10EDA800E98892B243F4805382830384BDE8F84033
:10EDB80097E74A880B8813438A881343CA88134302
:10EDC8000A8913434A8913438A8913439BB2A0F8DB
:10EDD800443070470023038043808380C3800381CD
:10EDE800438183817047B0F8443029B16FEA4343C7
:10EDF8006FEA53439BB201E05B045B0CA0F844301C
:10EE08007047838819B19BB243F0040303E023F0F1
:10EE180004031B041B0C83807047838819B19BB2C1
:10EE280043F0010303E023F001031B041B0C838060
:10EE3800704783899BB20AB1194301E023EA0101B3
:10EE48008181704781827047038A19420CBF002074
:10EE580001207047C94389B201827047038A8289B9
:10EE680011EA030092B203D011420CBF0020012026
:10EE78007047C94389B2018270470A43A0F8482005
:10EE8800704783899BB20AB1194301E023EA010163
:10EE980081817047838819B19BB243F0080303E06E
:10EEA80023F008031B041B0C83807047038923F09D
:10EEB80007031B041B0C03817047038923F07003AD
:10EEC8001B041B0C0B43038103899BB243F007030C
:10EED8000381704738B50D4611460122602D04465E
:10EEE80002D1FFF71AFB01E0FFF7FEFA238923F0AE
:10EEF80070031B041B0C1D43258123899BB243F01F
:10EF08000703238138BD038923F070031B041B0CFE
:10EF18000B4303817047838823F070031B041B0C89
:10EF2800838083889BB20B4383807047038923F0D7
:10EF380007031B041B0C038103899BB20B4303814A
:10EF48007047038923F080031B041B0C038103898A
:10EF58009BB20B430381704710B50489E4B20C439C
:10EF6800144344EA0324A4B2048110BD10B5044636
:10EF7800FFF7F2FF23899BB243F48043238110BD3E
:10EF880010B50446FFF7E8FF238923F077031B0435
:10EF98001B0C43F07703238110BD70B50489068BE1
:10EFA800058C26F44076ADB226F0030624F007045B
:10EFB800360425F022052404360C1543240C46F4A7
:10EFC800807645EA0315214346F00106ADB201817A
:10EFD8000683058470BD838819B19BB243F0800312
:10EFE80003E023F080031B041B0C83807047A0F808
:10EFF8005010704708B5234B984205D110200121C5
:10F00800FEF7F2FF102037E01F4B984207D14FF46C
:10F0180000300121FEF7DCFF4FF4003009E01B4B04
:10F0280098420BD14FF480200121FEF7D1FF4FF415
:10F0380080200021BDE80840FEF7CABF144B984263
:10F0480007D14FF400200121FEF7C2FF4FF4002042
:10F05800EFE7104B984207D14FF480100121FEF7DB
:10F06800B7FF4FF48010E4E70B4B984209D12020FA
:10F078000121FEF7B9FF20200021BDE80840FEF776
:10F08800B3BF08BD001001400044004000480040E4
:10F09800004C00400050004000140140038ACA8818
:10F0A8009BB223F4405330B513430D460382838942
:10F0B8000989AA8823F4B0530A43698923F00C0309
:10F0C8001B040A431B0C92B213438381838AAA89C7
:10F0D8009BB223F44073134385B083820446684689
:10F0E800FEF7A6FE1A4B9C4203D003F580639C42B0
:10F0F80001D1039B00E0029BA28912B2002A4FF0C3
:10F1080019012A6801FB03F101DA520000E09200BC
:10F118006423B1FBF2F1B1FBF3F21201100903FB16
:10F128001011A08900B2002806DAC9003231B1FBFB
:10F13800F3F303F0070305E009013231B1FBF3F300
:10F1480003F00F031A4392B2228105B030BD00BF0D
:10F15800001001404FF4165303600C2200238380F3
:10F16800C38003814281838170470B88028A10B56E
:10F178004C8823438C88C988234392B20B4322F4DA
:10F1880070629BB21343038210BD00230380438047
:10F198008380C3807047838919B19BB243F40053BD
:10F1A80003E023F400531B041B0C83817047038B7B
:10F1B80003F47F430383038B9BB20B4303837047A2
:10F1C800838929B16FEA43436FEA53439BB201E055
:10F1D8005B045B0C83817047838A19B19BB243F44B
:10F1E800006303E023F400631B041B0C8382704755
:10F1F800C905C90D818070478088C005C00D70475A
:10F20800038A23F00F031B041B0C0382038A9BB29F
:10F218000B4303827047838919B19BB243F0020301
:10F2280003E023F002031B041B0C838170478389CE
:10F2380023F400631B041B0C838183899BB20B435B
:10F2480083817047038A23F020031B041B0C03826D
:10F25800038A9BB20B4303827047038A19B19BB29E
:10F2680043F4804303E023F480431B041B0C038214
:10F27800704783899BB243F0010383817047838A77
:10F2880019B19BB243F0080303E023F008031B0401
:10F298001B0C83827047038BDBB20383038B9BB207
:10F2A80043EA012303837047838A19B19BB243F071
:10F2B800200303E023F020031B041B0C8382704708
:10F2C800838A19B19BB243F0100303E023F01003C3
:10F2D8001B041B0C83827047838A23F004031B04DE
:10F2E8001B0C8382838A9BB20B4383827047838A79
:10F2F80019B19BB243F0020303E023F002031B049D
:10F308001B0C83827047838A9BB20AB1194301E0C0
:10F3180023EA010181827047C1F3421310B501F05D
:10F328001F01012414FA01F1A34201D10C3004E0B9
:10F33800022B01D1103000E0143003680AB11943E0
:10F3480001E023EA0101016010BD038819420CBFE6
:10F35800002001207047C94389B20180704701220B
:10F3680010B501F01F03C1F342149A40012C01D1DA
:10F37800838903E0022C0CBF038A838A9BB2134063
:10F38800028892B243B1090A012313FA01F111422A
:10F398000CBF0020012010BD184610BD090A01232A
:10F3A8008B40DB439BB20380704700BF81F0004174
:10F3B80002E000BF83F0004330B54FEA41044FEA52
:10F3C800430594EA050F08BF90EA020F1FBF54EAED
:10F3D800000C55EA020C7FEA645C7FEA655C00F089
:10F3E800E2804FEA5454D4EB5555B8BF6D420CDD5A
:10F3F8002C4480EA020281EA030382EA000083EADD
:10F40800010180EA020281EA0303362D88BF30BD7C
:10F4180011F0004F4FEA01314FF4801C4CEA1131D2
:10F4280002D0404261EB410113F0004F4FEA033331
:10F438004CEA133302D0524263EB430394EA050FBC
:10F4480000F0A780A4F10104D5F1200E0DDB02FA2B
:10F458000EFC22FA05F2801841F1000103FA0EF2BF
:10F46800801843FA05F359410EE0A5F120050EF185
:10F47800200E012A03FA0EFC28BF4CF0020C43FAB6
:10F4880005F3C01851EBE37101F0004507D54FF0C3
:10F49800000EDCF1000C7EEB00006EEB0101B1F513
:10F4A800801F1BD3B1F5001F0CD349085FEA300059
:10F4B8004FEA3C0C04F101044FEA445212F5800F64
:10F4C80080F09A80BCF1004F08BF5FEA500C50F101
:10F4D800000041EB045141EA050130BD5FEA4C0CE4
:10F4E800404141EB010111F4801FA4F10104E9D16D
:10F4F80091F0000F04BF01460020B1FA81F308BF64
:10F508002033A3F10B03B3F120020CDA0C3208DD2F
:10F5180002F1140CC2F10C0201FA0CF021FA02F10A
:10F528000CE002F11402D8BFC2F1200C01FA02F17A
:10F5380020FA0CFCDCBF41EA0C019040E41AA2BF9F
:10F5480001EB0451294330BD6FEA04041F3C1CDA67
:10F558000C340EDC04F11404C4F1200220FA04F087
:10F5680001FA02F340EA030021FA04F345EA030131
:10F5780030BDC4F10C04C4F1200220FA02F001FAF3
:10F5880004F340EA0300294630BD21FA04F0294675
:10F5980030BD94F0000F83F4801306BF81F480110E
:10F5A8000134013D4EE77FEA645C18BF7FEA655C81
:10F5B80029D094EA050F08BF90EA020F05D054EA53
:10F5C800000C04BF1946104630BD91EA030F1EBF58
:10F5D8000021002030BD5FEA545C05D1400049415C
:10F5E80028BF41F0004130BD14F580043CBF01F54F
:10F5F800801130BD01F0004545F0FE4141F4700135
:10F608004FF0000030BD7FEA645C1ABF194610460F
:10F618007FEA655C1CBF0B46024650EA013406BF10
:10F6280052EA033591EA030F41F4002130BD00BFCF
:10F6380090F0000F04BF0021704730B54FF480648C
:10F6480004F132044FF000054FF0000150E700BF0D
:10F6580090F0000F04BF0021704730B54FF480646C
:10F6680004F1320410F0004548BF40424FF0000159
:10F678003EE700BF42004FEAE2014FEA31014FEA9C
:10F6880002701FBF12F07F4393F07F4F81F06051EB
:10F69800704792F0000F14BF93F07F4F704730B55A
:10F6A8004FF4607401F0004521F0004120E700BFED
:10F6B80050EA010208BF704730B54FF000050AE074
:10F6C80050EA010208BF704730B511F0004502D575
:10F6D800404261EB41014FF4806404F132045FEA77
:10F6E800915C3FF4DCAE4FF003025FEADC0C18BF1C
:10F6F80003325FEADC0C18BF033202EBDC02C2F112
:10F70800200300FA03FC20FA02F001FA03FE40EAA3
:10F718000E0021FA02F11444C1E600BF70B54FF0A3
:10F72800FF0C4CF4E06C1CEA11541DBF1CEA135585
:10F7380094EA0C0F95EA0C0F00F0DEF82C4481EAED
:10F74800030621EA4C5123EA4C5350EA013518BF0D
:10F7580052EA033541F4801143F4801338D0A0FBFA
:10F7680002CE4FF00005E1FB02E506F00042E0FBA7
:10F7780003E54FF00006E1FB03569CF0000F18BFAD
:10F788004EF0010EA4F1FF04B6F5007F64F5407455
:10F7980004D25FEA4E0E6D4146EB060642EAC621E8
:10F7A80041EA55514FEAC52040EA5E504FEACE2E55
:10F7B800B4F1FD0C88BFBCF5E06F1ED8BEF1004F58
:10F7C80008BF5FEA500E50F1000041EB045170BDD4
:10F7D80006F0004646EA010140EA020081EA030118
:10F7E800B4EB5C04C2BFD4EB0C0541EA045170BD14
:10F7F80041F480114FF0000E013C00F3AB8014F18E
:10F80800360FDEBF002001F0004170BDC4F10004D6
:10F81800203C35DA0C341BDC04F11404C4F1200557
:10F8280000FA05F320FA04F001FA05F240EA0200B2
:10F8380001F0004221F0004110EBD37021FA04F6E8
:10F8480042EB06015EEA430E08BF20EAD37070BDA2
:10F85800C4F10C04C4F1200500FA04F320FA05F001
:10F8680001FA04F240EA020001F0004110EBD37003
:10F8780041F100015EEA430E08BF20EAD37070BD73
:10F88800C4F1200500FA05F24EEA020E20FA04F34C
:10F8980001FA05F243EA020321FA04F001F00041FB
:10F8A80021FA04F220EA020000EBD3705EEA430E6C
:10F8B80008BF20EAD37070BD94F0000F0FD101F09B
:10F8C8000046400041EB010111F4801F08BF013CD4
:10F8D800F7D041EA060195F0000F18BF704703F012
:10F8E8000046520043EB030313F4801F08BF013D99
:10F8F800F7D043EA0603704794EA0C0F0CEA135555
:10F9080018BF95EA0C0F0CD050EA410618BF52EA0E
:10F918004306D1D181EA030101F000414FF0000014
:10F9280070BD50EA410606BF1046194652EA430622
:10F9380019D094EA0C0F02D150EA013613D195EA96
:10F948000C0F05D152EA03361CBF104619460AD1DE
:10F9580081EA030101F0004141F0FE4141F47001E8
:10F968004FF0000070BD41F0FE4141F4780170BDD8
:10F9780070B54FF0FF0C4CF4E06C1CEA11541DBF3D
:10F988001CEA135594EA0C0F95EA0C0F00F0A7F83F
:10F99800A4EB050481EA030E52EA03354FEA01316C
:10F9A80000F088804FEA03334FF0805545EA13137F
:10F9B80043EA12634FEA022245EA111545EA106547
:10F9C8004FEA00260EF000419D4208BF964244F1DE
:10F9D800FD0404F5407402D25B084FEA3202B61AFD
:10F9E80065EB03055B084FEA32024FF480104FF4D1
:10F9F800002CB6EB020E75EB030E22BFB61A754645
:10FA080040EA0C005B084FEA3202B6EB020E75EBD7
:10FA1800030E22BFB61A754640EA5C005B084FEA3F
:10FA28003202B6EB020E75EB030E22BFB61A75460C
:10FA380040EA9C005B084FEA3202B6EB020E75EB17
:10FA4800030E22BFB61A754640EADC0055EA060ED8
:10FA580018D04FEA051545EA16754FEA06164FEA1B
:10FA6800C30343EA52734FEAC2025FEA1C1CC0D1C7
:10FA780011F4801F0BD141EA00014FF000004FF054
:10FA8800004CB6E711F4801F04BF01430020B4F115
:10FA9800FD0C88BFBCF5E06F3FF6AFAEB5EB030CCD
:10FAA80004BFB6EB020C5FEA500C50F1000041EBCA
:10FAB800045170BD0EF0004E4EEA113114EB5C0497
:10FAC800C2BFD4EB0C0541EA045170BD41F480116A
:10FAD8004FF0000E013C90E645EA060E8DE60CEA72
:10FAE800135594EA0C0F08BF95EA0C0F3FF43BAF8F
:10FAF80094EA0C0F0AD150EA01347FF434AF95EA46
:10FB08000C0F7FF425AF104619462CE795EA0C0F29
:10FB180006D152EA03353FF4FDAE1046194622E7F6
:10FB280050EA410618BF52EA43067FF4C5AE50EAD0
:10FB380041047FF40DAF52EA43057FF4EBAE12E7C0
:10FB48004FF0FF3C06E000BF4FF0010C02E000BFA1
:10FB58004FF0010C4DF804CD4FEA410C7FEA6C5C84
:10FB68004FEA430C18BF7FEA6C5C1BD001B050EA27
:10FB7800410C0CBF52EA430C91EA030F02BF90EA12
:10FB8800020F0020704710F1000F91EA030F58BFD1
:10FB9800994208BF90422CBFD8176FEAE37040F033
:10FBA800010070474FEA410C7FEA6C5C02D150EAD1
:10FBB800013C07D14FEA430C7FEA6C5CD6D152EA8C
:10FBC800033CD3D05DF8040B704700BF8446104651
:10FBD80062468C461946634600E000BF01B5FFF750
:10FBE800B7FF002848BF10F1000F01BD4DF808ED20
:10FBF800FFF7F4FF0CBF012000205DF808FB00BFF1
:10FC08004DF808EDFFF7EAFF34BF012000205DF84A
:10FC180008FB00BF4DF808EDFFF7E0FF94BF012097
:10FC280000205DF808FB00BF4DF808EDFFF7CEFF98
:10FC380094BF012000205DF808FB00BF4DF808EDD7
:10FC4800FFF7C4FF34BF012000205DF808FB00BFA8
:10FC58004FEA410212F5001215D211D56FF47873EC
:10FC6800B3EB625212D94FEAC12343F0004343EA8F
:10FC7800505311F0004F23FA02F018BF404270476A
:10FC88004FF00000704750EA013005D111F00040F4
:10FC980008BF6FF0004070474FF00000704700BF8A
:10FCA8004A0011D212F5001211D20DD56FF47873F3
:10FCB800B3EB62520ED44FEAC12343F0004343EA48
:10FCC800505323FA02F070474FF00000704750EA93
:10FCD800013002D14FF0FF3070474FF000007047FD
:10FCE8004FEA4102B2F1E04324BFB3F5001CDCF156
:10FCF800FE5C0DD901F0004C4FEAC0024CEA50708E
:10FD0800B2F1004F40EB830008BF20F001007047BC
:10FD180011F0804F21D113F13872BCBF01F00040BF
:10FD2800704741F480114FEA5252C2F11802C2F1F1
:10FD3800200C10FA0CF320FA02F018BF40F0010072
:10FD48004FEAC1234FEAD32303FA0CFC40EA0C0024
:10FD580023FA02F34FEA4303CCE77FEA625307D161
:10FD680050EA01331EBF4FF0FE4040F44000704798
:10FD780001F0004040F0FE4040F40000704700BF32
:10FD88004BB942B9002908BF002802D04FF0FF3113
:10FD9800084600F037B882B0EC462DE9005000F074
:10FDA8001BF8DDF804E002B00CBC7047F8B5144647
:10FDB80006460F461D4600F027F804FB01F300FB3A
:10FDC8000535A4FB0023EB18069CB21A67EB030366
:10FDD800C4E90023F8BD00BFF8B5144606460F462F
:10FDE8001D4600F075F900FB05F5A0FB042304FB94
:10FDF8000155EB18069CB21A67EB0303C4E900230C
:10FE0800F8BD00BF704700BF00292DE9F0071D4667
:10FE1800C0F29E800024002DC0F2958007460D4652
:10FE280016469C46002B3ED18A4254D9B2FA82F338
:10FE380043B1C3F1200620FA06F501FA03F19A400E
:10FE480029439840160CB1FBF6F597B206FB15113D
:10FE58004FEA104C07FB05F34CEA01418B4209D9E4
:10FE6800891805F1FF3C80F015818B4240F2128120
:10FE7800023D8918C3EB010CBCFBF6F306FB13C16A
:10FE880080B207FB03F740EA0140874207D9591EB1
:10FE9800821880F00581974240F20281023B43EAD2
:10FEA8000542002303E08B420AD900231A46104674
:10FEB800194614B1404261EB4101BDE8F0077047B3
:10FEC800B3FA83F3002B40F087808C4501D382423C
:10FED800ECD80122EBE712B90123B3FBF2F2B2FA34
:10FEE80082F6002E3AD1891A150C1FFA82FC0123DA
:10FEF800B1FBF5F705FB17114FEA10480CFB07F6A5
:10FF080048EA01418E4207D9891807F1FF3802D221
:10FF18008E4200F2DA804746891BB1FBF5F605FBF5
:10FF2800161180B20CFB06FC40EA0140844507D953
:10FF3800711E821880F0B080944540F2AD80023E78
:10FF480046EA0742B3E7E443524263EB430365E7FB
:10FF5800404261EB41014FF0FF345CE7B240C6F12B
:10FF6800200521FA05F320FA05F701FA06F9150C20
:10FF7800B3FBF5F847EA09091FFA82FC05FB1837B5
:10FF88004FEA19410CFB08F341EA0747B040BB426E
:10FF98000AD9BF1808F1FF3180F09580BB4240F2C2
:10FFA8009280A8F10208BF18FE1AB6FBF5F305FB0C
:10FFB80013611FFA89F90CFB03F649EA01418E42E5
:10FFC80006D95F1E891878D28E4276D9023B8918E5
:10FFD800891B43EA08438BE7C3F1200726FA07F891
:10FFE8000CFA03F248EA020C21FA07F105FA03FABF
:08FFF8004FEA1C4920FA07F54D
:020000040801F1
:10000000B1FBF9F845EA0A0509FB18172A0C1FFA93
:100010008CFA0AFB08F142EA0747B94206FA03F6EE
:1000200009D917EB0C0708F1FF324ED2B9424CD96F
:10003000A8F1020867447F1AB7FBF9F209FB1271B5
:10004000ADB20AFB02FA45EA01418A4507D9551EBD
:1000500011EB0C0137D28A4535D9023A614442EAA4
:1000600008424FEA124C1FFA86F808FB0CF7360CD0
:1000700095B208FB05F806FB057505EB184506FB70
:100080000CFCAF4288BF0CF5803CCAEB01010CEBC5
:100090001546B14212D309D000230CE76546EDE6C0
:1000A0000E4646EA074206E70B46FCE61FFA88F8CA
:1000B00000FA03F308EB0545AB42EDD2013A002309
:1000C000F9E63B4688E72A46C9E79046B3E7884603
:1000D0006EE7023F891823E72DE9F00F1446054625
:1000E0000E46002B3FD18A424AD9B2FA82F343B17D
:1000F000C3F1200025FA00F201FA03F69C401643F2
:100100009D40210CB6FBF1F22F0CA0B201FB126C4A
:1001100000FB02F347EA0C46B34208D9571E3619D2
:1001200080F0FF80B34240F2FC80023A3619F61AA2
:10013000B6FBF1F301FB1361ADB200FB03F045EA3E
:100140000141884207D95E1E091980F0EC8088427F
:1001500040F2E980023B43EA02420023104619467E
:10016000BDE8F00F70478B4243D8B3FA83F4002CFC
:1001700042D18B42234601D382423BD80122EDE794
:1001800012B90123B3FBF2F4B4FA84F2002A40F06E
:100190008A80091B260CA7B20123B1FBF6F006FBEF
:1001A00010114FEA154C07FB00F24CEA01418A425C
:1001B00007D9091900F1FF3C02D28A4200F2D3802C
:1001C0006046C2EB010CBCFBF6F206FB12C1ADB2FD
:1001D00007FB02F745EA0145AF4207D9511E2C192A
:1001E00080F0A380A74240F2A080023A42EA004297
:1001F000B4E700231A46B1E7C4F1200722FA07F654
:1002000003FA04F3334321FA07FA4FEA134C01FAD5
:1002100004FB20FA07F141EA0B0BBAFBFCF70CFBDD
:1002200017A61FFA83F84FEA1B4508FB07F945EAB2
:100230000645A94502FA04FA04D97A1EED18C0F061
:1002400088801746C9EB0505B5FBFCF60CFB16527A
:100250001FFA8BFB08FB06F84BEA0241884503D9DD
:10026000721EC91870D3164646EA0742170C1FFAC9
:100270008AFC0CFB07F695B24FEA1A430CFB05FC0F
:1002800003FB056505EB1C4503FB07F3AE4288BF86
:1002900003F58033C8EB010103EB1543994250D3BA
:1002A00047D000235AE79440C2F12008260C20FAD8
:1002B00008F721FA08F501FA02F9B5FBF6F847EA62
:1002C000090906FB1855A7B24FEA194C4CEA054C30
:1002D00007FB08F3634500FA02F509D91CEB040C8F
:1002E00008F1FF323DD263453BD9A8F10208A4448E
:1002F000C3EB0C02B2FBF6F306FB13201FFA89F9DD
:1003000007FB03F249EA00418A4206D9581E09193F
:1003100025D28A4223D9023B0919891A43EA0843A4
:100320003BE73A4603E7334615E70A4642EA00420E
:1003300014E71FFA8CF100FA04F001EB0545A8421E
:10034000AFD2013A002309E788458CD9023EC9188B
:100350008AE7A9457FF675AF023FED1872E70346BD
:10036000DBE79046C4E7023809192AE7002103E0D9
:100370000A4B5B584350043109480A4B42189A42D1
:10038000F6D3094A02E0002342F8043B074B9A42A5
:10039000F9D3FAF7B5F900F00DF87047CCAF0508BE
:1003A00000000020FC0C0020000D00200453002061
:1003B000FEE70000B14BF7B54FF4FA661E60B04A95
:1003C000B04BB14F1A60B14AB14B1A60B14B42F217
:1003D00010721A60B04B64241C6001233B70F8F764
:1003E00086FDAE4B00251D70F7F714FFF5F7C0FF33
:1003F000F5F7CAFFF5F7D8FFF6F7D4FD2046F7F773
:1004000051FAF6F7F5FD2046F7F74CFAF7F7E8FE54
:10041000F7F7F6FCF7F754FA2046F7F743FAFAF73E
:10042000C1FA2046F7F73EFA4FF4FA50F7F7A6F96B
:100430002046F7F737FAF6F70DFD2046F7F732FAC0
:100440002846F7F711FB9648F7F72CFAF4F7D4FA99
:100450002046F7F727FA934B03F1100229468DE85F
:10046000240028465A681B68F4F7D8F83046F7F796
:1004700019FA2846F4F7AAFC4FF6FF70F4F7BCFC13
:1004800003213220884A2B46F4F7DAFD9620874A6A
:100490008C212B46F4F7D4FD9620A021844A2B46CC
:1004A000F4F7CEFD834A2B469620B421F4F7C8FD1D
:1004B000F8F7D4FC5021DC20F8F7A3FC3046F7F71E
:1004C000F1F97D4A2B46DC212846F4F7B9FD7B483B
:1004D000F7F7E8F92046F7F7E5F9F6F763FA20466B
:1004E000F7F7E0F99FED760AF7F7D6FA2046F7F727
:1004F000D9F9F7F7FFF9F5F76DF82046F7F7D2F9D4
:1005000014200146F5F7BCFF2846F6F70FF8204601
:10051000F7F7C8F9F6F790F92046F7F7C3F9F6F7B9
:1005200039FD2046F7F7BEF9F6F78CFA00B13D70B9
:10053000F6F794FA08B1F8F73BFC624B00241C7004
:10054000F1F730F8F4F7FCFF08B95F4802E05F4BC1
:100550005F481C70F1F741F8F5F766FCF8F775F99C
:10056000F8F7A8F9F8F71AFFF7F75CFFF8F743FC7C
:10057000FAF77AF9F8F792FC564B574D574C80280A
:1005800014BF4FF480504FF480601880404B1A68BD
:100590003C4B1B68D31A06EE903A3E4B1B68B8EEF4
:1005A000E67A06EE903AF8EEE67A2E46C7EE277A1D
:1005B00017EE900AFFF762F8494B0022FEF700FFA2
:1005C000FFF772FB474B01301880F6F75DFA2B7886
:1005D00033B1012B02D1F7F741FC01E0F7F766FCDC
:1005E00000273770F7F7E4FDF3F706F8F9F7F8FF9F
:1005F000237813B12770F1F765FC384B5B781BB19A
:1006000000236370F1F7DCF8374B1A8812B2012A25
:1006100013D136484FF40051FDF74BF9A3780BB9CD
:10062000F8F788FFF7F72EFD002230484FF400510D
:10063000FDF73FF92C4B00221A80E3783BB10020F4
:10064000E070F3F7BDFE2A4B1878F0F729FB237909
:1006500043B1F8F703FCF0209621F8F7D2FB2548C8
:10066000F6F716FF244F3846FBF787FC0028ACD07E
:100670003B78112BA9D1F8F713FBA6E7803E0020A9
:10068000E0673500B03E00202C0F002080C3C90178
:10069000CC440020A4440020603E002044460020BA
:1006A00000127A00E087010834A805084EA8050862
:1006B00059A8050865A805086EA80508002D310190
:1006C0000000FA44903E00205C110020483E0020CB
:1006D00048130020AC3E0020A84400200C0E00204F
:1006E0000000E03F0C480020F00D00200008024010
:1006F000C044002040420F00493E002010B4314C5D
:100700000180B1F5807F44608270C37052D00DD9F2
:10071000B1F5806F39D017D9B1F5006F2ED0B1F592
:10072000805F24D0FF2040B210BC704720293AD00F
:1007300014D9402930D08029F4D123494FF0201218
:10074000C26081600020EEE7B1F5007FEAD11F4B67
:100750004FF00811C16083600020E4E71029E1D167
:100760001B494FF00122C26081600020DBE7194B7A
:100770004FF00111C16083600020D4E7164A4FF0AA
:100780000213C36082600020CDE714494FF00412C9
:10079000C26081600020C6E7114B4FF04011C1607C
:1007A00083600020BFE70F4A4FF08013C360826070
:1007B0000020B8E70C4A4FF01013C360826000209D
:1007C000B1E700BFC4A6040802970508D296050841
:1007D000C2980508C4960508C6960508CA96050875
:1007E00042970508C2970508E29605082DE9F00F23
:1007F000B2B02E9030932E9B00882E9C5B68309F69
:10080000A4682D90451E03EB4506BF08209328944D
:100810002C952F911F921E96319700F03A814FEA46
:10082000900A4FEACA0B00F003002F99299003F1B8
:10083000080504EB0B00CDF884A0CDF8A8B01995FD
:100840001A921B97189617912B90179A189E138837
:100850003380B2F802C0A6F802C09488B480D7886A
:10086000F78008361896219F199E0832179256F87D
:10087000041C56F8082C4FF0000A4FF0000B002F14
:1008800000F06982CDE904ABCDE906ABCDE902AB5E
:10089000CDE900AB289CBC46029BDDF80C90256896
:1008A000C2FBC5394FF0000848EA030ACB46CDE940
:1008B00002AB049BDDF814B0C1FBC53BCDF824B0FE
:1008C000CDF82080DDE908ABC1EA02004AEA030A5C
:1008D000CDE904AB069BDDF81CB03268C0FBD53B0C
:1008E000CDF82CB0CDF82880DDE90AABC2EA0107CB
:1008F0004AEA030ACDE906AB9DE80108C7FBD50B20
:10090000CDF834B0CDF83080DDE90CAB4AEA000A0E
:1009100063680298CDE900AB0834DDF80CB0C1FB88
:10092000C30BCDF83CB0CDF83880DDE90EAB4AEA18
:10093000000ACDE902AB71680498DDF814B0C2FB7F
:10094000C30BCDF844B0CDF84080DDE910AB4AEAE6
:10095000000ACDE904AB0698DDF81CB0C7FBD30B49
:10096000CDF84CB0CDF84880DDE912ABC1EA020504
:100970004AEA000ACDE906AB9DE80108C5FBD30BA6
:10098000CDF854B0CDF85080DDE914AB08364AEA12
:10099000000ABCF1010CCDE900AB7FF47DAF2A9DCC
:1009A00019982B9B2E18299F002F35D01868039F6C
:1009B000029BC2FBC03700241D971C94DDE91C4537
:1009C00044EA0304CDE90245049B059DC1FBC03503
:1009D000002723952297DDE9224544EA0304CDE967
:1009E0000445C1EA0203079D069AC3FBD02525955D
:1009F0002497DDE9244544EA02043368C3EA01018F
:100A0000CDE9064553465D46C1FBD035279526976F
:100A1000DDE926AB4AEA030A069A029C0499039D83
:100A2000079FD30B059AE60BC90B46EA454043EAFC
:100A3000474441EA424604F30F0500F30F0C199BAB
:100A4000CCEA054706F30F001A9D1B9E2F604FEA64
:100A5000DA3A08334AEA4B4B0BF30F04C0EA04427C
:100A60006A600835711E19931A951B917FF4EDAEDB
:100A7000319A2F9E1E991F9BDDF880B0D000371849
:100A80000D182F970BEB000A1F181E951F97CDF816
:100A900080A0DDF8C0C01CF0030BCDF820B000F042
:100AA00086802D9BDDF8BC80CDF808B05808DDF8B5
:100AB00080A0DDF8A0B00690CDF81080049A1E9EAC
:100AC00032F8025B069826F8025B0492BAF80270CC
:100AD000BBF80230BAF80020BBF800401E9617FBA6
:100AE00003F112FB04F6451E4FEAE17711EB06080D
:100AF0002B4605F0010047EBE6790AF104020BF101
:100B00000401002D3BD0A8B1B2F800C0BBF80470BE
:100B1000548848881CFB07F518EB050749EBE57678
:100B200014FB00F917EB090846EBE97904320431AC
:100B3000013B24D00F88B2F800C0568848888C88C2
:100B400095881CFB07FC18EB0C0816FB00F7D088F7
:100B5000CE8849EBEC7C15FB04F518EB07084CEB51
:100B6000E77918EB050710FB06FC49EBE57417EB7A
:100B70000C0844EBEC7908320831023BDAD11F9AB9
:100B800002994FEAD83545EA494404F30F0322F8A5
:100B9000023B4F1E0AF1020A1F9202978ED1DDF826
:100BA00080A0DDF820B00AEB4B0ACDF880A02C9E87
:100BB0002E98B50840683FD0209F47EA000212F007
:100BC000030F00F1080307F1080214BF00210121FF
:100BD0009F4298BF904294BF00260126314277D0B1
:100BE00097E84200016001216C1EA942466004EAB8
:100BF000010419D044B192E81200196002215C602E
:100C000008320833A9420FD092E850001C605E60A1
:100C1000966802F1080BD2689E600231DA601033E8
:100C2000A9420BF10802EFD1DDF880C0ED000CEB1A
:100C3000050B4019CDF880B02C9C14F0030343D071
:100C40005A085400002A00F08E80209D40EA0507D3
:100C500017F0030F209F14BF00250125011D3E1D25
:100C6000012B94BF002505F001058F4298BFB042CB
:100C700094BF002101210D4275D039689200BF1840
:100C8000A342016020971044C4EB03011CD0209BB9
:100C9000013933F8024B0A4620F8024B01F00101FA
:100CA00092B129B133F8021B013A20F8021B0BD094
:100CB0001C46014634F802CB21F802CB5D88A31C08
:100CC0004580881C023AF3D132B0BDE8F00F70477E
:100CD000B7F800C0A0F800C07C884480BE88868039
:100CE000691EFE880C46BA4601F00101C680002C40
:100CF0009AD089B1B2F800B0A3F800B051885980F9
:100D0000B2F804C0A3F804C0B2F806B00832A3F8E1
:100D100006B00833013C87D016881E805188598060
:100D2000B2F804B0A3F804B0B2F806C0A3F806C045
:100D300016891E8103F1080B5189ABF802109389C3
:100D4000ABF80430D6891032023C0BF10803ABF843
:100D50000660E1D168E7289BCDE904ABCDE906AB9D
:100D6000CDE902AB1FE6194691E700BF2DE9F00F70
:100D70009CB006780F900F9C40880F9DA4686D680A
:100D80001990B3FBF6FA471E4FEA5A0804EB4709DD
:100D9000AAEB480340460A940D951A97CDF86C804B
:100DA0000C911492CDF82C901193002800F0B5818D
:100DB0001746199A199CCDF848809108CA001591D8
:100DC00004F00303A9181792169310971891760050
:100DD00075084FEA450C002D00F03B840B9FDDF8B1
:100DE000308047EA080010F0030F14BF00210121F2
:100DF00008F10404381D012E94BF002101F0010107
:100E0000804598BFA74294BF4FF000094FF00109F9
:100E100011EA090F00F01D84BB46D8F80020012319
:100E20006F1EAB42CBF8002007EA030721460246BB
:100E300014D237B1246802230431021DAB4204608E
:100E40000CD20C46104654F8047B40F8047B4968E9
:100E500002335160211D021DAB42F2D3DDF8308018
:100E6000DDF82CB04FEA4C05664508EB05020BEBAC
:100E70000503CCEB06001DD0013832F802CB014649
:100E800023F802CB00F00100A1B128B132F8029B97
:100E9000013923F8029B0DD014461F4634F8029BFB
:100EA00027F8029BB2F802A0A21CA3F802A0BB1C68
:100EB0000239F1D10C9ADDF83CC00B989CF8008007
:100EC000710053180A9E0C93159BCDF84C80451861
:100ED00006EB48020B950E92002B00F0B183002424
:100EE0000025CDE90445CDE9024507930D99134648
:100EF0000A9AB3F804A0B2F806B0CDF804A0B3F88B
:100F000006A00E881588CDF820B0CDF824A0DDE924
:100F100002AB15FB06F51AEB050A4BEBE57BCDE9B9
:100F200002AB1F884888B2F802C0B3F80290B2F84A
:100F300004808C88CDF81880DDE904AB16FB07F639
:100F40001AEB060A4BEBE67BDDE902671CFB00F5BA
:100F5000761910FB09F047EBE5771AEB000A4BEB2B
:100F6000E07BCDE902ABDDF818B0DDF804C0B1F8E4
:100F70000680099D1BFB04F016EB000A47EBE07BA3
:100F8000DDE9026714FB0CF4361947EBE477089CA3
:100F900014FB08F00831083208331AEB000418FB80
:100FA00005F84BEBE075079816EB080A47EBE87B72
:100FB0000138CDE90245CDE904AB079099D1179EE0
:100FC0000E9C0A9B1899A7199A190E97169F002F25
:100FD00073D00E9B31F8020B32F8024B33F8026BE0
:100FE000DDE90289DDE904AB14FB00F47D1E10FB92
:100FF00006F618EB040849EBE4791AEB060A4BEB0A
:10100000E67B2F4605F00100CDE90289CDE904AB6E
:10101000002D52D0002873D031F8024B32F8020B69
:1010200033F8025B10FB04F614FB05F0DDE9024522
:10103000DDE90489A41945EBE67518EB000849EBD6
:10104000E079013FCDE90245CDE9048935D0C246BA
:10105000CB46DDE902890D46144604972146284611
:101060001A4630F8026B31F8027B32F802CB6D88F9
:1010700064885B8817FB06F718EB070816FB0CF66D
:1010800049EBE7791AEB060714FB05FA4BEBE67B15
:1010900015FB03FC8C1C931C0499851C18EB0A0897
:1010A00049EBEA7917EB0C0A4BEBEC7B8A1ECDE996
:1010B00002890492D2D1CDE904AB029D0399049830
:1010C000DDF828A0059BEA0B109D42EA41481299E1
:1010D00008F30F09A5F80090DDF84C90C70B0AEB58
:1010E0008908281D4A1E47EA4346CDF8288006F3A2
:1010F0000F0410906C8012920AD00F9C267866E63E
:10110000DDE904AB0D4614460497DDE90289A5E745
:10111000149F1B9B07EB83061496119F002F00F072
:10112000A681DDF864B0DDF86480DDF834C04FEAF4
:101130009B09CDF81C904FEAC90908F0030A0CEB93
:10114000090BCDF82090CDF810A0CDF824B0DDF833
:101150003CC09CF8006075084FEA450C002D00F07B
:101160007E820C990B980B9F40EA010414F0030F48
:1011700014BF002201220C1D0430012E94BF002256
:1011800002F00102814298BFA74294BF00230123CD
:101190001A4200F06482BA4601230F68691EAB420E
:1011A000CAF80070024601EA0307214614D237B19B
:1011B00027680223211D021DAB4207600CD20C469A
:1011C000104654F8047B40F8047B496802335160B0
:1011D000211D021DAB42F2D3DDF83090DDF82C80EA
:1011E0004FEA4C05664509EB050208EB0503CCEB1D
:1011F00006001DD0013832F802BB014623F802BBBD
:1012000000F00100A1B128B132F8025B013923F8E6
:10121000025B0DD014461F4634F802AB27F802AB30
:10122000B2F802C0A21CA3F802C0BB1C0239F1D163
:10123000DDF82CA0DDF830B0079876000AEB060C3C
:101240000BEB0608CDF82CC0CDF83080002800F05C
:10125000F0810A9ADDF834805788B2F800A0DDF8F2
:1012600028909488B9F80690B8F8062084460D981E
:1012700041880588B8F8040017FB01F61AFB05F34E
:10128000B3461BEB03014FEAE67714FB00F047EB94
:10129000E3750F180A9B19FB02F145EBE0750CF1A1
:1012A000FF3617EB010AB14606F0010008F108020B
:1012B00003F1080345EBE17B002E00F0858048B385
:1012C000DDF834C01E88BCF80840588851889788DB
:1012D0009D88B2F80680B3F806C016FB04F41AEB3A
:1012E000040A10FB01F14BEBE4761AEB010415FB49
:1012F00007FB46EBE17014EB0B011CFB08F640EB1F
:10130000EB740832083311EB060A44EBE67BB9F1C3
:10131000010959D0CDE902ABCB46B3F80080B3F850
:1013200008901688CDF8389018FB06F6DDE902899A
:101330005D88548898889188B2F806C0DF88B2F832
:1013400008A015FB04F418EB060810FB01F149EBAB
:10135000E67918EB040817FB0CF749EBE47918EB76
:10136000010849EBE17918EB070849EBE779CDE98A
:101370000289DDF838905D89548998899189B2F89D
:101380000EC0DE8919FB0AF7DDE9028915FB04F4BA
:1013900018EB070810FB01F149EBE77918EB04089B
:1013A00049EBE47916FB0CF618EB010449EBE17507
:1013B00010321033A01945EBE671BBF1020BCDE9F9
:1013C0000201AAD182468B460DF1200898E816004A
:1013D0006318049D9DB332F802CB33F8026B16FB01
:1013E0000CF4013D1AEB040A294605F001004BEB11
:1013F000E47B25B358B132F8028B33F8020B10FBB3
:1014000008F71AEB070A4BEBE77B691E17D0144667
:10141000184634F8025B30F8027B52885B8817FB71
:1014200005F81AEB08064BEBE87713FB02FBA21C4E
:10143000831C16EB0B0A47EBEB7B0239E7D10F9DC0
:10144000DDF8508095F800C00A9A119E4FEADA3311
:1014500043EA4B4404F30F0028F8020B02EB4C075D
:10146000711E0A97CDF8508011917FF470AE1A9ECC
:101470000F9CB508A06842D00A9F47EA000616F004
:10148000030F07F1080200F1080314BF0021012136
:101490009F4298BF904294BF4FF0000A4FF0010A5C
:1014A00011EA0A0F7FD097E84200016001216C1E0B
:1014B000A942466004EA010419D044B192E812003E
:1014C000196002215C6008320833A9420FD092E80B
:1014D00050001C605E60966802F10804D2689E604D
:1014E0000231DA601033A94204F10802EFD1DDF8CD
:1014F00028A0ED000AEB05094019CDF82890DDF889
:1015000068A01AF003034AD05A085400002A00F0D9
:10151000A480DDF828B040EA0B0515F0030F14BFD6
:10152000002501250BF10406011D012B94BF0025A8
:1015300005F001058B4598BFB04294BF4FF0000CF9
:101540004FF0010C15EA0C0F00F08780DBF800105B
:1015500092009344A3420160CDF828B01044C4EB3C
:1015600003011CD00A9B013933F8024B0A4620F8CC
:10157000024B01F0010192B129B133F8021B013A8B
:1015800020F8021B0BD01C46014634F802CB21F890
:1015900002CB5D88A31C4580881C023AF3D11CB0A5
:1015A000BDE8F00F7047B7F80090A0F800907C8875
:1015B0004480BE888680691EFE880C46B84601F0CD
:1015C0000101C680002C92D091B111881980B2F827
:1015D00002C0A3F802C0B2F804A0A3F804A0B2F8B5
:1015E00006900832A3F806900833013C3FF47FAF21
:1015F00011881980B2F802C0A3F802C0B2F80490B2
:10160000A3F80490B2F806A0A3F806A016891E81DC
:1016100003F1080C5189ACF802109389ACF804303E
:10162000D6891032023C0CF10803ACF80660DFD119
:101630005DE70D9A0A9B4FF0000A4FF0000BC8E6D9
:1016400000260027CDE904670A9A0D99CDE90267C3
:10165000BCE430460B9B0C9A0EE4194682E73046F8
:101660000B9B0C9AC6E500BF00B553EC102B42F261
:10167000FB1223F00043C3F6E972934285B026DDE6
:101680004FF6FF72C7F6EF7293420BDD51EC100B71
:1016900002460B46FDF792FE02460B4643EC102B2A
:1016A00005B000BD684600F0EBFB00F00300012828
:1016B0009DED000B9DED021B1AD0022810D0F8B949
:1016C00000F0FEFE53EC102B10461946E4E79FEDA8
:1016D000101B00F0F5FE53EC102B10461946DBE70B
:1016E00000F0EEFE53EC102B104603F10041D3E75F
:1016F00001F022FC53EC102B104603F10041CBE724
:10170000012001F019FC53EC102B10461946C3E7D9
:1017100000000000000000002DE9F04759EC108B9C
:10172000C9F30A56A6F57E74073C132C4D46CA46EB
:10173000474626DC002C4FDB4FF6FF76C0F20F0643
:1017400046FA04F606EA090555EA080517D044A347
:10175000D3E9002351EC100BFDF732FE00220023E9
:10176000FEF770FA00284AD0B9F1000F6EDB2AEAC2
:10177000060A4FF000085346424643EC102BBDE8E2
:10178000F087332C0CDDB4F5806FF8D151EC100BE1
:101790003A460B46FDF714FE41EC100BBDE8F0870E
:1017A000A6F58265033D4FF0FF3323FA05F515EAF0
:1017B000080FE4D02AA3D3E9002351EC100BFDF766
:1017C000FFFD00220023FEF73DFAC0B1B9F1000F82
:1017D0001CDB28EA050813E021A3D3E9002351EC20
:1017E000100BFDF7EDFD00220023FEF72BFA38B1B8
:1017F000B9F1000F1BDB4FF00008C24600E0CA46FB
:101800005346424643EC102BBDE8F087142C09D018
:10181000C6F5866303334FF0010808FA03F818EBA6
:101820000708D6D30AF1010A28EA0508E8E729F0F3
:10183000004848EA07084FF0000AD045CBF6F07A96
:1018400008BFCA4618BF4FF00008D9E74FF480130D
:1018500043FA04F409EB040A89E700BFAFF3008000
:101860009C7500883CE4377E00B553EC102B42F2A7
:10187000FB1223F00043C3F6E972934285B027DDE3
:101880004FF6FF72C7F6EF7293420BDD51EC100B6F
:1018900002460B46FDF792FD02460B4643EC102B29
:1018A00005B000BD684600F0EBFA00F00300012827
:1018B0009DED000B9DED021B1DD0022812D008BB30
:1018C000012001F039FB53EC102B10461946E3E7D9
:1018D00000209FED111B01F02FFB53EC102B104645
:1018E0001946D9E7012001F027FB53EC102B1046D5
:1018F00003F10041D0E700F0E3FD53EC102B10465C
:101900001946C9E700F0DCFD53EC102B104603F13B
:101910000041C1E7AFF300800000000000000000BC
:1019200010EE103A0BB902207047B3F1004FFAD015
:10193000A3F500016FF00142914201D804207047E5
:1019400003F1FF419142F9D94FF6FE72591EC0F2E0
:101950007F02914201D80320704703F10041013911
:101960009142F8D9B3F1FF4F05D013F5000F14BF22
:101970000020012070470120704700BF00F0E4B84C
:10198000D0B52DED048BB0EE408AF0EE608A3C4C71
:101990008AB000F0D9F994F90030B0EE409AF0EE38
:1019A000609A013335D0B0EE480AF0EE680A01F0D3
:1019B0004DFD00282DD051EC180B00220023FEF71E
:1019C0002DF930B32F4B24780193002308938DED2C
:1019D000028B8DED048B002C23D000270026CFF640
:1019E000F07751EC180B00220023CDE90667FEF7D3
:1019F00001F9002825D002239C42009336D0684686
:101A000001F05CFD002831D0089B002B27D19DED13
:101A1000069BB0EE490AF0EE690A0AB0BDEC048BF1
:101A2000D0BD4FF6FF774FF06046CCF2EF7751EC28
:101A3000180B00220023CDE90667FEF7DBF800282B
:101A4000D9D10123022C009315D0684601F036FD50
:101A500088B10D4801F034FD8DED060BD4E701F09F
:101A6000EDFF089B9DED069B0360D2E701F0E6FFCA
:101A700022230360C8E701F0E1FF21230360E8E7C8
:101A800038040020D0AA050830AD050810B52DEDAA
:101A9000048BB0EE408AF0EE608A294C8AB000F0E8
:101AA0002BFC94F90030B0EE409AF0EE609A0133CE
:101AB0002BD0B0EE480AF0EE680A01F0C7FC20B364
:101AC00051EC180B00220023FEF79EF8E8B11D4BE5
:101AD0002478019301230093002308938DED048B58
:101AE0008DED028BCCB10020002102460B46FDF7A4
:101AF00043FF022CCDE9060115D101F09FFF212300
:101B00000360089BABB99DED069BB0EE490AF0EE71
:101B1000690A0AB0BDEC048B10BD0022002343EC1F
:101B2000172B8DED067B684601F0C8FC0028E8D134
:101B3000E3E701F083FF089B9DED069B0360E4E76C
:101B400038040020D8AA0508F8B5B0EE407AF0EEC7
:101B5000607A53EC112B544210461D46002125F0AB
:101B60000047044353EC102B47EAD474C7F6F071D6
:101B70008C4216463DD85442344323F0004242EA98
:101B8000D4748C4235D805F1404101F580110143F0
:101B90004FD0AC1704F00204164344EAD37435D096
:101BA000384341D00021C7F6F0718F424FD0002159
:101BB000C7F6F0718A4237D0D21B12153C2A42DC9C
:101BC000002D7DDB53EC112B51EC170BFDF7D4FEF0
:101BD00041EC100B01F030FC01F06AFA51EC100BF3
:101BE000012C68D0022C57D0002C48D141EC170BA7
:101BF00007E051EC170B53EC112BFDF7E1FB41EC27
